:020000040800F2
:100000000000022041340108499700084B9700087E
:100010004D9700084F970008519700080000000016
:1000200000000000000000000000000053970008DE
:1000300055970008000000005797000859970008DE
:1000400085340108853401088534010885340108A8
:100050008534010885340108853401088534010898
:10006000853401088534010885340108417A000887
:100070008534010885340108853401088534010878
:100080008534010885340108853401088534010868
:1000900085340108853401088534010889990008F0
:1000A0008534010885340108853401088534010848
:1000B0005599000885340108853401088534010804
:1000C0008534010885340108853401088534010828
:1000D00085340108853401089D9A0008853401089B
:1000E00085340108853401085D97000885340108CE
:1000F00085340108853401088534010885340108F8
:1001000085340108853401088534010885340108E7
:1001100085340108853401088534010885340108D7
:1001200085340108853401088534010885340108C7
:1001300085340108853401088534010885340108B7
:100140008534010885340108853401088D9700083D
:100150008534010885340108853401088534010897
:100160008534010885340108853401088534010887
:100170008534010885340108853401088534010877
:080180008534010885340108F3
:100188003CB8050800000020300C0020300C00208E
:10019800D43C002008B5074B186809F06FFA0EF038
:1001A800EBF8054B054806221A70BDE8084001F037
:1001B800B0BC00BF40260020CD250020A80F00209D
:1001C80008B5034801F0A5FC024B00221A7008BDCF
:1001D800FC170020CD25002008B5054B0122002082
:1001E8001A7005F0EDFE0348BDE8084001F091BC27
:1001F800582C00206C1500202DE9F041144C2046A5
:1002080004F03DF800201349134A03F0EFFD1349A9
:10021800134A0746002003F0E9FD1249124A064630
:10022800002003F0E3FDD22105463A4623460A2082
:1002380003F0F4FED22132462346FA2003F0EEFE04
:100248005A20D2212A462346BDE8F04103F0E6BEF3
:10025800801300206EA40508C901000877A40508CA
:10026800E10100087FA405089D01000808B5054BB9
:10027800012200201A7005F0A3FE0348BDE80840DB
:1002880001F047BC582C00206C15002008B5034825
:1002980001F03FFC024B00221A7008BDFC17002039
:1002A800CD25002008B5054B07221A700EF064F81A
:1002B8000348BDE8084001F02CBC00BFCD25002054
:1002C800801300202DE9F041144C204603F0D7FF9D
:1002D80000201349134A03F089FD1349134A0746BE
:1002E800002003F083FD1249124A0646002003F05D
:1002F8007DFDD22105463A4623460A2003F08EFEAC
:10030800D221324623465A2003F088FEAA20D22161
:100318002A462346BDE8F04103F080BEA80F00201E
:100328006EA405089502000888A40508AD02000817
:1003380091A4050875020008014801F0EABB00BF56
:100348009411002010B5094C204603F098FF0020B6
:100358000749084A03F04AFDD221024623464FF4D2
:100368008270BDE8104003F059BE00BFB4160020EB
:100378009AA405084103000870B50C4C0C4D206880
:100388004FF6E076314603F075F82068294603F009
:100398001FF86068314603F06DF86068294603F07D
:1003A80017F8BDE8704004F0A3B900BF300C002076
:1003B80090AA050838B52B4CFFF7DEFF002005F0A2
:1003C800FFFD237A23B90A203221274A05F006FFC8
:1003D800637A23B90A206421244A05F0FFFE214CE0
:1003E800A37A23B90A209621214A05F0F7FEA37AB9
:1003F8001C4DFBB16B7AEBB12B7ADBB100232B726E
:100408006B72AB721B4B286801221A704FF6E071B1
:1004180003F030F82868184902F0DAFF68681749CD
:1004280002F0D6FF0BF03FFC04F062F9144804F028
:10043800A3F90DE00B4C4FF47841206803F01AF84B
:100448002068104902F0C4FF60680F4902F0C0FF3D
:10045800FFF792FF00200BF0E9FB0C48BDE838409D
:1004680001F057BB300C0020A1A40508AFA4050873
:10047800BEA40508CD250020CCA4050891AA05082E
:1004880080969800E0A4050893AA0508FC170020A8
:1004980008B500200BF0CAFB0248BDE8084001F08F
:1004A80038BB00BFFC17002038B5FFF765FF0DF01B
:1004B8007BFF3C213F220023DF2005F071FE4FF433
:1004C80080600EF0AFFC124C3E223C21DF2000235E
:1004D80005F066FE012323720E4B4FF6E07518688F
:1004E80009F0CCF82068294602F0C4FF20680A49C0
:1004F80002F06EFF6068294602F0BCFF6068074999
:1005080002F066FF04F0F4F8054B00221A7038BDBB
:10051800300C002040260020F2A4050805A5050897
:10052800CD25002038B5FFF727FF0DF03DFF6E21E0
:100538003F220023DF2005F033FE4FF486400EF003
:1005480071FC124C3E226E21DF20002305F028FEAC
:10055800012363720E4B4FF6E075186809F08EF8A8
:100568002068294602F086FF20680A4902F030FF19
:100578006068294602F07EFF6068074902F028FF9C
:1005880004F0B6F8054B00221A7038BD300C002074
:100598004026002018A5050829A50508CD25002016
:1005A80010B5FFF7E9FE0DF0FFFEA0213F22002362
:1005B800DF2005F0F5FD4FF402400EF033FC114C3E
:1005C8003E22A021DF20002305F0EAFD0123A372CB
:1005D8000D4B186809F052F820684FF6E07102F0E8
:1005E80049FF2068094902F0F3FE6068084902F0F3
:1005F800EFFE04F07DF864200BF0E4F9054B0022CF
:100608001A7010BD300C0020402600203AA50508BD
:1006180091AA0508CD2500202DE9F74F3A4D3B4E0C
:100628000024284603F02BFE224623464FF6FF718E
:1006380037480094019402F0E1FE4FF6E078042771
:10064800F06041462246234632480097019402F062
:10065800D5FE23463060414622462F480097019434
:1006680002F0CCFE2D4970602D4A204603F0BEFBF7
:100678002C492D4A0746204603F0B8FB2B492C4A43
:100688008046204603F0B2FB2A492B4A8146204681
:1006980003F0ACFB29492A4A8346204603F0A6FB0F
:1006A80021468246F2682B46204603F0B7FC5A21C1
:1006B80032682B460A2003F0B1FC6E2172682B4683
:1006C8000A2003F0ABFC9B213A462B46FA2003F0A4
:1006D800A5FC692142462B46FA2003F09FFC3721EE
:1006E8004A462B46FA2003F099FCC82152462B466D
:1006F800AA2003F093FCF020C8215A462B4603B0E9
:10070800BDE8F04F03F08ABC24140020300C002010
:100718004EA5050856A5050869A5050878A5050884
:10072800A905000880A505082D05000870A505087D
:10073800B104000888A50508990400088FA50508D4
:10074800BD03000838B50C4C4FF6E0752068294603
:1007580002F090FE2068094902F03AFE60682946D6
:1007680002F088FE6068064902F032FE03F0C0FF1E
:10077800BDE8384003F0BCBF300C002056A5050882
:1007880096A5050870B52DED028B9FED248A88B0DB
:100798000A26F0EE488A03E0B0EE608AF0EE418A5D
:1007A8000CF04FFD8DED000ACDED010A9DE8030028
:1007B80004AB83E80300F0EE680AB0EE480A9DED4A
:1007C800041ADDED051A8DED028ACDED038A0CF0D1
:1007D800D9FACDED010A8DED000A9DE8030002ADBE
:1007E80085E80300013E6C46DDED020A9DED031A23
:1007F800D2D19FED0B0A0CF01BFD8DED000ACDED5B
:10080800010A9DE8030085E80300DDED030A9DED7C
:10081800020A08B0BDEC028B70BD00BF00000000EA
:10082800CDCCCC3D2DE9F74F564D574CDFF86491B0
:10083800DFF864814FF6E07005F096FB286811F048
:1008480003FD064668680F4611F0FEFC3246CDE906
:1008580000013B464946204616F088FB2246002305
:100868000520372105F0BAFC2869484F484E11F099
:10087800EBFC824668698B4611F0E6FC5246CDE9EE
:1008880000015B463946204616F070FB22460023DD
:100898000520692105F0A2FC286B11F0D5FC8246E1
:1008A800686B8B4611F0D0FC5246CDE900015B46DF
:1008B8004146204616F05AFB002305209B2122467C
:1008C80005F08CFC31462A6C204616F04FFB224678
:1008D80000239B21A22005F081FC4FF4FC6005F069
:1008E80043FBA86811F0B0FC8246E8688B4611F01B
:1008F800ABFC5246CDE900015B464946204616F05E
:1009080035FB224605205021002305F067FCA86925
:1009180011F09AFC8246E8698B4611F095FC524624
:10092800CDE900015B463946204616F01FFB2246FA
:1009380000230520822105F051FCA86B11F084FCEE
:100948008246E86B8B4611F07FFC5246CDE90001E8
:100958005B464146204616F009FB00230520B421DA
:10096800224605F03BFC31466A6C204616F0FEFA3A
:10097800A220B4212246002303B0BDE8F04F05F0C1
:100988002DBC00BF603A0020400C0020BBA5050824
:10099800DEA50508A9A50508CDA5050808B5002008
:1009A80005F00EFB0A4B1B780B2B0BD8DFE803F086
:1009B8000A0A0A0A0A0A08060A0A0A0A054802E08E
:1009C800054800E00548BDE8084001F0A2B800BFAE
:1009D800CD25002080130020A80F0020FC17002040
:1009E8002DE9F14F2D4C204603F049FC00202C49FD
:1009F8002C4A03F0FBF92C492C4A8146002003F0CD
:100A0800F5F92B492B4A0746002003F0EFF92A494C
:100A18002A4A0646002003F0E9F92949294A0546E9
:100A2800002003F0E3F92849284A8046002003F013
:100A3800DDF92749274A8246002003F0D7F9D22159
:100A480083464A462346E62003F0E8FA28203A4639
:100A58002346014603F0E2FA46213246234628207F
:100A680003F0DCFA64212A462346282003F0D6FA4C
:100A7800822142462346282003F0D0FA52462346D4
:100A88002820A02103F0CAFA28205A46BE2123466E
:100A980001B0BDE8F04F03F0C1BA00BF6C150020EB
:100AA800E3A50508A5090008ECA505083514000804
:100AB800F7A505081114000801A60508ED1300089C
:100AC8000CA60508C913000817A60508A5130008F1
:100AD80021A6050881130008023810B50A2800F27B
:100AE8003484DFE810F00B000F00D0003A01250233
:100AF800BB01D002EA0232049903ED03BDE81040BD
:100B08000BF03EB900204FF6E0710BF08FFA64202D
:100B18004FF6E0710BF08AFAC8204FF6E0710BF03F
:100B280085FA4FF6FF7005F01FFA00237D20DC21BF
:100B3800B14A05F053FB4EF29C7005F015FAAF4B25
:100B48001C78022C32D0052C6CD0012C40F0FD838F
:100B5800B4204FF4F0610BF069FA05202146A84A49
:100B6800002305F03BFB05205221A64A002305F08F
:100B780035FBB621A44A0023052005F02FFB4FF4CE
:100B8800F06005F0F1F940F2131021469C4A002369
:100B980005F024FB40F2131052219B4A002305F074
:100BA8001DFB40F21310B621984A2CE0A0204FF408
:100BB800F0610BF03BFA05200121924A002305F071
:100BC8000DFB05205221924A002305F007FBB621B0
:100BD8008D4A0023052005F001FB4FF4F06005F075
:100BE800C3F940F213100121864A002305F0F6FAF2
:100BF80040F213105221844A002305F0EFFA854A87
:100C080040F21310B621002305F0E8FA4EF29C706A
:100C180005F0AAF90520A2217F4A0023BDE810406B
:100C280005F0DCBA64204FF4F0610BF0FFF92046C0
:100C380001217A4A002305F0D1FAB621724A00232D
:100C4800204605F0CBFA4FF4F06005F08DF940F23C
:100C580013100121714A002305F0C0FA40F2131065
:100C68005221694A002305F0B9FAB62140F213105F
:100C78006B4A002305F0B2FA4EF29C7005F074F945
:100C880020465221C8E700204FF6E0710BF0CEF95C
:100C980031204FF6E0710BF0C9F963204FF6E0718F
:100CA8000BF0C4F995204FF6E0710BF0BFF9C7209F
:100CB8004FF6E0710BF0BAF94EF29C7005F054F95A
:100CC800052001210023574A05F088FA0520202134
:100CD8000023554A05F082FA052052210023534A81
:100CE80005F07CFA052084210023514A05F076FAA4
:100CF800B6210520444A002305F070FA4FF4F0604D
:100D080005F032F9012140F213100023454A05F09D
:100D180065FA40F213102021464A002305F05EFAD6
:100D280040F213105221384A002305F057FA40F2D6
:100D380013108421404A002305F050FAB6213F4A97
:100D480040F21310002305F049FA4FF6FF7005F042
:100D58000BF97D20DC213A4A5FE700204FF6E0716D
:100D68000BF064F927204FF6E0710BF05FF94F2084
:100D78004FF6E0710BF05AF977204FF6E0710BF05F
:100D880055F99F204FF6E0710BF050F9C7204FF648
:100D9800E0710BF04BF94EF29C7005F0E5F8052078
:100DA80001210023184A05F019FA0520162100230D
:100DB800244A05F013FA05203E210023224A05F0B3
:100DC8000DFA052066210023204A05F007FA8E2136
:100DD800002305201E4A05F001FA05201D4AB62108
:100DE800002305F0FBF94FF6FF7005F0BDF87D20F4
:100DF800DC21194A11E700BFF7A505081C030020EC
:100E080027A6050830A60508FBAB050826A6050891
:100E18002BA605082FA6050862A6050835A605080D
:100E280034A605084EA6050839A6050849A60508EA
:100E38003EA6050843A6050848A605084DA60508C8
:100E480001A6050851A6050855A6050859A60508CE
:100E58005DA6050861A6050865A6050800204FF6E9
:100E6800E0710BF0E3F831204FF6E0710BF0DEF89B
:100E780063204FF6E0710BF0D9F895204FF6E0713A
:100E88000BF0D4F8C7204FF6E0710BF0CFF84EF214
:100E98009C7005F069F8052001210023BF4A05F080
:100EA8009DF9052020210023BD4A05F097F905206A
:100EB80052210023BB4A05F091F905208421002323
:100EC800B94A05F08BF9B6210520B84A002305F088
:100ED80085F94FF4F06005F047F8012140F213104E
:100EE8000023B34A05F07AF940F213102021B14AE1
:100EF800002305F073F940F213105221AB4A002386
:100F080005F06CF940F213108421AB4A002305F078
:100F180065F9B621A94A40F21310002305F05EF9DD
:100F28004FF6FF7005F020F87D20DC21A44A74E616
:100F3800A44B1C78022C32D0052C5DD0012C40F03B
:100F48008B8000204FF6E0710BF070F834204FF6DC
:100F5800E0710BF06BF864204FF6E0710BF066F867
:100F68004FF6E07198200BF061F84EF29C7004F097
:100F7800FBFF05202146944A002305F02FF90520A0
:100F88002021924A002305F029F905205021904A92
:100F9800002305F023F9052084218E4A59E000201A
:100FA8004FF6E0710BF042F852204FF6E0710BF06B
:100FB8003DF890204FF6E0710BF038F84FF6E071ED
:100FC800B4200BF033F84EF29C7004F0CDFF0520EE
:100FD8000121814A002305F001F905203E217C4AC0
:100FE800002305F0FBF805207C217A4A002305F050
:100FF800F5F80520A0212BE000204FF6E0710BF05A
:1010080015F82E204FF6E0710BF010F87F204FF600
:10101800E0710BF00BF84FF6E071AD200BF006F81D
:101028004EF29C7004F0A0FF204601216B4A002379
:1010380005F0D4F820463221654A002305F0CEF8A1
:1010480020466B21634A002305F0C8F82046992101
:10105800634A002305F0C2F84FF4F06004F084FFFF
:10106800604A00230520B62105F0B8F84FF4FC616A
:10107800C8200AF0DBFF4FF6FF7004F075FF8720E9
:10108800DC21594AC9E500204FF6E0710AF0CEFF8D
:1010980063204FF4FC610AF0C9FF4FF6E071C720E6
:1010A8000AF0C4FF4FF6FF7004F05EFF002005F061
:1010B8005DF8A520D7214D4AAFE5042005F056F884
:1010C80000204FF6E0710AF0B1FF31204FF6E071D1
:1010D8000AF0ACFF63204FF6E0710AF0A7FF9520F5
:1010E8004FF6E0710AF0A2FFC7204FF6E0710AF050
:1010F8009DFF4EF29C7004F037FF0520012100236C
:101108003B4A05F06BF8052020210023314A05F001
:1011180065F8052052210023364A05F05FF80520BE
:1011280084210023344A05F059F80520B621334AB2
:10113800002305F053F84FF6E07004F015FF40F275
:101148000B1001212E4A002305F048F840F22B101D
:1011580020212C4A002305F041F840F223105221A7
:10116800294A002305F03AF840F21B108421274A47
:10117800002305F033F8B621254A002340F2131066
:1011880005F02CF84FF6FF7004F0EEFE002004F096
:10119800EDFF6E20D2211F4ACFE000BF71A60508DF
:1011A80075A6050892A6050879A60508FBAB0508EB
:1011B80082A605087EA605087DA6050881A605085D
:1011C80086A605081C03002035A605085AA60508AA
:1011D80052A60508A1A6050862A6050856A6050890
:1011E80091A6050812AD050821A60508A9AA0508B3
:1011F80095A60508A0A60508A3A60508A7A605089C
:10120800ACA605084EA60508B3A60508B7A60508A6
:10121800BCA60508C2A60508042004F0A7FF002004
:101228004FF6E0710AF002FF27204FF6E0710AF04E
:10123800FDFE4F204FF6E0710AF0F8FE77204FF6DA
:10124800E0710AF0F3FE9F204FF6E0710AF0EEFE1F
:10125800C7204FF6E0710AF0E9FE4EF29C7004F0E8
:1012680083FE052001210023384A04F0B7FF05203A
:1012780016210023364A04F0B1FF05203E21002341
:10128800344A04F0ABFF05206621334A002304F0FA
:10129800A5FF05208E21314A002304F09FFFB621C7
:1012A8002F4A0023052004F099FF4FF6FF7004F041
:1012B8005BFE002004F05AFF6420D221294A3CE05A
:1012C800042004F053FF00204FF6E0710AF0AEFE50
:1012D80043204FF6E0710AF0A9FE85204FF6E07131
:1012E8000AF0A4FE4FF6E071C7200AF09FFE4EF206
:1012F8009C7004F039FE052001211B4A002304F0EC
:101308006DFF05204521194A002304F067FF0520D9
:101318008721134A002304F061FFB621144A0023F1
:10132800052004F05BFF4FF6FF7004F01DFE00205F
:1013380004F01CFF0F4A7D20D221002304F04EFF49
:101348000420BDE8104004F011BF10BDC8A6050870
:101358007EA6050883A60508CDA60508D0A605081B
:1013680062A60508D3A60508DCA6050835A6050863
:10137800FBAB05086FAB050810B5064C06480623FD
:10138800237000F0C6FB2078FFF7A6FBBDE81040ED
:101398000DF016BD582C00205817002010B5064C2B
:1013A80006480723237000F0B4FB2078FFF794FB6E
:1013B800BDE810400DF004BD582C0020581700203F
:1013C80010B5064C06480523237000F0A2FB2078D0
:1013D800FFF782FBBDE810400DF0F2BC582C00204E
:1013E8005817002010B5064C06480423237000F057
:1013F80090FB2078FFF770FBBDE810400DF0E0BCD3
:10140800582C00205817002010B5064C0648032316
:10141800237000F07EFB2078FFF75EFBBDE81040EC
:101428000DF0CEBC582C00205817002010B5064CE3
:1014380006480223237000F06CFB2078FFF74CFB72
:10144800BDE810400DF0BCBC582C002058170020F7
:1014580038B5094C05464FF6E071206802F00AF8E5
:1014680020680DB1054900E0054901F0B1FFBDE86C
:10147800384003F03DB900BF5C0C0020E0A6050829
:10148800F3A60508194B10B51C78012C05D006D316
:10149800022C0CBF3024002402E0002400E01024B9
:1014A80004F1C80006F01EFB11490246114815F068
:1014B8005DFD04F1CC0006F015FB0D4902460E480F
:1014C80015F054FD04F1D00006F00CFB0849024663
:1014D8000A4815F04BFD04F1D40006F003FB04495B
:1014E80002460748BDE8104015F040BD1C0E00201C
:1014F800DEA5050810260020342600204A2C0020EE
:10150800FC25002010B5E82006F0ECFA0F4C024646
:1015180021460F4815F02AFDEC2006F0E3FA214693
:1015280002460C4815F022FDF02006F0DBFA2146B1
:101538000246094815F01AFDF42006F0D3FA0246CF
:1015480006482146BDE8104015F010BDDEA5050887
:1015580010260020342600204A2C0020FC250020DC
:101568000E4A012310B513700D4A002414700D4A59
:10157800204613700AF05AFB204604F021FD0A4B5E
:1015880003221A700AF0B0FE0BF0F5FB074B08486F
:101598001C70BDE8104000F0BCBA00BF582C0020F9
:1015A800770D0020750D0020CD250020343800204F
:1015B8003812002038B50D4B0D4D00241C700D4B12
:1015C80028681C700C4B4FF6E0711C7001F052FF3C
:1015D80028680A4901F0FCFE03F08AF8204604F066
:1015E800EFFC0748BDE8384000F093BAD40D00205E
:1015F8005C0C0020770D0020CD25002095AA050859
:10160800FC17002007B50E4B0E481A78D2F10102DC
:1016180038BF00221A700C4B05221A7000F079FAB4
:10162800022201238DE80C00B02060211022322311
:101638000DF06AFD03B05DF804EB03F059B800BF84
:10164800D40D0020F0100020CD2500202E4A0023C4
:1016580010B513702D4A13700DF0AAF9044600282E
:1016680042D02B4C4FF6E071206801F003FF206850
:10167800284901F0ADFE60684FF6E07101F0FAFE0E
:101688006068254901F0A4FEA0684FF6E07101F0FA
:10169800F1FEA068214901F09BFE03F029F84FF400
:1016A8007A600AF08FF920684FF6E07101F0E2FEE7
:1016B80020681B4901F08CFE60684FF6E07101F06C
:1016C800D9FE6068164901F083FEA0684FF6E07104
:1016D80001F0D0FEA068124901F07AFE03F008F884
:1016E800BDE8104003F004B80CF046FE204604F0B4
:1016F80067FC0C4B0C4804221A7000F00AFABDE88B
:101708001040FFF71FB800BFD40D0020770D002050
:101718005C0C002006A705081AA705082AA70508D3
:1017280094AA0508CD250020241400202DE9F04FA7
:101738006A4DDFF8F4916A4E85B000244FF6FF78C1
:10174800284602F09CFD41462246234665480094FF
:10175800019401F053FE0427039041462246234694
:1017680048460097019401F049FE41463060224600
:10177800234648460097019401F040FE41467060B8
:101788002246234648460097019401F037FEA8F503
:101798000048B060414622462346534800970194CA
:1017A80001F02CFE4146F060224623464F48009740
:1017B800019401F023FE41463061224623464C48FD
:1017C8000097019401F01AFE2346706141462246B3
:1017D80048480097019401F011FE4749B061474A13
:1017E800204602F003FB4649464A8046204602F05E
:1017F800FDFA4549454A8246204602F0F7FA44492F
:10180800444A0746204602F0F1FA4349434A8146D2
:10181800204602F0EBFA4249424A8346204602F04B
:10182800E5FA21468446039ACDF808C02B4620469F
:1018380002F0F4FB052132682B46A02002F0EEFBF3
:10184800692172682B46782002F0E8FB7D21B26896
:101858002B46782002F0E2FB2821F2682B4605206F
:1018680002F0DCFB4B2132692B46052002F0D6FB47
:10187800052072696E212B4602F0D0FB9121B269D6
:101888002B46052002F0CAFBD2213A462B460520FA
:1018980002F0C4FBD22142462B46602002F0BEFB78
:1018A800D2214A462B46B02002F0B8FBD22152463C
:1018B8002B464FF4807002F0B1FBB4215A462B46F8
:1018C800052002F0ABFBDDF808C06020B4216246B9
:1018D8002B4605B0BDE8F04F02F0A0BBC8140020AD
:1018E8005C0C00203AA7050844A705084BA7050883
:1018F80051A7050857A705085DA70508551600084C
:1019080065A70508BD1500086DA705080D16000890
:1019180076A70508691500087EA705080D150008B3
:1019280087A705088D14000891AA05085B4B2DE9C7
:10193800F04100251D705A4B1D705A4B01221A7038
:10194800594B1B789342044605D003D3022B08BF9A
:10195800302500E01025012C03D0022C40F09780A0
:101968001FE021464FF4747006F0A3F80AF0E2FB7A
:10197800204605F073FA2046FFF76AFD4A4B1978AE
:10198800012907D003D3022940F0818005E04020D7
:10199800002103E04020214600E0402007F07CFAC7
:1019A80075E005F1C80006F09DF8044605F1CC0085
:1019B80006F098F8074605F1D00006F093F80646B9
:1019C80005F1D40006F08EF805460AF0B3FB374B54
:1019D80037491A68A242184602DB0B68BB4212DD7F
:1019E800344B04601E60344B0F601D600AF0DEF853
:1019F8002C4B01221A70314A0520B4210023BDE87E
:101A0800F04104F0EBBB944218D19F4216D1294B08
:101A18001B689E4212D1284B1B689D420ED1214B58
:101A2800012119704FF4747006F043F8244B00221A
:101A38001A60244B4FF07E521A6028E0194B022599
:101A48001D7029464FF4747006F033F8174B1B6865
:101A580006EE906A1C1BF8EEE67A06EE904AB8EE9F
:101A6800E67A174B87EE277A284683ED007A114BE2
:101A78001B6806EE903AB8EEE67A124BC7EE277A64
:101A8800C3ED007A05F0EAF90020FFF7E1FC0AF05F
:101A9800ECFABDE8F04102F02BBE00BFD40D0020E7
:101AA800770D0020C90100201C0E00204C260020C4
:101AB800642C0020402C0020F825002090A7050861
:101AC800C82500200826002008B500F053FFFEF7BF
:101AD80093FB00F04FF800F06FF8FEF79DFDFEF75E
:101AE800F1FBFEF77DFF01F055FBFFF71FFE01F04C
:101AF80027F9FEF727FC01F049FA00F073FB00F024
:101B080087FD00F091FE00F065FABDE8084000F09E
:101B180033BB10B5044628B90F48104A104B53215F
:101B280003F00EF80F4B1868844213D010B1C36944
:101B380000219847002004F043FA002004F02AFA14
:101B48004FF6FF7004F010FAE36920460121984728
:101B5800044B1C6010BD00BFA4A705085C25040841
:101B6800C0A70508780C00200048D2E7FC17002021
:101B78000CF0DEBE10B5084C204602F080FB0020B9
:101B88000649074A02F032F9D22102462346FA20D2
:101B9800BDE8104002F042BA600E0020DEA705083A
:101BA800791B0008024B034801221A70FFF7B1BFE6
:101BB800CD250020C81400202DE9F743374D384FB4
:101BC800384E0024284602F05AFB2246234647F6A0
:101BD800FF7135480094019401F010FC4FF6FF782E
:101BE800814641462246234638460094019401F036
:101BF80005FC41463060224623463846009401944D
:101C080001F0FCFB414670602246234638460094AA
:101C1800019401F0F3FB2346B06041462246384662
:101C28000094019401F0EAFB2049F060204A204624
:101C380002F0DCF81F49204A0746204602F0D6F891
:101C4800214680464A462B46204602F0E7F93C21C9
:101C580032682B46192002F0E1F95A2172682B46A6
:101C6800192002F0DBF97821B2682B46192002F01E
:101C7800D5F99621F2682B46192002F0CFF9D22126
:101C88003A462B46EC2002F0C9F99C20D221424664
:101C98002B4603B0BDE8F04302F0C0B9381200206B
:101CA80091AA05087C0C0020D0A70508DDA7050827
:101CB800AD1B0008E6A70508891E000870B5474E49
:101CC800474C327847492DED028B142592B005FB1D
:101CD80002420C320FA815F049F933780E2B05FB98
:101CE80003F504EB050332D8D3ED016A9B6807EED0
:101CF800103A6359B8EEE68A06EE903ADFED3A7A82
:101D0800F8EEC78AB8EEE67A88EE278AC8EEA78A80
:101D1800C7EE277A17EE900A10F096FA02460B469D
:101D28006846324915F022F918EE100A10F08CFABC
:101D380002460B4605A82E4915F018F918EE900A28
:101D480010F082FA02460B460AA82A4929E093EDC8
:101D5800017A9B6807EE903A635906EE903AF8EEDE
:101D6800E78AF8EEE67AB8EEC78A17EE900A10F01E
:101D78006BFA02460B4668461F4915F0F7F818EE4D
:101D8800100A10F061FA02460B4605A81B4915F027
:101D9800EDF818EE900A10F057FA0B46184902466B
:101DA8000AA8184C15F0E2F82068174901F010FB52
:101DB80020680FA901F00CFB6068694601F008FB78
:101DC800A06805A901F004FBE0680AA901F000FB7E
:101DD80002F08EFC12B0BDEC028B70BD46260020CE
:101DE80000000020EFA7050800007A44FAA70508BC
:101DF8000BA805081CA805082DA805083EA8050875
:101E08004FA805087C0C00209AAA050808B5144BB1
:101E1800144A1B780D2B01D8012104E00E2B01D1A7
:101E2800022100E000211170142253430E49C858C2
:101E3800CA184FF47A730D4958430860516892687C
:101E48004B430B490B600B4B1A6009F0AFFE0A4B72
:101E58000A4801221A70BDE80840FFF75ABE00BFC1
:101E6800462600201C0E0020000000204C260020E2
:101E7800642C0020402C0020CD250020C814002010
:101E8800C4E700BF4FF6FF7070474FF6FF7070470A
:101E98001FB5002947D04FF2DE7004F091F80020FA
:101EA80004F064F90F2004F05FF81F4C1F4A412129
:101EB80001230A2004F092F9042004F057F923685A
:101EC80028209621042B24DC0123194A04F086F9E2
:101ED80003A90DF10E02206804F006FC0F2004F09F
:101EE80043F8BDF80C00BDF80E1014380F24282252
:101EF800002380B2009404F067F8BDF80E10BDF816
:101F08000C000094143989B22822012304F05CF8EB
:101F180009E0084A012304F061F91E20A521064AB8
:101F2800012304F05BF91FBD8C0C002060A8050894
:101F380073A805088FA80508A5A8050837B51E4C7D
:101F48002368042B05462BDC01A80DF1060104F0DB
:101F5800C9FBBDF80630BDF80420184904200DF06F
:101F680027FA2368002B04DA1548164A164B59211C
:101F780005E0042B05DD1248124A144B5A2102F0E1
:101F8800DFFD04EB8302BDF8041001339180BDF836
:101F980006102360052BD18008D1201D04F024FCF5
:101FA80000230B482360FFF7B4FD03E02846012116
:101FB800FFF76EFF3EBD00BF8C0C0020BCA80508D3
:101FC80001A905086E25040823A905083AA90508EA
:101FD8001016002037B50B4C204602F050F90A4B7A
:101FE8000A49009300250120094A0A4B019501F08E
:101FF800EEFF294602462346284603B0BDE8304096
:1020080002F00CB8DC120020991E00088D1E000892
:10201800931E0008451F00084FF6FF7070474FF6E3
:10202800FF70704730B54FF6E07087B003F0C8FF17
:10203800002004F09BF80F2003F096FF00212C4AA3
:102048002C4C01230A2004F0C9F8002003F08CFF6F
:10205800042004F08BF80A201921274A012304F0F0
:10206800BDF82521254A01230A2004F0B7F81F20CE
:1020780003F07AFF01230A203721214A04F0AEF841
:102088002378002B31D001231E2096211D4A04F00D
:10209800A5F862881C4902A814F068FF01231E20D5
:1020A800A22102AA04F09AF8A288184902A814F0FA
:1020B8005DFFAE2102AA01231E2004F08FF80F2035
:1020C80003F052FF6088A188143880B20F252822B7
:1020D8000023009503F078FFA188608800951439E3
:1020E80089B22822012303F06FFF07B030BD00BF7B
:1020F80068A90508A40C00207AA905089AA905086A
:10210800BAA90508DDA90508EFA90508FCA905086D
:1021180001B187E7704713B50DF1060101A804F076
:1021280095FA144B01221A705988BDF80420891AAF
:102138000E311C2919460AD89C88BDF80600201AB9
:102148000E301C2803D899680131996001E00023FA
:102158008B60084B9968012905DD00229A601A7086
:10216800FFF702FD05E05A80BDF806209A80FFF7C8
:1021780059FF1CBDA40C002037B50B4C204602F0BB
:102188007EF80A4B0A49009300250120094A0A4BA8
:10219800019501F01CFF294602462346284603B054
:1021A800BDE8304001F03ABF1016002019210008A0
:1021B80021200008272000081F21000808B5064B29
:1021C80000221A70054B186814F066FB0448BDE835
:1021D8000840FFF79EBC00BFCD2500202036002018
:1021E800FC1700202DE9F04F514D524E85B00024C8
:1021F800284602F044F82246234647F6FF714E4827
:102208000094019401F0FAF84FF6FF7703903946ED
:102218002246234649480094019401F0EFF83946D4
:1022280030602246234646480094019401F0E6F8BF
:102238004FF001087060224623464FF6E07141488E
:10224800CDF80080019401F0D9F82346B0603946F2
:1022580022463D48CDF80080019401F0CFF83B4973
:10226800F0603B4A204601F0C1FD3A493A4A074628
:10227800204601F0BBFD3949394A8046204601F025
:10228800B5FD3849384A8146204601F0AFFD374947
:10229800374A8246204601F0A9FD3649364A834628
:1022A800204601F0A3FD21468446039ACDF808C0D4
:1022B8002B46204601F0B2FE3C2132682B46142002
:1022C80001F0ACFE3C2172682B46EC2001F0A6FE22
:1022D800B421B2682B460F2001F0A0FED2213A4665
:1022E8002B46E62001F09AFE642142462B46052043
:1022F80001F094FE4A462B460520872101F08EFE08
:1023080052462B460520D22101F088FED2215A469A
:102318002B46502001F082FEDDF808C09B20D22118
:1023280062462B4605B0BDE8F04F01F077BE00BF0E
:10233800040F0020B00C002009AA050813AA0508FC
:102348008DA705088FAA050891AA0508DDA7050825
:10235800C521000870A50508AD23000880A505085B
:10236800AD2400081CAA0508B525000824AA0508FC
:10237800712500082CAA05082D25000808B50CF0C1
:1023880013F84FF441400CF04DFD044B186807F06A
:1023980075F9034B09221A7008BD00BF40260020BA
:1023A800CD25002010B50C4CFFF7E8FF0B4A0023A1
:1023B800B420052103F012FFA0684FF6E07101F088
:1023C80059F8A068064901F003F80BF0EDFFBDE8E5
:1023D800104002F08DB900BFB00C002097AA050884
:1023E80034AA0508264B2DE9F7431888C00014F0D5
:1023F8004BFA054628B90520B421224A2B4603F09A
:10240800EDFE214BDFF878801D6000240BF0CCFF37
:1024180026461E4FDFF8889023E009F005FA3B684E
:10242800D9F8000045F8083C7B6845F8043C184B8F
:102438001B68C01807F022F9164B186809F0C2FA91
:10244800B8F8000094FBF0F080B24FF4FC630093FE
:1024580028210246322303F013FD04F59E74013649
:102468000334B8F800300835B342D6DA0A4B186896
:1024780007F004F9094B09221A70BDE8FE8300BF72
:102488002C3A00204DAA050820360020EC37002001
:10249800C4250020F825002040260020CD25002056
:1024A8002836002010B5094CFFF79CFFA0684FF6AE
:1024B800E07100F0DFFFA068054900F089FF0BF02C
:1024C80073FFBDE8104002F013B900BFB00C002044
:1024D8005BAA050810B5074C4FF6E071A06800F03C
:1024E800C9FFA068044900F073FFBDE8104002F07E
:1024F800FFB800BFB00C002075AA050810B5074C3E
:102508004FF6E071A06800F0B5FFA068044900F03C
:102518005FFFBDE8104002F0EBB800BFB00C002030
:102528008BAA050810B50C4C0B2323700B4B01220A
:102538001A70002003F012F80948FFF7EAFA207829
:10254800FEF7CAFA074B032093ED000A0BF03BFF96
:10255800BDE81040D2E700BF582C0020780D0020BD
:10256800581700202403002038B50C4D0C232B707D
:102578000B4B01241C70002002F0F0FF0948FFF704
:10258800C8FA2878FEF7A8FA074B204693ED000A08
:102598000BF019FFBDE83840B0E700BF582C002009
:1025A800780D0020581700202403002010B50C4C8B
:1025B800092323700B4B01221A70002002F0CEFF72
:1025C8000948FFF7A6FA2078FEF786FA074B02209B
:1025D80093ED000A0BF0F7FEBDE810408EE700BF50
:1025E800582C0020780D00205817002024030020C4
:1025F8000CF064BA034A044800231370034A1370AA
:10260800FFF787BA34380020FC170020CD250020BA
:102618002DE9F743384D394EDFF8FC800024284671
:1026280001F02DFE2246234647F6FF7134480094F8
:10263800019400F0E3FE4FF6FF77814639462246C3
:10264800234630480094019400F0D8FE39463060A3
:102658002246234640460094019400F0CFFE3946B6
:1026680070602246234640460094019400F0C6FE5E
:102678002346B0603946224640460094019400F053
:10268800BDFE2149F060214A204601F0AFFB2049F8
:10269800204A0746204601F0A9FB214680464A46C3
:1026A8002B46204601F0BAFC3C2132682B462820F4
:1026B80001F0B4FC5A2172682B46192001F0AEFCD7
:1026C8007821B2682B46192001F0A8FC9621F268FF
:1026D8002B46192001F0A2FCD2213A462B46EC20C9
:1026E80001F09CFC0520D22142462B4603B0BDE8F0
:1026F800F04301F093BC00BF4C100020C00C002038
:10270800A5AA0508ADAA0508DDA70508FD25000846
:10271800B8AA0508F925000891AA050870B5064663
:1027280000200D46144603F021FD4FF6FF7003F01C
:102738001BFCF2B273208621002303F031FDEAB2BC
:102748007320AE21002303F02BFDE2B27320D621C3
:102758000023BDE8704003F023BD08B5084B2020D6
:102768001860084B1860084B58221A600146FFF79A
:10277800D5FF0648064B1860BDE8084006F07EBF46
:10278800D8010020D4010020D0010020C0E1E400DD
:10279800EC25002008B5094B20201860084B58216B
:1027A8001960084B02461860FFF7B8FF0648074B48
:1027B8001860BDE8084006F061BF00BFD8010020DE
:1027C800D4010020D001002080969800EC2500203C
:1027D80008B5094B58201860084B20211960084B90
:1027E8000A461960FFF79AFF0648074B1860BDE8CC
:1027F800084006F043BF00BFD8010020D4010020E4
:10280800D0010020404B4C00EC250020034A04482E
:1028180000231370034A1370FFF77BB93438002084
:10282800FC170020CD2500202DE9F74F444D454EDB
:10283800DFF83C810024284601F021FD224623468A
:1028480047F6FF7140480094019400F0D7FD4FF619
:10285800FF7783463946224623463C480094019434
:1028680000F0CCFD394630602246234640460094AD
:10287800019400F0C3FD3946706022462346404665
:102888000094019400F0BAFD2346B0603946224610
:1028980040460094019400F0B1FD2D49F0602D4AA6
:1028A800204601F0A3FA2C492C4A0746204601F09D
:1028B8009DFA2B492B4A8046204601F097FA2A496F
:1028C8002A4A8146204601F091FA214682465A4614
:1028D8002B46204601F0A2FB3C2132682B461920EA
:1028E80001F09CFB5A2172682B46192001F096FBD7
:1028F8007821B2682B46192001F090FB9621F268E6
:102908002B46192001F08AFBD2213A462B46EC20AF
:1029180001F084FB822142462B46192001F07EFB00
:10292800AA214A462B46192001F078FB1920524665
:10293800D2212B4603B0BDE8F04F01F06FBB00BFBA
:10294800A0180020D00C0020C0AA0508CEAA0508AF
:10295800DDA7050815280008DBAA0508D9270008FF
:10296800E4AA05089D270008EDAA050863270008C2
:1029780091AA050810B50B4C204601F080FC0020F8
:102988000146224600F09AFD00200749074A01F057
:102998002DFAD221024623464FF48270BDE810403A
:1029A80001F03CBB58170020F6AA0508DD290008ED
:1029B80070B5C9240AE0A8B200223146013502F0F8
:1029C8005DFCF02DF7D10134EF2C02D00025A6B222
:1029D800F1E770BD10B51A4C2378092B08D1194AB4
:1029E80000231370184A1370FFF7E2FF174823E01B
:1029F8000A2B0ED1164B186813F04EFF154A002308
:102A08001370114A1370144A1370FFF7D1FF13485B
:102A180012E0002002F0A2FD114A00231360114ABF
:102A280013800D4B02221A700F4B186806F026FE11
:102A380022780E4B0E481A70BDE81040FFF769B8AF
:102A4800CD250020780D0020770D0020040F0020F0
:102A580020360020790D0020343800204C1000204A
:102A6800C40D0020D20D002040260020EA250020B9
:102A780094110020034B01224FF4FC601A7003F0FC
:102A880073BA00BF770D0020044B054800221A7066
:102A9800044B0C221A70FFF73CB800BF770D0020DA
:102AA800A0180020CD25002007B50A4A002313707E
:102AB80004228DE80C00C6201022232356210CF096
:102AC80023FB054B05480A221A7003B05DF804EB96
:102AD800FFF71FB8770D0020CD2500204C100020EF
:102AE80007B50A4A0023137004228DE80C009720CA
:102AF8001022232356210CF007FB054B0548092219
:102B08001A7003B05DF804EBFFF703B8770D0020E7
:102B1800CD250020040F002007B50B4B00221A70AA
:102B2800082203238DE80C004920102223233D218D
:102B38000CF0EAFA054B064801221A7003B05DF85A
:102B480004EBFEF7E6BF00BF770D0020CD2500207F
:102B5800C814002008B501214FF080400EF023FC76
:102B68000A4B002018700A4B18700A4B18700A4B51
:102B780008221A70094B187003F022FA084B09480A
:102B880001221A70BDE80840FEF7C3BFF0250020F7
:102B9800D40D0020770D0020CD250020582C0020D2
:102BA80038360020600E002070B51F4C1F4E20687C
:102BB8004FF6E075294600F05DFC20681C4900F0DE
:102BC80007FC6068294600F055FC6068194900F068
:102BD800FFFBA068294600F04DFCA068164900F0EC
:102BE800F7FB01F085FD4FF47A6008F0EBFE2068F2
:102BF800294600F03FFC2068314600F0E9FB606898
:102C0800294600F037FC6068314600F0E1FBA06817
:102C1800294600F02FFCA068314600F0D9FBBDE83A
:102C2800704001F065BD00BFE00C002094AA0508C3
:102C380006A705081AA705082AA705080C4B10B50A
:102C480000241C700B4B01221A70204608F0EEFF7E
:102C5800204603F0B5F9084B0B221A7009F044FB23
:102C68000AF089F80548BDE81040FEF752BF00BFDA
:102C7800770D0020582C0020CD2500206C15002051
:102C88000F4A002310B513700E4A13700BF090FE14
:102C9800044628B1FFF788FFBDE8104001F028BDC1
:102CA80003F08EF909F046FA074B1C70074B072210
:102CB8001A7009F039FA0648BDE81040FEF729BF36
:102CC800D40D0020770D0020582C0020CD250020A1
:102CD8008013002010B54FF0804001210EF063FBF7
:102CE800114A00231370114A1370114A13700BF024
:102CF8005FFE044628B1FFF757FFBDE8104001F01A
:102D0800F7BC03F05DF909F015FA06F013FD094B5D
:102D18001C70094B06221A7009F006FA0748BDE82C
:102D28001040FEF7F6BE00BFF0250020D40D0020AD
:102D3800770D0020582C0020CD250020A80F00205A
:102D48002DE9F04F6D4DDFF810928BB000244FF64F
:102D5800FF78284601F093FA414622462346684800
:102D68000094019400F04AFB4FF6E07604270490A3
:102D780031462246234663480097019400F03EFB03
:102D880031460590224623465F480097019400F09B
:102D980035FB414606902246234648460097019453
:102DA80000F02CFB594E41463060224623464846E7
:102DB8000097019400F022FB2346706041462246AA
:102DC80048460097019400F019FB5149B060514AF8
:102DD800204601F00BF85049504A0746204601F0BA
:102DE80005F84F494F4A8046204600F0FFFF4E49FC
:102DF8004E4A8146204600F0F9FF4D494D4A824629
:102E0800204600F0F3FF4C494C4A8346204600F028
:102E1800EDFF4B494B4A84462046CDF80CC000F0E4
:102E2800E5FF49490790494A204600F0DFFF484935
:102E38000890484A204600F0D9FF21460990049A94
:102E48002B46204601F0EAF82146059A2B46C82071
:102E580001F0E4F80A21069A2B46C82001F0DEF8B2
:102E6800552132682B46782001F0D8F8692172681C
:102E78002B46782001F0D2F87D21B2682B467820C5
:102E880001F0CCF805203A4628212B4601F0C6F877
:102E9800D22142462B46052001F0C0F8D2214A46ED
:102EA8002B46562001F0BAF8D22152462B46A620CE
:102EB80001F0B4F8B4215A462B46052001F0AEF8CB
:102EC800DDF80CC0B42162462B46562001F0A6F866
:102ED800B421079A2B46A62001F0A0F8B421089A3D
:102EE8002B46F62001F09AF8099AF620D2212B46B3
:102EF8000BB0BDE8F04F01F091B800BFFC170020FF
:102F0800FBAA050804AB050811AB0508E00C002076
:102F18001CAB0508212B000824AB0508452C00082C
:102F28002DAB0508DD2C000836AB0508892C0008F8
:102F38003FAB05085D2B000848AB0508E92A0008E7
:102F480051AB0508B12A00085AAB0508912A0008B8
:102F580062AB05087D2A000891AA050807B5032376
:102F680008228DE80C004920102223233D210CF073
:102F7800CBF8044B044801221A7003B05DF804EB47
:102F8800FEF7C7BDCD250020C81400202DE9F74362
:102F9800314E324F324D0024304601F070F922464E
:102FA800234647F6FF712F480094019400F026FA53
:102FB8004FF6FF788146414622462346384600941C
:102FC800019400F01BFA4146286022462346384601
:102FD8000094019400F012FA4146686022462346A4
:102FE80038460094019400F009FA2346A860414647
:102FF800224638460094019400F000FA1A49E86025
:103008001A4A204600F0F2FE214607464A46334651
:10301800204601F003F83C212A683346192000F0C5
:10302800FDFF5A216A683346192000F0F7FF78211E
:10303800AA683346192000F0F1FF9621EA68334662
:10304800192000F0EBFFEC20D2213A46334603B0BA
:10305800BDE8F04300F0E2BFF010002091AA050897
:10306800EC0C00206AAB0508DDA70508652F0008F1
:103078001C4B1A781C4B10B51A7009F03BF91B4B06
:103088001B4A00241C6002202346CA2103F0A6F82C
:10309800204608F0CBFD174B1C80174B1C70174BB4
:1030A8001B78023B052B1CD8DFE803F003070B1342
:1030B800170FBDE81040FEF7B9B9BDE81040FEF79C
:1030C800A3B9BDE81040FEF78DB9BDE81040FEF782
:1030D80065B9BDE81040FEF773B9BDE81040FEF7CA
:1030E8004BB910BDEA250020CD250020C40D0020D5
:1030F80090AA05083436002034380020582C0020C7
:1031080008B5084B186806F0B9FA002002F058FF15
:1031180009F0EAF8044B05480B221A70BDE808408C
:10312800FEF7F7BC40260020CD2500206C150020B6
:10313800114B10B500241C70104B186806F09EFA4D
:10314800204602F03DFF0E4B1B780B2B0ED8DFE814
:1031580003F006060D0D0D0D0A080D0D0D060948A4
:1031680002E0094800E00948FEF7D3FC084B1C7050
:10317800BDE8104009F0B8B8582C002040260020BF
:10318800CD250020FC17002080130020A80F002068
:10319800343800202DE9F041144C204601F06FF836
:1031A80000201349134A00F021FE1349134A074629
:1031B800002000F01BFE1249124A0646002000F0CB
:1031C80015FED22105463A462346E62000F026FFA2
:1031D8004B2132462346642000F020FF64206921F9
:1031E8002A462346BDE8F04100F018BF941100209C
:1031F800E3A505083931000872AB05080931000854
:103208007EAB05087930000808B508B143682BB9CA
:103218000348044A044B9B2101F092FC586908BDFD
:103228008BAB050880250408ADAB050808B5FFF78A
:10323800EBFF8068123080B208BD08B5FFF7E4FFE5
:103248004068063080B208BD2DE9F84F044688462C
:10325800FFF7DAFF6689E589074606F1030905F1F4
:103268000F0AB8F1000F1FD01F2002F07DFE204684
:10327800FFF7DCFF83462046FFF7DFFF29460346BA
:103288005FFA8BF2F0B202F0AFFE042002F06EFF9C
:103298000B364FF6FF70033502F066FEB0B2A9B2E6
:1032A8003A68012302F09AFF3D69204641464A46A2
:1032B8005346A847BDE8F88F13B504460DF106013B
:1032C80001A803F0C3F92046FFF79EFF6389BDF804
:1032D8000410BDF80620C91AE389D21A0339C36855
:1032E8000F3A204698471CBDF7B5044614200D46F2
:1032F80016461F4613F0C8FA089BC7600361064BC1
:103308000649074A80E8700000930190054B0020A9
:1033180000F05DFEFEBD00BF5132000843320008D8
:1033280035320008C1320008704708B508B1436853
:103338002BB90448044A054BAD2101F001FC58693A
:1033480008BD00BFCCAB050898250408ADAB05083F
:10335800F8B505460E46FFF7E8FF836B04461BB138
:1033680028463146984700E018466F8994F83C3063
:10337800ED890EB9034310D0208E02F0F5FD608E62
:1033880002F008FE94F8350002F0F0FE94F83430AC
:1033980038462946224602F021FF002384F83C30B3
:1033A800F8BD08B5FFF7C1FF90F83500BDE8084043
:1033B80002F0F1BE38B5FFF7B8FF044613F05CFE23
:1033C800054694F8350002F0E1FE684380B238BD46
:1033D80038B50D46FFF7A9FF29462E22044613F0FB
:1033E8007BFE50B1204629462E2213F0C7FE00234B
:1033F80084F82E30012384F83C3038BD2DE9F7439A
:10340800074640200E461546984613F03DFA0446F6
:1034180028B91148114A124B4E2101F091FB114B6A
:10342800114A12498DE818000020114B00F0CFFD19
:1034380039468146FFF7CCFF9DF82830268684F868
:1034480035300B9B6586A363002384F8348084F8A9
:103458003C304846BDE8FE83CCAB0508B0250408DF
:10346800EAAB050859330008AB330008BD33000840
:103478003133000810B50C46FFF757FF01230486C7
:1034880080F83C3010BD00BF4FF4A0707047C820D2
:1034980070477047074B1B78022B07B508D1064BBE
:1034A8001B78022B04D001A80DF1060103F0CEF819
:1034B8000EBD00BF34380020582C002073B50A4BCD
:1034C80006460D461446009300200849084A094B51
:1034D800019000F07CFD294602462346304602B0A2
:1034E800BDE8704000F09ABD9B3400089134000894
:1034F800973400089D34000813B502AB03E90600B1
:10350800436843B1027C0124082A9C7004D11B69DA
:103518002146984700E01C4620461CBD30B50028CF
:103528002BD0058B002425E0036A1A7C012A05D1DB
:103538005B681A888A421BD1187F30BD052A06D1DC
:103548005B681A888A4213D193F82C0030BD032A8D
:1035580006D15B681A888A420AD193F8250030BDE3
:10356800062A05D15B681A888A4201D1D87A30BD0B
:1035780001340430AC42D7D3002030BD08B1817586
:1035880001207047F8B504460D46D0B1E175D0F872
:1035980098309847012D0DD12746002606E0F86996
:1035A80000F10802436906CA98470136238B04379D
:1035B8009E42F4D3D4F898302046294698470120F3
:1035C800F8BDF8BDF8B50546084617460E4613F08F
:1035D80053FD013FB84234BF04463C463CB128463F
:1035E8003146224613F0CAFD00232B55F8BD2C7036
:1035F800F8BDF7B5044600200090019000296CD072
:103608000E8B68E000F1080351F823301D7C042D6F
:1036180004D15D682D88954247D0013000F1080338
:1036280051F823301D7C012D04D15D682D88954209
:103638003BD0013000F1080351F823301D7C052DE3
:1036480004D15D682D8895422FD0013000F1080320
:1036580051F823301D7C032D04D15D682D889542D7
:1036680023D0013000F1080351F823301D7C022DCE
:1036780004D15D682D88954217D0013000F1080308
:1036880051F823301D7C072D04D15D682D8A9542A1
:103698000BD0013000F1080351F823301D7C062DB2
:1036A80008D15D682D88954203D103F108012046B1
:1036B80015E0013000F1080351F823502B7C082B4A
:1036C80009D16F683F88974204D105F10801204667
:1036D8001A4605E00130B04294D3204669460822D4
:1036E80013F082FB2046FEBDF8B505460F46164688
:1036F800002830D04388032B2FD0202013F0C4F8A3
:10370800044600282BD040F80C5B39460C22FFF702
:1037180059FF1820E66113F0B7F80646B8B102233E
:103728000374012363760F4B446063600E4BA36000
:10373800002323766B8805EB830201339BB2012BB0
:1037480050606B800CD16A685268137608E0204696
:1037580013F0A2F804E0064602E0002600E0064660
:103768003046F8BDFCA404089AA1040837B545689A
:1037780002AB03E906003DB3037C0124042B85F862
:10378800314022D1688E02F0EFFB95F8300002F04C
:10379800EDFC95F8343043B9BDF80200BDF80610C9
:1037A800AA1C234602F01AFD0FE0012B03D108489A
:1037B80040F2395104E0022B07D1054840F241514B
:1037C800044A054B01F0BCF92C4620463EBD00BF1B
:1037D800FDAB050870700408FBAB0508F8B5044696
:1037E8000F46164610B3838A0A2B20D0202013F0E8
:1037F8004BF80546E8B14460102200F1080039464C
:10380800FFF7E0FE4FF6FF73A08A2B801F236B8023
:1038180000232B76831D013080B20128EE6144F825
:103828002350A08207D1A3691876F8BDF8BD0020FF
:10383800F8BD0120F8BD0120F8BD2DE9F3471D466C
:103848004B1C984282460C461746BDF828600DDD91
:1038580095420BDC01320AF101035B1A521BC8B214
:10386800D2B29BB22946009602F0B6FBAAF1020A30
:103878003046C4EB0A0A02F077FB4FF000084FF01D
:1038880001091FFA8AFA0BE0601C08EB050180B2F7
:1038980089B252460023009602F096FB09F101090D
:1038A8007B1B08F1010899451FFA88F8ECD3BDE89D
:1038B800FC87F8B5C7B2144638461E460D4602F0D6
:1038C80095FB621E92B23846294602F08FFB3046BD
:1038D80002F04AFB022606E0A21B92B238462946AD
:1038E80002F084FB0136A642F6D3F8BD73B5044650
:1038F8000E4600F11E001546009200233C2280B2BD
:103908001E3E02F061FBB1B220463C220123009525
:1039180002F05AFB7CBD73B504460E4601381546C5
:1039280000920023032280B2013E02F04DFBB1B2A7
:10393800204603220123009502F046FB7CBDF7B523
:10394800089D2E7BEF7A1C463604AB7A06EB0726D9
:10395800F618431A687B06EB00602D1800200190CA
:10396800121B08462146009501F026FFFEBD30B522
:10397800456885B004AB03E906007DB101242C73CA
:103988006D68BDF80800BDF80A109DF80C209DF878
:103998000E300095FFF7D3FF204600E0284605B01B
:1039A80030BD2DE9F04385B004AB03E90600446857
:1039B800BDF80860BDF80C70002C41D0012384F8D4
:1039C800263094F825300BB9A26800E06268FFB28F
:1039D800BDF80A109DF80E30009230463A46FFF7BF
:1039E800AEFF04F10C08022002F0C0FB404613F0C1
:1039F80043FB054600B1451E0F3F0024153E1FFA44
:103A080087F90DE002F0BCFB02F0C0FB04FB10617B
:103A180089B248462022002302F0FAFB0134E4B2BE
:103A2800AC42EFD3002002F09FFAB8B2B1B24246DE
:103A3800012302F0EDFB002002F098FB012000E0DA
:103A4800204605B0BDE8F0832DE9F04385B004AB0E
:103A580003E906004568BDF80860BDF80C70002D44
:103A68003CD001236B762B7EBDF80A10012B0CBFCE
:103A78006A68AA689DF80E300092FFB23A4630464E
:103A8800FFF75DFF0C35022002F070FB284613F0AB
:103A9800F3FA0E3F81460024163E1FFA87F80DE020
:103AA80002F06EFB02F072FB04FB106189B2404623
:103AB8002022002302F0ACFB0134E4B24C45EFD9DC
:103AC800002002F051FAB8B2B1B22A46012302F03E
:103AD8009FFB002002F04AFB012000E0284605B0C9
:103AE800BDE8F0832DE9F04F85B00546DDF840903C
:103AF800029148469046039313F0BEFADDF838A0C9
:103B0800DDF83CB00646294600242F4611E024B1D2
:103B1800B4420CBF5B46534600E0039B01F1080525
:103B2800ADB200932846029A4346FFF708FF0134D6
:103B38002946B442EBDD002002F016FA022002F01A
:103B480015FB7D1D08F10508A8B21FFA88F14A4641
:103B5800012305B0BDE8F04F02F040BB70B54068E6
:103B680086B006AB03E9060000282ED0012380F8B2
:103B78002D308668164BF21A534243EB020390F835
:103B88002C205AB1002B134D134B144A08BF1D4665
:103B9800134B00F11C0418BF13460AE0002B0D4D0F
:103BA8000D4B0E4A18BF1D460D4B00F10C0408BF03
:103BB8001346BDF81200BDF81410BDF81620009683
:103BC80001950294FFF78EFF012006B070BD00BF7B
:103BD800E07904081C760408C27B0408FE77040810
:103BE800A47D040870B5446886B006AB03E90600F6
:103BF80004B301236377A668104B227FF11A4B4266
:103C080043EB01030AB10BB904E01BB966680C4D1C
:103C18000C4B01E00C4D0D4BBDF81200BDF8141013
:103C2800BDF8162000960C3401950294FFF75AFF50
:103C3800012000E0204606B070BD00BF2C850408B6
:103C4800688104084A83040802870408D88804089D
:103C58002DE9F04385B004AB03E906004468BDF8DC
:103C68000860BDF80A90BDF80C50BDF80E80002C15
:103C780000F08C800123A3740220676802F076FAB2
:103C88004FF6FF7002F086F9002002F06DF9EDB2F0
:103C98005FFA88F8A6F1160189B230462A464346EB
:103CA8000097FFF74CFE277A002F2ED1A28A2346D1
:103CB80000E00137974204D29969097E043300294C
:103CC800F7D002F05DFA02F061FAA9F116091FFABD
:103CD80089F90E2101FB10914FF6FF7208F10108D6
:103CE8005FFA88F389B2009248462A46FFF7A5FD95
:103CF800022002F03BFA1F2002F036F9A38A002BBB
:103D080038D0103DE8B2303E2CE0E3685C68A28A07
:103D18002346013A002700E00137974204D2996907
:103D2800097E04330029F7D002F02AFA02F02EFAAD
:103D38000E2101FB10914FF6FF7208F101085FFA9E
:103D480088F389B2009248462A46FFF776FD02209A
:103D580002F00CFA1F2002F007F9A38A53B1103DB4
:103D6800E8B21A3E0637B1B254F8272001230832C8
:103D780002F04EFA002002F0F9F94FF6FF7002F057
:103D880009F91F2002F0F0F8012000E0204605B0F4
:103D9800BDE8F0832DE9F0410546362088461446F3
:103DA8001F4612F071FD0646E0B120F8025B41465D
:103DB8002E22FFF707FCBDF8183086F834407386CA
:103DC8001820012386F8307086F8313012F05CFD37
:103DD800044618B104234660037404E0304612F028
:103DE8005BFD00E004462046BDE8F081F8B50646D4
:103DF80024200F46154612F047FD0446D8B10F4B54
:103E0800068083600E4B39464360102200F10C0097
:103E1800FFF7D8FB01260023182025622377667751
:103E280012F032FD054610B14460067404E02046E5
:103E380012F032FD00E005462846F8BD2C8504083E
:103E4800867F0408F8B506462C200F46154612F062
:103E58001BFD0446E8B120F80C6B39461922FFF720
:103E6800B1FB0D4BA562A3600C4B6360002384F883
:103E780025301820012384F8263012F005FD054668
:103E880018B103234460037404E0204612F004FDD3
:103E980000E005462846F8BD389E0408D69A04086E
:103EA80010B50446142012F0EFFC20B10023438023
:103EB800014B0480036110BDF136000838B5054692
:103EC800442012F0E1FC0446C0B10E4B0582436069
:103ED8000D4B0360012383740023037283820B4B11
:103EE8000364182012F0D0FC054618B1072344607B
:103EF800037404E0204612F0CFFC00E00546284693
:103F080038BD00BFCC960408C2920408E537000803
:103F18002DE9F04105463420884614461F4612F024
:103F2800B3FC064620B3144B05808360134B41460F
:103F38004360102200F10C00FFF744FB214606F114
:103F48001C001022FFF73EFB002386F82C301820B7
:103F58000123376386F82D3012F096FC044618B119
:103F680005234660037404E0304612F095FC00E037
:103F780004462046BDE8F081E07904083A74040854
:103F88002DE9F041044614200D461646984612F0D5
:103F98007BFC0746B8B1069B048003610023C3720B
:103FA80001234560068180F80A800373182012F007
:103FB8006BFC044618B106234760037404E03846D6
:103FC80012F06AFC00E004462046BDE8F0812DE9C5
:103FD800F041044618200D461646984612F054FC47
:103FE8000746B8B101238370069B04800361079BD1
:103FF80045608660C0F80C804361182012F044FCCC
:10400800044618B108234760037404E0384612F0E8
:1040180043FC00E004462046BDE8F0812DE9F34169
:1040280098461B8B1D2B05460C4617464FF0000083
:1040380000F2B480B5F5A07F0090019000F2AE8048
:10404800F02900F2AB80127CADF80610511EADF8D5
:104058000250072900F28A80DFE801F045595E0422
:10406800456A14767B684E4A7A611A8893F8343028
:104078003A80013BDBB2012B7FD8ADF80240ADF8A6
:1040880006507AE005F11602ADF8002004F1160298
:10409800ADF8042002AE434A16E903007A6107F13D
:1040A800080282E8030003F10802013348F822708D
:1040B800A8F818307B681A8A187A3A8000286CD1D8
:1040C800FFF7FCFE3849436859603849DF6001262C
:1040D800163D196002461E72A8B2E1B24346FFF7C8
:1040E8009DFF30465AE0012A0CBF314B314B7868AE
:1040F8007B6130F80C3B3B8012F0BEFF431CDB00B9
:104108001A34ED18ADF80440ADF8005035E07B687E
:10411800294A1B687A6102E0284A7B687A611B8811
:1041280014353B80ADF800501434ADF8044024E059
:104138007B68234A7A611A883A801A899B7AAD1873
:10414800ADF80050E418F0E77E681E4B7B613388B9
:1041580038463B8073689847013D4519ADF80050D3
:10416800B36838469847013C0419DEE71648174AF1
:10417800174B40F21A3100F0E3FC02AA12E90300DF
:1041880007F1080383E80300B8F8183003F10802C0
:10419800013348F82270A8F818300120BDE8FC81E6
:1041A80075370008593C0008B88E0408AE8A040820
:1041B800ED3B0008653B0008513A0008AB390008A0
:1041C8007739000801350008FDAB05088070040840
:1041D800FBAB0508F8B51646002834D01378002B39
:1041E8002ED0028B002327E0046A257C042D21D1E0
:1041F80065682F888F421DD195F8313053B16F8E85
:1042080001F0D8FE04F1080268866369204606CAF0
:1042180098476F86A81C31462E22FFF7D3F995F8E8
:1042280031307BB104F108026369204606CA984719
:104238000120F8BD013304309342D5D30020F8BDE6
:104248001846F8BD0120F8BD70B5B8B1068B044614
:10425800002310E0256A287C04280AD16D68288884
:10426800884206D11046A91C2E22FFF7ABF901207F
:1042780070BD01330434B342ECD3002070BD38B5AF
:10428800044620B3134BC361134BC0F89830134B4B
:10429800C0F89C30124B00257822C0F8A0308575F4
:1042A800C5750583294600F1200012F0DFFDD4F81A
:1042B80098302046294698470A4A1388312B07D850
:1042C800094941F8234001331380012038BD38BD26
:1042D800284638BD8D350008853500082535000885
:1042E800FB350008FC0C0020441900202DE9F041A2
:1042F8000446002800F0B380078B02460025A8E09A
:10430800136A1E7C042E00F08780012E23D1586882
:1043180003888B4240F09B8005F1080712F0BCFA35
:1043280054F827004FF00008C0F8048012F0B4FADF
:10433800228B531E9D4208D00732238354F8221043
:1043480044F8271044F8228002E044F827802583A7
:104358003046BDE8F081052E5ED0032E5CD0022EDB
:1043680013D15B68186803888B4270D14388013B7E
:104378009BB243800BB912F08FFA05F1080654F886
:104388002630586812F088FA4EE0072E21D15E6870
:10439800338A8B425BD1002706E0BB1D013756F8F4
:1043A800230012F079FAFFB2B38ABB42F5D800278E
:1043B800B78205F1080654F82630586812F06CFAEE
:1043C80054F8260033E044F8267025830120BDE820
:1043D800F081062E1ED1586803888B4237D105F12B
:1043E800080612F059FA54F826000027476012F020
:1043F80053FA228B531E9D4209D00833013A54F8D0
:104408002310228344F8261044F82370DEE744F88A
:1044180026701AE0082E1AD1586803888B4216D1E4
:1044280012F03AFA05F1080654F82600002747600A
:1044380012F032FA228B531E9D42C4D0073254F830
:10444800221044F8261044F822702383BEE7013571
:104458000432BD42FFF454AF0020BDE8F081BDE84E
:10446800F08170B5044600282AD0068B751E0836E0
:1044780000EB86061EE056F8043D1A7C042A13D089
:10448800012A11D0052A0FD0032A0DD0022A02D101
:104498005B681B6809E0072A02D15B68198A05E096
:1044A800062A01D0082A04D15B6819882046FFF73C
:1044B8001DFF013D681CDED100232383012070BD50
:1044C80070BDF0B528B30023068B1A461EE0046AB7
:1044D800257C072D18D16468258A8D4214D1A78AB6
:1044E800002504EB83040DE004EB050C0435DCF82F
:1044F80018C09CF818C0BCF1010F03F1010301D1E9
:10450800D8B2F0BDBB42EFD301320430B242DED3A1
:104518000020F0BD70B508B3048B00231BE0026ACD
:10452800157C072D15D15268158A8D4211D10023AB
:10453800958A11461C46012007E013B99669307622
:1045480001E08E69347601330431AB42F5D30120A2
:1045580070BD01330430A342E1D3002070BD2DE9C2
:10456800F04128B30023078B1A461EE0046A257C15
:10457800072D18D16468258A8D4214D1B4F814C067
:10458800002504EB83040CE066190435B66996F837
:104598001880B8F1010F03D106F10800BDE8F081D9
:1045A80001336345F0D301320430BA42DED3002030
:1045B800BDE8F0812DE9F04700282FD00023B0F89E
:1045C80018C01D4627E0046A267C072E21D164689E
:1045D800268A8E421DD1B4F81480002604EB830984
:1045E80015E009EB0604A7693C7E012C0DD192F871
:1045F80000A0BAF1000F08D007F1080011461022F8
:10460800FEF7E0FF2046BDE8F08701330436434556
:10461800E7D3013504306545D5D30020BDE8F087E0
:10462800F0B5B0B1068B002510E0046A277C062F90
:104638000AD1646827888F4206D123819DF81430F7
:104648006260A3720120F0BD01350430B542ECD39D
:104658000020F0BD10B500210446FEF793FF204668
:104668000121BDE81040FEF78DBF38B598B1048B25
:10467800024600230CE0106A058804328D4206D1F8
:1046880000F10802436906CA9847012038BD013382
:10469800A342F0D3002038BD10B50C460021FEF728
:1046A80071FF20460121BDE81040FEF76BBF13B52E
:1046B80002AC04E90C00BDF80230834206D8BDF80C
:1046C8000030834234BF0020012000E00020BDF804
:1046D80006308B4206D8BDF804308B4234BF002127
:1046E800012100E00021002818BF0846C0B21CBD07
:1046F80038B5114B114A1988002319E052F8045FA4
:10470800A87D012812D100240CE004F1080355F813
:104718002300037C082B03D1436800211B699847B9
:104728000134A4B22B8BA342EFD838BD01339BB21E
:104738008B42E3D138BD00BFFC0C0020401900209B
:10474800704770B5094CA5787DB9094B1E78012EC4
:104758000BD16368013363606268064B9A4204D9DF
:10476800284601F0C5FCA670656070BDFC0C0020F1
:104778009801002040420F00054A9060134602E06D
:1047880099680139996091680029F9D1704700BF8B
:10479800FC0C0020F0B585B001F056FF002800F0B1
:1047A8004981002502A80DF10A01ADF80850ADF8BD
:1047B8000A5001F04BFF03A80DF10E01ADF80C50A3
:1047C800ADF80E5001F08EFFBDF80C10BDF80820B2
:1047D8000091BDF80E10BDF80A3001912C46964D97
:1047E800964908200AF0E4FDA878012803D101F0D1
:1047F8007FFCAC7019E1924B5B78012B40F015817E
:10480800AB78002B40F011816B6029888D4A09E153
:1048180052F8046FB07D012840F002810025FAE0CB
:1048280005F10803BDF8080056F82340BDF80A1042
:1048380004F108030CCBFFF73AFF002800F0E980E9
:10484800237C013B062B00F29F80DFE803F004295C
:10485800159D1F9D4C006668012304F108053377F8
:1048680095E8060063692046984700233377204679
:10487800636995E8060086E0636893F8252012F1DD
:10488800FF3218BF012283F8252077E0636893F888
:104898002C2012F1FF3218BF012283F82C206DE082
:1048A8006268137E1568002B6ED16E882F462946E4
:1048B800184606E051F804EFDEF804E001338EF8FC
:1048C8001800B342F6D301231376002607E057F801
:1048D800040F00F10802436906CA984701366B883D
:1048E8009E42F4D350E0656820892E68A37B227B22
:1048F8000096A0F1160189B2FFF721F81420FFF7FE
:104908003BFF2B7AC3B9AF8A29461A461E4609E0EF
:10491800886990F818E00676BEF1010F08BF1346C3
:1049280004310132BA42F3D301220BB9AB6924E056
:10493800053355F8233020E06368DB685A680023A4
:10494800908A154619461F4609E0AE6996F818E0A0
:104958003776BEF1010F08BF0B460435013181429D
:10496800F3D3411E8B4203D1053052F8203003E0C7
:1049780004D2073352F8233001221A7604F10802D0
:1049880006CA636920469847237C013B072B4CD80D
:10499800DFE803F00410074B0A0D123A63681B6A3C
:1049A80034E063689B6A2DE063681B6B2AE06368E8
:1049B8001B6927E0636824E063681A7A7AB9988AE1
:1049C8001946013800E00132824204D28C69247E03
:1049D8000431002CF7D0063253F8223011E0DB689E
:1049E8005A68908A11460138002300E00133834257
:1049F80004D28C69247E0431002CF7D0063352F897
:104A08002330DB69984710E06368DB6820469847E5
:104A18000BE00135ADB2338BAB423FF601AF04E09A
:104A280001339BB28B427FF4F3AE01F053FE0F20AB
:104A3800FFF7A2FE05B0F0BDFC0C002023AC050872
:104A48009801002040190020034B9A6812B19A6817
:104A5800013A9A60704700BFFC0C00202DE9F3472B
:104A68000120DFF8D080DFF8D09001460CF03AF84A
:104A7800012400254FF480760227404669460096B7
:104A88008DF804708DF805408DF806508DF80740B4
:104A98000BF080FC4046082122460BF0FBFC244B1F
:104AA800DFF898801A6844F2A243B2FBF3FA0AF1DD
:104AB800FF3A204621461FFA8AFA0CF043F8C8F854
:104AC80004A048464146A8F80050A8F80250A8F8A3
:104AD800085088F80A500CF0D1FB7023A8F80C3065
:104AE8000423A8F810300AF1FF3A6323642203FB79
:104AF8000AF3B3FBF2F39BB2C8F8143008F10C01C7
:104B08004846A8F80E40A8F81870A8F81A50A8F84F
:104B18001C60A8F81E500CF0CFFC484621460CF04B
:104B280042FC484621460CF048FFBDE8FC8700BF20
:104B3800E401002000000240000001400C0D0020AC
:104B480083B50E460746154910201C4615460AF03F
:104B58002FFC102012490AF02BFC102011490AF0F2
:104B680027FC10200E490AF023FC002310200E49D0
:104B780001930AF01DFC334610200C493A460AF00E
:104B880017FC10200A492A460AF012FC102009498D
:104B980022460AF00DFC019B0133E7E75DAC0508EE
:104BA80062AC050882AC050892AC0508A2AC050801
:104BB800B7AC0508C8AC050808B5164B1A6A013227
:104BC8001A621A6A012A1A4603D0134840F21D21B4
:104BD8000FE05862194602E04B6A013B4B62506A8B
:104BE8000C4B0028F8D11A6A012A06D00A484FF45B
:104BF8000A710A4A0A4BFFF7A3FF1A6A013A1A62B6
:104C08001B6A2BB10448054A064B40F22A21F2E7F9
:104C180008BD00BF0C0D0020D9AC05085EA804082B
:104C280003AD050814AD050810B5084C0221002293
:104C380020460BF024FC44F6FF70FFF7BDFF20462A
:104C480002210122BDE810400BF019BC000402400B
:104C58000C4B0D491A6844F2A2436428B2FBF3F3E3
:104C6800D4BF20EAE0706420013B9BB24B60013B5B
:104C780058436422B0FBF2F080B2486103480C311B
:104C88000CF09DBBE40100200C0D00200000014049
:104C980010B5134B93F828202AB11248124A134B27
:104CA8004FF442710EE0012283F8282066234FF06A
:104CB800C042013BDBB2108033B90A480A4A0C4BA8
:104CC80040F21231FFF73CFF1488A4B28442F0D1BD
:104CD800084B1980024B002283F8282010BD00BF22
:104CE8000C0D0020D9AC050868A8040825AD0508F6
:104CF800FBAB05080000026010B5FFF7AFFE6420AB
:104D0800FFF7A6FF21210720FFF7C2FF3220FFF798
:104D180053FF01210020FFF7BBFF3220FFF74CFFB4
:104D280023210720FFF7B4FF3220FFF745FF0021BA
:104D38001020FFF7ADFF41F28830FFF73DFF332128
:104D48000720FFF7A5FF3220FFF736FF112046F6B0
:104D58003001FFF79DFF3220FFF72EFF4FF4C061AF
:104D68000220FFF795FF3220FFF726FF122046F6B4
:104D7800EB41FFF78DFF3220FFF71EFF03204AF6B5
:104D8800A401FFF785FF3220FFF716FF00210C2052
:104D9800FFF77EFF3220FFF70FFF0D2040F60C01D2
:104DA800FFF776FF3220FFF707FF0E204FF42C5154
:104DB800FFF76EFF3220FFF7FFFEB0211E20FFF73E
:104DC80067FF3220FFF7F8FE012042F63F31FFF778
:104DD8005FFF3220FFF7F0FE05200021FFF758FFA4
:104DE8003220FFF7E9FE00210620FFF751FF3220AD
:104DF800FFF7E2FE16204EF61C71FFF749FF32203E
:104E0800FFF7DAFE172040F20311FFF741FF3220C7
:104E1800FFF7D2FE00210B20FFF73AFF3220FFF701
:104E2800CBFE00210F20FFF733FF3220FFF7C4FE2F
:104E380041200021FFF72CFF3220FFF7BDFE422062
:104E48000021FFF725FF3220FFF7B6FE002148209A
:104E5800FFF71EFF40F23F143220FFF7ADFE214658
:104E68004920FFF715FF3220FFF7A6FE00214A2050
:104E7800FFF70EFF3220FFF79FFE00214B20FFF7C0
:104E880007FF3220FFF798FE44204FF46F41FFF7E9
:104E9800FFFE3220FFF790FE00214520FFF7F8FEC5
:104EA8003220FFF789FE21464620FFF7F1FE322027
:104EB800FFF782FE302040F20771FFF7E9FE32204B
:104EC800FFF77AFE31204FF40171FFF7E1FE32203F
:104ED800FFF772FE32204FF40171FFF7D9FE40F25E
:104EE80002543220FFF768FE21463320FFF7D0FE38
:104EF8003220FFF761FE342040F20751FFF7C8FE69
:104F08003220FFF759FE35204FF40171FFF7C0FE3C
:104F18003220FFF751FE36204FF40171FFF7B8FE3B
:104F28003220FFF749FE21463720FFF7B1FEA4F5EE
:104F380000743220FFF740FE21463A20FFF7A8FE12
:104F48003220FFF739FE2F2041F2BE21FFF7A0FEE5
:104F58003220FFF731FE21463B20FFF799FE322031
:104F6800FFF72AFE00212320FFF792FE3220FFF7E9
:104F780023FE00212420FFF78BFE3220FFF71CFEC2
:104F880025204FF40041FFF783FE3220FFF714FE7F
:104F980000214F20FFF77CFE3220FFF70DFE4E2048
:104FA8000021FFF775FE3220BDE8104004E608B581
:104FB800124B93F829202AB11148124A124B40F299
:104FC80022310FE0012283F82920222166234FF0A5
:104FD800C042013BDBB2118033B90948094A0B4B87
:104FE80040F23B31FFF7ACFD108880B22228F0D1A7
:104FF800024B002283F8292008BD00BF0C0D0020B9
:10500800D9AC050875A8040825AD0508FBAB05084B
:1050180010B51E4B032826D8DFE800F0021A080E48
:105028001C8841F2280246F628000AE01C8841F252
:10503800080246F6080004E01C8841F2300246F6F1
:10504800300049F241318C4214BF014611460BE051
:10505800188846F6200249F24131884214BF1146A9
:105068004FF4815100E000211B8848F689129342D1
:1050780005D049F22032934204D1032000E01120E8
:10508800FFF706FEBDE8104091E700BF9A01002037
:10509800014B18800A208FE5000002604FF0C043E2
:1050A800188003F500331A881A88188880B2704768
:1050B8004FF0C04322221A8003F5003382B01A88C9
:1050C80092B2ADF806201B889BB2ADF80630BDF849
:1050D800060080B202B07047072040F27311D7E58E
:1050E80007200021D4E582B0044BADF80600BDF8D6
:1050F800062092B25A8502B0704700BF0C0D0020FE
:1051080082B0044BADF80600BDF8062092B25A8072
:1051180002B070479A010020014B80B21880704796
:10512800000002604FF0C04380B218807047024B05
:1051380080B21880704700BF000002604FF0C04383
:1051480080B218807047024B80B21880704700BF49
:105158000000026082B0044B0190019ADA62DA6AB8
:10516800002AFCD102B070470C0D002070B54FF03A
:10517800C0452A242C800A4C060AC0B2268020800A
:10518800100AD2B2208022802B222A800A0A22808A
:10519800C9B21A0ADBB221802280238070BD00BF09
:1051A8000000026010B50B4614460246FFF7DEFF0A
:1051B8004FF0C0432C22A0B21A80BDE8104067E728
:1051C800114B1B8848F68912934210B504460BD040
:1051D80049F22032934212D1C1F1EF01202089B265
:1051E800FFF756FD212006E0C1F1EF014E2089B2FC
:1051F800FFF74EFD4F202146BDE8104048E5024626
:105208000B46BDE81040B1E79A01002008B5FFF74A
:10521800D7FF0F4B1B78012B4FF0C0420D4B0FD11E
:105228002E2111801A881A881B8892B202F0FC007D
:1052380002F4784242EAC000C3F3C423184308BD0D
:10524800222111801A881A88188880B208BD00BFE8
:10525800141A00200000026070B5074D06460124AC
:1052680021463046FFF7D2FF0134A4B2C82C25F8F6
:10527800020FF5D170BD00BF3638002010B5084BBD
:105288001B78012B144602D1BDE810408AE7FFF7CE
:1052980097FFFFF78CFE2046BDE81040F8E600BFF8
:1052A800141A002070B5074D064601242146013422
:1052B80035F8022F3046A4B2FFF7E0FFC82CF5D12D
:1052C80070BD00BF3638002070B505460E46FFF7A2
:1052D800C3FF01242146013428463246A4B2FFF711
:1052E800CDFFC82CF6D170BD2DE9F04104460D461E
:1052F8001646BDF81880032B39D8DFE803F00B35C4
:105308001927381980B2294642460137FFF7B6FFF8
:10531800BFB200E00027B742F3D1BDE8F081E01B3F
:1053280080B2294642460137FFF7A8FFBFB200E026
:105338000027B742F3D1BDE8F081E91B89B22046C6
:1053480042460137FFF79AFFBFB200E00027B74295
:10535800F3D1BDE8F081791989B220464246013778
:10536800FFF78CFFBFB200E00027B742F3D1BDE8DA
:10537800F08170B5194B1A4A598E92F90040641899
:105388000025A4B28AB0AC4208BF0124C62C28BFAD
:10539800C62415700F264FF6FF721E865C865A8546
:1053A80019202B46009221460A22FFF79DFF21462D
:1053B8003046FFF72BFF224603460A4902A811F0A0
:1053C800D5FD02AA06A8084911F0D0FD3220D22145
:1053D80006AA2B4600F002FF0AB070BD0C0D002093
:1053E800811A00203AAD050842AD05082DE9F341C0
:1053F800BDF820500C4690461F461A460023064624
:105408000095FFF771FF611E414430463A4600237C
:1054180089B20095FFF768FF3046214642460123CE
:105428000095013EFFF760FFBF19B8B2214642461A
:105438000123089502B0BDE8F04155E72DE9F04198
:105448000D46C5F1F008411E5E18C2EB0802C5F111
:10545800EF039BB292B2B6B29A422CBF90469846DE
:105468009A4234BF11461946864234BF374607462A
:1054780040F23F13864238BF06469E4228BF1E466A
:10548800174B1B8848F68912B8F1EF0F28BF4FF069
:10549800EF089342044610D049F2203293421AD1C1
:1054A8005020FFF7F5FB51204146FFF7F1FB522052
:1054B8003946FFF7EDFB53200AE041EA082189B29B
:1054C8004420FFF7E5FB45203946FFF7E1FB46207E
:1054D8003146FFF7DDFB20462946BDE8F0416FE67F
:1054E8009A01002000200146F0224FF4A073A5E79E
:1054F80070B580B202FB03F489B292B29BB2FFF797
:105508009DFF0020FFF784FD0025064E04E0708D06
:1055180080B2FFF7BDFD0135A542F8DBBDE870405C
:10552800E0E700BF0C0D002070B54FF0C0452A24FD
:105538002C80094C060A26802080080A20802180B9
:105548002B212980110A218022801A0A2280238097
:105558002C232B8070BD00BF0000026070B5114B7A
:105568001B78012B044607D1002040F23F11024668
:10557800EF23FFF7D9FF04E0FFF7B4FF0020FFF7A0
:1055880047FDF02509E0013E2046B6B2FFF780FD51
:10559800002EF8D1013DADB215B14FF4A076F2E777
:1055A80070BD00BF141A00202DE9F04F1C463E4B79
:1055B80087B01B78039183469DF844101098059195
:1055C800012B039B049092461FFA8BF09AB208D1E4
:1055D800411E531E0919534489B29BB2FFF7A4FF19
:1055E80009E01FFA8AF51146A3B22A46FFF726FFFB
:1055F8000020FFF70DFD0027DDF80C803E4640F245
:105608003F1CA14639E0BBF1000F2EDB65452CDCC1
:105618000398002829DBB8F1EF0F26DC220702D116
:10562800002CC8BF013621492140002903DA01397D
:1056380061F00F010131059A0AB1C1F10F01049817
:1056480030F8162003FA01F10A4012B26AB118497B
:105658004A8D029392B2A8B21FFA88F1CDF804C01D
:10566800FFF70CFEDDF804C0029B013401354C4500
:10567800C9DB0136013708F10108574503DA5D46F1
:1056880000240123F3E7084B1B78012B08D10020E5
:1056980040F23F110246EF2307B0BDE8F04F43E761
:1056A80007B0BDE8F04F1DE7141A00200F00008076
:1056B8000C0D00202DE9F74F1F463B4BDDF83080DD
:1056C8001B7816469DF83420012B044601920D469E
:1056D80080B28AB208D1411E531EC9199B1989B2DA
:1056E8009BB2FFF721FF09E01FFA86FE1146BBB205
:1056F8007246FFF7A3FE0020FFF78AFC4FF0000B6D
:10570800DA463DE0002C30DB09EB040340F23F129F
:1057180093422ADC002D28DB0BEB0503EF2B24DC5E
:1057280019F00F0F04D1B9F1000FC8BF0AF1010A2F
:105738001E4B09EA0303002B03DA013B63F00F0356
:105748000133019A0AB1C3F10F03012202FA03F3EC
:1057580038F81A2013401BB213B1154B588D01E0CD
:10576800144A508880B2FFF793FC09F1010901E05F
:105778004FF00009B945C5DB0AF1010A0BF1010B2D
:10578800B345F5DB084B1B78012B08D1002040F20C
:105798003F110246EF2303B0BDE8F04FC4E603B063
:1057A800BDE8F04F9EE600BF141A00200F000080ED
:1057B8000C0D00209A0100202DE9F0411C4F069C99
:1057C8003F789DF81C60012F02FB03F580B28FB271
:1057D80009D1411ECB1899B27B1E9A1893B23A464A
:1057E800FFF7A2FE07E092B29BB23946FFF726FE0A
:1057F8000020FFF70DFC002709E034F8020B1EB16A
:10580800030A43EA002080B2FFF742FC0137AF42A7
:10581800F3DB074B1B78012B07D1002040F23F1127
:105828000246EF23BDE8F0417EE6BDE8F04159E6C7
:10583800141A00202DE9F0431F2093B0FFF78EFEC5
:105848004FF47840FFF78AFE4FF6E0754FF4FC609E
:10585800FFF784FE2846FFF781FE0020514CFFF732
:105868007DFE00204FF6FF79014664220346A4F826
:105878002A90CDF80090FFF737FD00200A21642216
:105888000346CDF80090FFF72FFD00200146642263
:1058980001234FF4784765850095FFF725FD7720AC
:1058A800EF21C82200234FF4FC6667850097FFF7B5
:1058B8001BFDBD213222012340F23F106685009670
:1058C800FFF712FDA0203222002378216785009778
:1058D800FFF70AFDA0207821322201234FF01F088C
:1058E80066850096FFF700FDA0207821322202236A
:1058F800A4F82A80CDF80080FFF7F6FCA0207821D4
:105908003222032365850095FFF7EEFC264B2749D5
:10591800A3F8028002AD3C22284611F065FAEB207C
:10592800C3210522302300950025A4F82A9001956B
:10593800FFF7C0FE32210A2096220B4667850097A2
:10594800FFF754FD32213C2096220B4666850096CF
:10595800FFF74CFD32210B4696226E20A4F82A80D0
:10596800CDF80080FFF742FDFFF7BAFBFFF7B4FB65
:105978003220FFF76DF92846FFF76AF96420FFF730
:1059880067F90B4B03F110028DE8240028465A688A
:105998001B682946FFF710FF1195119B01331193DE
:1059A800FBE700BF0C0D00209A0100208AA804081C
:1059B80048CD01082DE9F14FFFF750F84FF0C045E9
:1059C8006420FFF745F90127FFF72EF94FF0280962
:1059D8006D48FFF7F1F82F800520A5F8009003F037
:1059E8004DFACF232B80694B002683221E801A8014
:1059F80030221A80ED222A804FF064080322A3F88F
:105A080000801A8012221A8081221A80E8222A80B5
:105A180085221A8079221F801A80CB222A80392277
:105A28001A804FF0340C02242C21F72219801E8092
:105A3800A3F800C01C802A8020221A80EA222A802B
:105A4800C0221E80C1211E802A8026221A80298019
:105A580011211980C5212980352119803E211980FD
:105A6800C7212980BE211980362129803A20552155
:105A7800A3F8009028801980B12129804FF0100BDD
:105A8800F2211E80A3F800B02980082119802A80FD
:105A9800E0221F804FF01F092A801A22A3F80090E5
:105AA8004FF0180A1A800F210A22A3F800A01A80C2
:105AB80019800621198045211980872119803221F2
:105AC800198007211A804FF0E10E19801C800524E7
:105AD80019801C801E80A5F800E04FF0250E1E805E
:105AE800A3F800E04FF0270EA3F800E01C80A3F80D
:105AF80000B04FF0090BA3F800B04FF0780B1880F6
:105B0800A3F800B04FF04D0BA3F800B01C800D2493
:105B1800A3F800A01C8038241C8018802A20A3F831
:105B28000090EF2428802B201E801E801E801C8061
:105B380028803F201E801E801F801880B720A5F86F
:105B480000C028801980B62129801A8082221A80F4
:105B58001122A3F800E040461E8029272A8003F07E
:105B68008DF940462F8003F089F90948FFF724F89A
:105B78002C232F8030462B8040F23F11324623469B
:105B880001B0BDE8F04FCFE4400D03000000026013
:105B980040420F002DE9F041022098B00121002475
:105BA8000AF0A0FF012502268048169616A98DF84E
:105BB8005D408DF85E408DF85F408DF85C500AF0CE
:105BC800E9FB182029460AF08DFF284629460AF0E5
:105BD800A1FF21460C2276480AF05CFC0C2274488E
:105BE80029460AF057FC04210C2271480AF052FC9D
:105BF80005210C226E480AF04DFC07210C226C4846
:105C08000AF048FC08210C2269480AF043FC0921E3
:105C18000C2267480AF03EFC0A2165480C220AF06B
:105C280039FC0B2162480C220AF034FC0E210C22AC
:105C38005F480AF02FFC0F210C225D480AF02AFC6D
:105C480007210C225B480AF025FC08210C22594840
:105C58000AF020FC09210C2256480AF01BFC0A21F4
:105C68000C2254480AF016FC0B210C2251480AF069
:105C780011FC0C210A464F480AF00CFC0D210C229D
:105C88004C480AF007FC0E210C224A480AF002FC94
:105C98000C2248480F210AF0FDFB4CF6B373444828
:105CA800169316A98DF85C608DF85E408DF85F40FC
:105CB8008DF85D500AF06EFB16A94FF680733D48CB
:105CC80016938DF85C608DF85E408DF85F408DF816
:105CD8005D500AF05FFB40F6B830FEF76DFFFEF747
:105CE800A3FF40F6B830FEF767FF0F2311934FF478
:105CF800805310270DF13C08099368464FF40023A0
:105D08001094129414941594009401940294039797
:105D180004940694079408940A9405940B940C939D
:105D2800CDF834800F9513950AF0ADF80523684631
:105D380011930F961094129414941594CDF83880FA
:105D480013950AF0A0F8294620460AF01CF940F6F7
:105D5800B830FEF731FF2046FFF7A0F90446164990
:105D6800164E3846224609F023FB41F289239C420D
:105D780048F68918124F01D044450ED1FEF7BCFFF2
:105D880000233B70A6F8008010200E4948F68912BF
:105D980041F2892309F00CFB05E0FFF70BFE49F2FD
:105DA80041333D70338018B0BDE8F08100040240F3
:105DB800000C02400010024047AD05089A0100207F
:105DC800141A00205EAD05084FF0C04336221A8031
:105DD80003F50033012814BF682048201880704755
:105DE80070B5244B01228CB01A7000240AE0A9B2C5
:105DF8001F2230460135FFF741FA642DF7D10134EF
:105E0800642C02D00025A6B2F1E7322001460246F2
:105E18000346FFF7ABF94FF0C0432E221A8003F573
:105E2800003300201A881C881D88A4B200F09CF852
:105E3800ADB20023224600930F492B4603A811F068
:105E480095F800230A20C82103AA00F0C7F904F036
:105E5800FC0204F4784444EAC20242EAD522074923
:105E680003A811F083F80A20DC2103AA002300F01C
:105E7800B5F9FEE7141A00209DAD0508B5AD050873
:105E88002DE9F04F40F23F19484534BF04464C46CF
:105E9800EF2B34BF98464FF0EF084A4538BF91467C
:105EA800EF2934BF0D46EF25C4EB090AC5EB0807F7
:105EB80085B0BAF1000FB8BFCAF1000A002FB8BF09
:105EC8007F424FF6FF734C452CBF1A4601221FFA3A
:105ED8008AFA454538BF0123BFB202930FFA8AF602
:105EE8003BB29E42BDF838B0019202DDC6F34F06C0
:105EF80007E0022693FBF6F67642B6B201E01E46AC
:105F080003E00FFA8AF35B420393144A1378022BD7
:105F1800204629465A4602D1FDF7FDFC01E0FFF76D
:105F2800ADF94C4501D1454514D0039A33B293429B
:105F380005DD019AF31BA4189BB2A4B200E0334616
:105F480036B23AB29642DADA029A5344AD189BB2A4
:105F5800ADB2D4E705B0BDE8F08F00BF582C0020E3
:105F6800004870471C1A002082B0064BADF80600A6
:105F7800BDF8062092B21A80188880B202B0FFF7E6
:105F8800B2B800BF181A0020014B188880B27047B9
:105F9800181A002082B0064BADF80600BDF806209E
:105FA80092B21A80188880B202B0FFF7A9B800BF71
:105FB8001A1A0020014B188880B270471A1A00205C
:105FC800FFF7CCBAFFF73ABA10B5BDF8084002940B
:105FD800BDE81040FFF788B910B5BDF80840029435
:105FE800BDE81040FFF702BAFFF782BA2DE9F04F7B
:105FF8004FEA420800253D4C85B082468B46C8F1E1
:10600800030817462E461FFA87F909EB0B0C22885E
:1060180005EB0A031FFA8CFC9BB26146184692B244
:10602800CDF804C00293FFF729F9C9EB0B0292B22D
:106038000392029B22880399184692B2FFF71EF931
:10604800DDF804C02288C5EB0A039BB261461846F6
:1060580092B20293FFF712F9029B2288039918461D
:1060680092B2FFF70BF905EB0B0292B2039209EB20
:106078000A03228803999BB2184692B20293FFF74B
:10608800FDF8029B2288C5EB0B0C1FFA8CFC184606
:10609800614692B2CDF804C0C9EB0A09FFF7EEF8E1
:1060A800228803991FFA89F992B24846FFF7E6F861
:1060B8002288DDF804C092B248466146FFF7DEF850
:1060C800B8F1000F04DA08EB860808F1060805E0C5
:1060D800F31B08F10A0808EB8308013F0136013574
:1060E800BE42ADB28FD905B0BDE8F08F181A0020B6
:1060F80008B9FEF7F5BF012801D1FEF7EDBF7047DB
:10610800704700200146F0224FF4A073FFF796B9BC
:10611800704708B505280CD8DFE800F0121403050D
:106128000709094808BD094808BD094808BD0948C4
:1061380008BD0948094A0A4B40F24111FEF700FD23
:10614800084808BD084808BD8801002078010020DB
:106158007001002068010020C0AD0508C6A8040829
:10616800FBAB0508900100208001002010B5044613
:10617800FFF7CFFF014B18601C7110BDA001002074
:10618800014B1879704700BFA001002008B5FFF740
:10619800C0FF808808BD08B5FFF7BBFFC08808BDF1
:1061A800F7B51F460B4B0C4E1D681446EA882B6842
:1061B800203C5443A4B2AE1B03EB440418BF012691
:1061C800AB888DE8500017B1FFF7EEF901E0FFF753
:1061D80071FAFEBDA0010020900100202DE9F041D8
:1061E8000F46984615460446084E08E020464346A2
:1061F8003946FFF7D5FF33689B88E418A4B215F831
:10620800012B002AF2D1BDE8F08100BFA0010020D7
:1062180010B5044608462146BDE81040DEE7094BA4
:1062280070B5044618790E461546FFF7B4FFC6F157
:10623800F001091A89B220462A460023BDE87040B9
:10624800CCE700BFA0010020704700BF044B1A68CC
:106258000AB9044A1A601A6810181860104670477C
:10626800400D0020D43C00204FF0FF30704708B5A7
:106278000248034A034B3721FEF762FCDFAD0508ED
:10628800DCA80408FBAB05080120704710B50446DC
:106298000A4802210AF0ACFE0028F9D00748214636
:1062A8000AF06FFE054801210AF0A2FE0028F9D085
:1062B8000248BDE810400AF061BE00BF0038004047
:1062C80010B5194802210AF093FE0028F9D01648A3
:1062D80000210AF056FE144801210AF089FE002820
:1062E800F9D011480AF04AFE0402A4B2002301E0E2
:1062F80001339BB2002BFBD00B4802210AF078FE39
:106308000028F9D0084800210AF03BFE0648012180
:106318000AF06EFE0028F9D003480AF02FFE204349
:10632800C0F3CB0010BD00BF003800402DE9F04796
:106338008AB00AAF0A2001210AF0D4FB4FF4604367
:1063480047F8143D474EDFF824A1012400254FF0FB
:106358000208304639468DF81A508DF818808DF8A5
:1063680019808DF81B400AF015F830460D210522DA
:106378000AF090F830460E2105220AF08BF8052223
:1063880030460F210AF086F821464FF480400AF083
:10639800CDFB50460AF0A8FC4FF48273ADF80230EA
:1063A8004FF40073ADF80A303823ADF80C3050467E
:1063B80007236946ADF81030ADF80050ADF8045029
:1063C800ADF80650ADF80850ADF80E500AF0BEFC16
:1063D800504621460AF055FDA9468DF81A50304618
:1063E8004FF48055394605958DF818408DF8198079
:1063F8008DF81B4009F0CEFF304629460AF03BF8DD
:106408004025394618488DF818908DF819808DF870
:106418001A908DF81B40059509F0BCFF21464FF4F2
:1064280080400AF08FFB062103200AF019FE0C2396
:1064380007A88DF8213007958DF820908DF8224017
:1064480009F09CFC17238DF8243009A80F238DF838
:1064580025308DF826308DF8274002F02DFF0AB040
:10646800BDE8F08700040240000C024000380040FC
:10647800014B1878704700BF440D0020024B5A8822
:106488009B8802800B807047440D0020014B00223E
:106498001A707047440D0020F0B593B0684600218B
:1064A800482210F0E3FC6D46002464484FF4805104
:1064B80009F0E3FF002301E001339BB2002BFBD07E
:1064C8009020FFF7E3FE002301E001339BB2002B8D
:1064D800FBD0FFF7F5FE4FF480510746574809F007
:1064E800CAFF002301E001339BB2002BFBD05348C5
:1064F8004FF4805109F0C1FF002301E001339BB242
:10650800002BFBD0D020FFF7C1FE002301E00133B0
:106518009BB2002BFBD0FFF7D3FE4FF48051064609
:10652800464809F0A8FF45F8047B01342E62444828
:106538004021E4B209F08DFF10B9092CB5D101E072
:10654800092C78D19DE80C00D218029B0398069973
:10655800D218049BC018059BC018079BCB18089934
:10656800032490FBF4F092FBF4F25B1893FBF4F332
:10657800151AC11A9C1A002DB8BF6D420029B8BF60
:106588004942002CB8BF6442502D03DD502909DD73
:10659800502C50DC8D4205DAAC424FF0020405DB8A
:1065A800111806E08C424FF0020401DAD11800E01D
:1065B800C1180A9B099A0C980F9DD2180B9BD218E8
:1065C8000D9BC0180E9BC018109BEB18119D91FBDA
:1065D800F4F1032492FBF4F290FBF4F05B1993FBC3
:1065E800F4F3161AC41A9D1A002EB8BF7642002C6E
:1065F800B8BF6442002DB8BF6D42502E89B203DD8A
:10660800502C09DD502D16DCA64205DAB5424FF0B4
:10661800020405DB131806E0A5424FF0020401DA74
:10662800D31800E0C318074A93FBF4F39BB2938096
:1066380001235180137013B0F0BD00BF0004024065
:10664800000C0240440D0020FFF712BFF7B50546C5
:106658000C4601A80DF10601FFF710FF1B4BBDF812
:106668000660BDF8040093E80600724301FB0022AF
:1066780099685218164992FBF1F207EE102AF8EEC3
:10668800C77A40F23F17FCEEE77A17EE902A92B2EB
:10669800B2F5207F28BF3A462A801D69DA685B690F
:1066A8006E4302FB0060C01890FBF1F107EE101A70
:1066B800F8EEC77AFCEEE77A17EE903A9BB2B3F59C
:1066C800F07F28BFEF232380FEBD00BF4C0D0020C4
:1066D80040420F00FFF7DABE014B187E704700BF3B
:1066E8004C0D0020FFF7CABE042808B505D9074895
:1066F800074A084B7D21FEF723FA054B03EB800080
:10670800038B0B80438B138008BD00BF00AE0508C8
:10671800E2A804081EAE050808B5082001F0BAF979
:1067280042F69643C31A584240EB030008BD10B521
:106738000A2001F0D7F90C4C20600E2001F0D2F9A4
:106748006060122001F0CEF9A060162001F0CAF9AD
:10675800E0601A2001F0C6F920611E2001F0C2F99C
:1067680001236061237610BD4C0D002010B5FFF7A2
:10677800DDFD01F06DFA044601F076FA074903469B
:106788002246202008F014FEFFF7C6FF28B101F0CA
:1067980079FA10B9BDE81040C9E710BD5AAE05082E
:1067A80010B5104C0A20216801F083F961680E20A9
:1067B80001F07FF9A168122001F07BF9E168162049
:1067C80001F077F921691A2001F073F961691E2037
:1067D80001F06FF9082042F69641BDE8104001F03B
:1067E8004BB900BF4C0D00202DE9F04F0346A7B070
:1067F800B0F800C01C898688DF885D89CDF810C094
:10680800B249B0F802C0B3F80C90B3F80E80CDF8D6
:1068180024C00FFA84FB30B201220FFA87FE0BEB7B
:10682800000C0A7629B20FFA89FACDF888C001EB74
:106838000E0C0FFA88F2CDF890C00AEB0B0CCDF8CD
:1068480030C002EB010CCDF858C0B3F810C05B8A19
:10685800CDF800C00FFA8CFC06910CEB00010A91F0
:1068680002930CEB0A011BB2239103EB0E010E916C
:1068780099182591049900FA81F0584450446044CD
:10688800DDF824C006990EFA8CFEDDF810C01FFA58
:1068980080FB1CFB0CF08E4416FB0600964414FB90
:1068A8000400009A19FB09009E4412FB02001FFA1B
:1068B8008EFA0BF0A7FCDDF824C0029ACDE912018C
:1068C8001CFB0CF017FB070015FB050018FB080064
:1068D80012FB02000BF096FCDDF824C0029ACDE909
:1068E800140104991CFB01F317FB063615FB04661B
:1068F800009B18FB096612FB03600BF083FCDDE9C3
:106908001423CDE90001DDE912010BF0F1FC044686
:106918000D46DDE9000102460B460BF0E9FC024694
:106928000B46204629460BF02FFBCDE918015846A7
:106938000BF078FCCDE91001DDE91023DDE9000159
:106948000BF0D6FCCDE9060150460BF06BFC8046F7
:1069580089464246DDE912014B460BF0C9FCDDE9E8
:106968001023CDE91C01DDE914010BF0C1FC002264
:1069780006460F46564BDDE918010BF0B9FC4246B6
:1069880004460D464B46DDE906010BF0B1FC024614
:106998000B460BF0FBFA02460B46204629460BF045
:1069A800F5FA424604460D464B46DDE91C010BF05C
:1069B8009FFC02460B46204629460BF0E5FADDE926
:1069C800102304460D46304639460BF091FC02462A
:1069D8000B46204629460BF0D7FADDF828C0CDE94A
:1069E80002014FEA8C10DDF830C000EB0C20DDF816
:1069F80010C0A0241CFB04000BF004FCDDF838C018
:106A0800CDE90A014FEA8C10DDF858C000EB0C20E4
:106A1800DDF824C01CFB04000BF0F4FBCDE90C01ED
:106A280050460BF0EFFBDDE91023CDE91601DDE957
:106A38000C010BF05DFC4246CDE91E014B46DDE939
:106A48000A010BF055FC4246CDE920014B46DDE931
:106A580000010BF04DFC32463B460BF095FACDE9B0
:106A68000E0158460BF0CEFBDDE91C23CDE91A01D7
:106A7800DDE906010BF088FADDF88CC0C024CDE909
:106A8800060104FB0CF0DDF888C0302505FB0C007E
:106A9800DDF810C078261CFB06000BF0B3FBDDF810
:106AA80094C0824604FB0CF0DDF890C005FB0C0096
:106AB800DDF824C01CFB06008B460BF0A3FBDDE9C8
:106AC800102306460F460BF013FC03E04C0D002084
:106AD800000014404246CDE904014B465046594651
:106AE8000BF006FCDDE9142380468946DDE90A013E
:106AF8000BF0FEFBDDE9002304460D46DDE90C0141
:106B08000BF0F6FB02460B46204629460BF03CFAF2
:106B18000022A14B0BF0ECFBDDE9202304460D46D7
:106B2800DDE91E010BF030FA02460B46DDE91601DD
:106B38000BF0DEFB02460B46204629460BF026FAF0
:106B4800002204460D46954BDDE90E010BF0D0FB03
:106B580002460B46204629460BF018FADDE90223C7
:106B68000BF0F0FC88A3D3E900230BF0C1FB0BF07A
:106B780059FE8B490860DDE91223DDE90C010BF0B1
:106B8800B7FBDDE9002304460D46DDE90A010BF0F9
:106B9800AFFB02460B46204629460BF0F5F90022CA
:106BA8007D4B0BF0A5FBDDE91E2304460D46DDE910
:106BB80020010BF0E9F902460B46DDE91A010BF05A
:106BC80097FB02460B46204629460BF0DFF90022C8
:106BD80004460D46714BDDE906010BF089FB0246C0
:106BE8000B46204629460BF0D1F9DDE902230BF0CC
:106BF800A9FC65A3D3E900230BF07AFB0BF012FE86
:106C0800674A5060DDE90E23DDE90A010BF070FBED
:106C1800DDE9062304460D46DDE90C010BF068FBAF
:106C280002460B46204629460BF0B0F900220446DE
:106C38000D465A4BDDE918010BF05AFB02460B468C
:106C4800204629460BF0A2F9DDE902230BF07AFC75
:106C58004DA3D3E900230BF04BFB0BF0E3FD504BA6
:106C680059469860DDE9142350460BF041FBDDE9F5
:106C7800002304460D46304639460BF039FB0246E0
:106C88000B46204629460BF07FF90022424B0BF0B9
:106C98002FFB424604460D464B46DDE904010BF046
:106CA80073F902460B46DDE916010BF021FB02469B
:106CB8000B46204629460BF069F935A3D3E9002392
:106CC80004460D46DDE90E010BF012FB02460B46A9
:106CD800204629460BF05AF9DDE902230BF032FC75
:106CE80029A3D3E900230BF003FB0BF09BFDDFF88E
:106CF800B0C0DDE91223CCF80C00394630460BF061
:106D0800F7FADDE9002304460D46504659460BF0D4
:106D1800EFFA02460B46204629460BF035F90022C9
:106D28001D4B0BF0E5FADDE9042304460D46404609
:106D380049460BF029F902460B46DDE91A010BF02A
:106D4800D7FA02460B46204629460BF01FF910A336
:106D5800D3E9002304460D46DDE906010BF0C8FA25
:106D680002460B46204629460BF010F9DDE90223BE
:106D78000BF0E8FB04A3D3E900230BF0B9FA0BF0FE
:106D880051FD074908610DE00000000080842E4194
:106D98000000000000C0824000001440000089404C
:106DA8004C0D0020DDE90E23504659460BF0A0FAA1
:106DB800DDE9062304460D46304639460BF098FABD
:106DC80002460B46204629460BF0E0F811A3D3E90A
:106DD800002304460D46DDE918010BF089FA024646
:106DE8000B46204629460BF0D1F8DDE902230BF0CB
:106DF800A9FB0AA3D3E900230BF07AFA0BF012FDE2
:106E0800034A506127B0BDE8F04FC9E4AFF30080F2
:106E18004C0D00200000000000C08240000000006F
:106E280080842E41AFF30080064A074B1A60074A58
:106E3800074B1A60074B42F210721A60064B642225
:106E48001A60704740420F004C26002080C3C901D9
:106E5800642C0020402C0020F8250020012808B5CB
:106E680003D05AD3022851D13CE02C4B1B78012B7C
:106E780003D013D3022B49D121E0294BC82019682C
:106E880000F017FE274BCC20196800F012FE264BA5
:106E9800D020196800F00DFED42033E0204BD82014
:106EA800196800F006FE1F4BDC20196800F001FE8F
:106EB8001D4BE020196800F0FCFDE42022E0184B8F
:106EC800F820196800F0F5FD164BFC20196800F051
:106ED800F0FD154B4FF48070196800F0EAFD4FF48F
:106EE80082700FE00E4BE820196800F0E2FD0D4BB0
:106EF800EC20196800F0DDFD0B4BF020196800F05C
:106F0800D8FDF420094B196800F0D3FD04F0C0FE49
:106F180018B9BDE8084004F0CCBE08BD1C0E00201E
:106F28004C260020642C0020402C0020F82500204E
:106F380008B52E4B1B78012B02D0022B55D140E00F
:106F48002B4B1B78012B03D013D3022B4DD121E0FF
:106F5800C82000F0C7FD274B1860CC2000F0C2FD08
:106F6800254B1860D02000F0BDFD244B1860D420BC
:106F780022E0D82000F0B6FD1E4B1860DC2000F09F
:106F8800B1FD1D4B1860E02000F0ACFD1B4B1860F4
:106F9800E42011E0F82000F0A5FD164B1860FC2055
:106FA80000F0A0FD144B18604FF4807000F09AFDBB
:106FB800124B18604FF4827000F094FD104B18606B
:106FC80008BDE82000F08EFD0A4B1860EC2000F0A8
:106FD80089FD094B1860F02000F084FD074B18600C
:106FE800F42000F07FFD064B186008BDC9010020A1
:106FF8001C0E00204C260020642C0020402C002071
:10700800F825002008B504F043FE10B1BDE808409B
:107018008EE7BDE8084007E7064B07495960C021DD
:10702800002219721E211A70D9601A745A611A76D0
:10703800DA617047481A002040787D0110B50321B5
:10704800FF22C02001F020FC1F4C1021802220606C
:10705800C02001F019FC112180222060C02001F01D
:1070680013FC122180222060C02001F00DFC1321A6
:1070780080222060C02001F007FC142180222060BB
:10708800C02001F001FC152180222060C02001F001
:10709800FBFB802220601621C02001F0F5FB206058
:1070A800C0201721802201F0EFFB80222060B72149
:1070B800C02001F0E9FB054B00221A745A611A76C8
:1070C800DA6101221A7010BD20260020481A00201B
:1070D80038B5C0200321FF2201F0D6FB0B4D002458
:1070E8002B19615D5A78C020023401F0CDFBC82C01
:1070F800F6D1B121AC22C02001F0C6FBC02003218B
:10710800002201F0C1FB002038BD00BF0EA9040811
:107118002DE9F34706460F4692461D461AB90C1F3D
:10712800E401914635E005EE902A06EE903AB8EE75
:10713800657AF8EE667AFC01C7EE277AA4F5007442
:107148009FED5C7A67EE877A17EE900A0BF07CF871
:1071580041EC100B0DF0A8F959EC108B494640464C
:107168000BF088FB24184FEACA100BF04BF8CDE956
:10717800000128460BF046F84B4642460BF0B8F89B
:1071880002460B46DDE900010AF0FEFE0BF072FB39
:107198008146002E14BF4FF022084FF01A08C5F39D
:1071A80007224146C02001F06FFB08F10101EAB255
:1071B800C02001F069FBC4F3014208F10201C020BC
:1071C80001F062FBC4F3072208F10301C02001F0BB
:1071D8005BFBE2B208F10401C02001F055FBC9F3E2
:1071E800034305F4702243EA123208F10501C02076
:1071F80001F04AFB08F10601C9F30722C02001F09B
:1072080043FB08F107015FFA89F2C02001F03CFB5B
:10721800C020B121A02201F037FB07EE107A264CDE
:10722800F8EEC77A0EBBD4ED015A06EE90AAB8EE76
:10723800657A05EE905AB8EE666AF8EE656A01233B
:10724800C6EE266A237477EEA67A67EE277A17EEDB
:10725800900A0AF0F9FF41EC100B0DF025F951ECFA
:10726800100B0BF007FB606120E005EE90AAD4ED4F
:10727800016AB8EE656A05EE905AB8EE667AF8EEDD
:10728800656A0123C6EE266A237677EEA67A67EE4C
:10729800277A17EE900A0AF0D7FF41EC100B0DF091
:1072A80003F951EC100B0BF0E5FAE0610020BDE8A2
:1072B800FC8700BF00000043481A00200022012379
:1072C80026E7012838B50D4604D002280CBF3C2417
:1072D8002C2400E034242146C02001F04FFB05F0A7
:1072E800070200F00F0040EA02122146C020BDE864
:1072F800384001F0C9BA2DE9F3470A9C1D460746F4
:107308008A461646524B01E06D0864089C42FBD839
:107318002DB906F10076043EF601A94634E006EEE2
:10732800905AB8EE667A06EE904AF8EE667AF6015A
:10733800C7EE277AA6F500769FED467A67EE877A3C
:1073480017EE900A0AF080FF41EC100B0DF0ACF834
:1073580059EC108B494640460BF08CFA3618E80178
:107368000AF050FFCDE9000120460AF04BFF4B46DA
:1073780042460AF0BDFF02460B46DDE900010AF06D
:1073880003FE0BF077FA8146022F9BBF324BDB19C5
:107398004FF0000893F8C880C4F307224146C02084
:1073A80001F072FA08F10101E2B2C9B2C02001F09D
:1073B8006BFA08F10201C9B2C6F30142C02001F01C
:1073C80063FA08F10301C9B2C6F30722C02001F02D
:1073D8005BFA08F10401C9B2F2B2C02001F054FA14
:1073E80004F47024C9F3034308F1050143EA143295
:1073F800C9B2C02001F048FA08F10601C9B2C9F3C0
:107408000722C02008F1070801F03EFA5FFA89F266
:107418005FFA88F1C02001F037FABAF1010F0CBF0A
:107428002F220F220DB942F04002012F06D002D3BD
:10743800022F0AD105E0C020102104E0C02011214C
:1074480001E0C020122101F01FFA0020BDE8FC87EE
:10745800FFFF0F00000000430EA9040807B5012331
:1074680000930023FFF747FF0EBD00280CBFFF2243
:10747800002208B5C020032101F006FA002008BD4B
:1074880008B5C020B121AC2201F0FEF9002008BDEA
:1074980008B50420012109F025FB4FF48070012173
:1074A800BDE8084009F04EBB07B50223009303234B
:1074B8008DF804300348002369468DF8073008F03A
:1074C80069FF0EBD0008024030B5124D8BB0002494
:1074D80006A8069407940894099408F029F90094DA
:1074E8008DF804408DF805400294039404942846CE
:1074F800012469468DF8144008F0EBF828460B2162
:107508002246062308F060F92846214608F02AF9A1
:107518000BB030BD0020014010B500210446012207
:10752800302001F0B1F9C0B9012001F0A7FC002C0E
:10753800B8BF4034E4B210212246302001F0A4F94B
:10754800012001F09BFC30201121224601F09CF91A
:107558000120BDE8104001F091BC10BD10B500211C
:1075680004460122302001F08FF9C0B9012001F052
:1075780085FC002CB8BF4034E4B2122122463020EA
:1075880001F082F9012001F079FC30201321224614
:1075980001F07AF90120BDE8104001F06FBC10BD80
:1075A80038B5012205460C463020002101F06CF95F
:1075B800F0B9012001F062FC25EAE5725F2AA8BF54
:1075C8005F223B21D2B2302001F05EF9012001F0A8
:1075D80055FC24EAE4725F2AA8BF5F22D2B23020A9
:1075E8003C2101F051F90120BDE8384001F046BCCA
:1075F80038BD302810B504460ADC10F17F0F02DBD5
:10760800002802DB05E06FF07E0404F5807400E0DA
:107618003024002130200A4601F036F9A8B90120AB
:10762800E4B201F02BFC41212246302001F02CF974
:10763800012001F023FC30204221224601F024F9E8
:107648000120BDE8104001F019BC10BD282810B574
:10765800044609DC10F1180F02DB002802DB04E005
:107668006FF017047F3400E02824002130200A46F8
:1076780001F00AF9A8B90120E4B201F0FFFB532197
:107688002246302001F000F9012001F0F7FB3020FC
:107698005421224601F0F8F80120BDE8104001F01D
:1076A800EDBB10BD08B530200021012201F0ECF837
:1076B80060B9012001F0E2FB30203321402201F0C3
:1076C800E3F80120BDE8084001F0D8BB08BD10B5BB
:1076D80030200021012201F0D7F8044660B90120CA
:1076E80001F0CCFB30203321224601F0CDF80120F7
:1076F800BDE8104001F0C2BB10BD10B5302000211C
:10770800012201F0C1F80446A0B9012001F0B6FB3E
:1077180034212246302001F0B7F8012001F0AEFBF9
:1077280030203721224601F0AFF80120BDE8104093
:1077380001F0A4BB10BD4020EEE640200EE708B5DE
:1077480000210122302001F09FF8012001F096FB72
:1077580030203421024601F097F8012001F08EFB19
:1077680030203721024601F08FF80120BDE808409B
:1077780001F084BB08B500210122302001F084F813
:10778800012001F07BFB302034210C2201F07CF831
:107798000120BDE8084001F071BB000000000000B6
:1077A8002DE9F04F984B994A1968994B002914BF55
:1077B80091469946974B2DED048BC3F80090964B54
:1077C8000025002287B01A80AA46AB46A8465AE090
:1077D800A2004046CDF804C002920AF035FD0746E3
:1077E800584601F100460AF02FFD02460B4638467E
:1077F80031460AF0C9FB39F9243007EE103AF8EEA1
:10780800C77A064617EE900A0F460AF01DFD024693
:107818000B46304639460AF0B9FB0BF04BF80746E1
:1078280050460AF011FD0446284601F100460AF0C8
:107838000BFDCDE90401DDE90423204631460AF0B9
:10784800A3FB029A09EB02030446B3F9023007EEE0
:10785800103AF8EEC77A0D4617EE900A0AF0F4FCD3
:1078680002460B46204629460AF090FB0BF022F808
:10787800DDF804C0684A0CF1010CC3465546A2F86D
:1078880000C08246B846644BB3F800C00FFA8CF4C7
:10789800B32C9DDD58460AF0D7FCCDE902014046DD
:1078A8000AF0D2FC002206460F465C4BDDE90201D5
:1078B8000AF01EFD02460B46304639460AF066FBC2
:1078C8000022574B0AF03EFE0AF0F4FF4CA3D3E91E
:1078D800002309EE900ADDE902010AF009FD002201
:1078E8004F4B0AF02FFE0AF0E5FF09EE100A284672
:1078F8000AF0AAFC044650460D460AF0A5FC0022F0
:1079080006460F4620462946444B0AF0F1FC02463B
:107918000B46304639460AF039FB0022404B0AF044
:1079280011FE0AF0C7FF36A3D3E9002308EE900A38
:10793800294620460AF0DCFC0022394B0AF002FEF8
:107948000AF0B8FF08EE100A69EE287A58EE297A8C
:1079580017EE900A0AF078FC68EE097A48EEA97AE0
:10796800044617EE900A0D460AF06EFC45EC104BE3
:1079780041EC110B0CF09CFE51EC100B0AF09AFF35
:1079880028EE088A08EEA88A07EE100A254B264C2E
:10799800F1EE477AC3ED007A18EE100A0AF054FCAB
:1079A80041EC100B0CF092FF29EE099A51EC100BE8
:1079B80009EEA99A0AF07EFF206019EE100A0AF073
:1079C80043FC41EC100B0CF081FF51EC100B0AF05A
:1079D80071FFD4ED007A07EE100A87EE877A134B11
:1079E8001860134BFDEEE77A83ED007A114BC3ED77
:1079F800007A07B0BDEC048BBDE8F08FAFF30080D0
:107A0800912B50E67AB6EB3F701A0020F222002044
:107A1800521D00206C1A0020781A00200000E03F58
:107A280000005940682C0020802C0020742C002075
:107A3800702C0020741A002010B5084C204608F05D
:107A4800F6F8074B1860FFF7ABFE064B0649012214
:107A580020461A80BDE8104008F06AB9106002405C
:107A6800701A0020680D002020800010014B186853
:107A7800704700BF741A002038B505460C4601351A
:107A8800C1F3072101F008FAA8B2E1B201F004FA43
:107A980000B238BD38B5044601F038F8013405465F
:107AA800A0B201F033F8EDB2C0B240EA052000B24E
:107AB80038BD37B50B0E8DF804300B0C8DF805303A
:107AC8000B0A8DF806308DF80710002400E02846D0
:107AD80001AB451CE15C013401F0DEF9042CADB2C8
:107AE800F5D13EBD37B5002400E02846451C01F01D
:107AF8000DF801ABADB2E0540134042CF5D19DF87A
:107B080005009DF80430000440EA03609DF8073042
:107B180018439DF8063040EA03203EBD37B50023E0
:107B28000193002400E02846451C00F0EFFF01AB5C
:107B3800ADB2E0540134042CF5D19DED010A3EBDEF
:107B48007047000038B50446642001F097F925789D
:107B58006068AD00EDB2257008F081FC237A40FA28
:107B680003F000F003000543104B257005F00F05E6
:107B78005A5D6378D218D2B2D3B20132D2B2022A95
:107B8800637001D80022A2705BB2012B03DD0123D0
:107B9800A3700023637094F90130013303DAFF23E3
:107BA800A3700023637094F9020038BDDAA90408B1
:107BB800F7B504200121234F08F094FF02AD0121FD
:107BC8004FF48040012408F0BDFF00264FF4B07345
:107BD8003846694645F8083D8DF804608DF8074039
:107BE80008F0D8FB1020214608F07CFF782369466E
:107BF800154800938DF804608DF8074008F0CAFB1B
:107C08000420214608F06EFF21464FF4804008F01A
:107C180099FF1C233846694600938DF804608DF857
:107C2800074008F0B7FB0220214608F05BFFB023AD
:107C380006488DF8046069468DF80740009308F0FF
:107C4800A9FBFEBD000802400010024000040240EB
:107C5800802108B5034808F0FCFBD0F1010038BFCB
:107C6800002008BD0004024008B54FF480710448A4
:107C780008F0EFFBD0F1010038BF002008BD00BFBD
:107C88000008024008B5FFF7E3FF08B1FFF7ECFF73
:107C9800C0B208BD70B500283AD01E4B1A788018BB
:107CA8001D4AC0B292F90020187040B282421B4AA5
:107CB80002DD11780139197093F9001092F900204A
:107CC80091FBF2F402FB14141549E4B21C700A8803
:107CD800144B1A80144B154A18881080144A92F9CC
:107CE800000064B2013094FBF0F200FB1240114C2A
:107CF8002688114C258800FB065008800F49088803
:107D08000F49098802FB00121A800E4B01221A70D3
:107D180070BD00BF0E3A002039360020153600200D
:107D2800443A00205A3600200C3A00200C38002033
:107D3800463A002068370020A83A0020D43A0020AC
:107D4800EA37002014360020F0B5264A264C0023D6
:107D58001370264A25681678254A12680FE0D45C05
:107D68002F197F7817F0040F07D0302C02D1202369
:107D7800135431E01B4A137003E00133DBB29E4217
:107D8800EDDA184B1B788342194B16D9A9B11A683A
:107D9800164C3121115430210BE01A681518125C69
:107DA8002E2A19D0303AD2B2092A88BF2970013058
:107DB800C0B222788242F0DA0EE01B681A5C79B110
:107DC8002E2A0DD05118C9B2392903D82F2998BFA6
:107DD800302100E039211954BDE8F040FCF788BC97
:107DE800F0BD00BF6C0D002048030020C83B0020F8
:107DF800303A002010B5642001F040F88248FFF7BF
:107E0800A1FE824B1B7804460C2B00F25F81DFE851
:107E180013F00D000D005D017500750037008C0032
:107E28008C00B700BA00D4008C003901FFF71CFFA2
:107E380018B10120F9F77AFD48E1754B1888754BA0
:107E48001B88C01A744B1B8890FBF3F0734B1A887D
:107E5800734B1B88D31A734A128893FBF2F3DBB275
:107E6800C0B2032B00F2CC80DFE803F0020406085E
:107E78006D4A40E06D4A3EE06D4A3CE06D4A3AE0AA
:107E8800FFF7F2FED8B100210A226B4810F0BEF9C4
:107E98006A4B002118600A22694810F0B7F9694B4B
:107EA80018600420FEF762F996200521664A00232F
:107EB800FEF794F90020FEF759F906F0EBFF544B52
:107EC8001888544B1B88C01A534B1B8890FBF3F03F
:107ED800524B1A88524B1B88D31A524A128893FB6A
:107EE800F2F3DBB2C0B21BB1012B40F0898001E094
:107EF800514A00E0524A554B1A6081E0002800F0D0
:107F0800E580534B1A7806DD0132D2B2102A1A7076
:107F180008D9112205E0013AD2B2112A1A7001D902
:107F280000221A70F9F7CAFED0E0002800F0CE80CF
:107F3800484B1A788418E4B20322B4FBF2F102FB2E
:107F48001144E4B21C70444B444A1B5D022B13706D
:107F580009D0052B0CD0012B40F0B8804FF491705C
:107F680069213F4A08E04FF4917069213D4A03E0D6
:107F78003D4A4FF4917069210023FEF72FF9A5E0DF
:107F88003A4B1870A2E0FFF76FFEA0B10021384805
:107F980010F088F8374B042083ED000AFEF7E6F866
:107FA800B4200521344A0023FEF718F9FAF792FAAB
:107FB8000020FEF7DBF82E4A16E0FFF755FE90B1D9
:107FC80000212E4810F06EF82D4B042083ED000A96
:107FD800FEF7CCF896200521274A0023FEF7FEF885
:107FE8000020FEF7C3F8254A184B1A60084B18887A
:107FF800084B1B88C01A084B1B8890FBF3F0C0B2D3
:108008002146FFF7A1FE61E0A8010020CD25002050
:10801800443A0020A83A0020683700200C3A002093
:10802800EA370020D43A0020102600203426002009
:108038004A2C0020FC250020B03A0020C401002072
:10804800203A0020C001002095AE0508303A0020F3
:1080580046260020D50D0020300300201C030020F8
:10806800A5AE0508A8AE0508ABAE05083C3A002049
:108078002C36002024030020AEAE05085036002020
:1080880020030020FFF7F0FD08B107F0DBF814B17A
:10809800254B01221A70254B1A68A41814F5967FEF
:1080A800B8BF234A1C60B8BF1A601B68B3F5967F37
:1080B80003DD1E4B4FF496721A601B4C23782BB1CC
:1080C8001C4B186801F0DAFA002323701A48FFF7EE
:1080D80039FD1A4B1B78013B0A2B24D8DFE803F043
:1080E800062323232015152311111500FFF7D2FDB0
:1080F800FFF7AEFD002816D00220BDE81040F9F7C2
:1081080015BC0F4B1B78022B0AD100280D4B01D14F
:10811800187010BD01DD012200E0FF221A7010BDA9
:10812800BDE81040B6E510BD48260020403A0020C2
:10813800D4FEFFFFEC250020B4010020CD2500204F
:1081480034380020811A002010B58CB01E490F2247
:1081580068460EF049FE1D490F2204A80EF044FEA1
:108168001B490F2208A80EF03FFE002108223020EC
:1081780000F08AFB012000F081FE002404AB1DF80A
:108188000420E15C302000F07FFB0134012000F086
:1081980075FE0F2CF2D100210922302000F074FB6B
:1081A800012000F06BFE002408AB1DF80420E15C00
:1081B800302000F069FB0134012000F05FFE0F2C35
:1081C800F2D10CB010BD00BFECA90408FBA904084B
:1081D8000AAA040810B58CB01E490F2268460EF092
:1081E80003FE1D490F2204A80EF0FEFD1B490F22B5
:1081F80008A80EF0F9FD00210822302000F044FB09
:10820800012000F03BFE002404AB1DF80420E15CD3
:10821800302000F039FB0134012000F02FFE0F2C34
:10822800F2D100210922302000F02EFB012000F0BD
:1082380025FE002408AB1DF80420E15C302000F086
:1082480023FB0134012000F019FE0F2CF2D10CB0F1
:1082580010BD00BF19AA040828AA040837AA0408F0
:1082680010B58CB01E490F2268460EF0BDFD1D49A1
:108278000F2204A80EF0B8FD1B490F2208A80EF023
:10828800B3FD00210822302000F0FEFA012000F0A2
:10829800F5FD002404AB1DF80420E15C302000F05B
:1082A800F3FA0134012000F0E9FD0F2CF2D100218E
:1082B8000922302000F0E8FA012000F0DFFD002458
:1082C80008AB1DF80420E15C302000F0DDFA013431
:1082D800012000F0D3FD0F2CF2D10CB010BD00BF6F
:1082E80046AA040855AA040864AA040807B5022087
:1082F800012108F0F7FB012300938DF804300223D5
:108308008DF805300448002369468DF806308DF84D
:10831800073008F03FF80EBD0004024010B5084CC5
:1083280001210022204608F0AAF840F2FF4000F0A0
:10833800A5FD012120460A46BDE8104008F09FB877
:108348000004024008B5FFF7E9FF00210A46302083
:1083580000F09AFA012000F091FD01210A46302030
:1083680000F092FA012000F089FD0021012230205E
:1083780000F08AFA012000F081FD01210822302056
:1083880000F082FA012000F079FD0221012230205C
:1083980000F07AFA012000F071FD00210A46302031
:1083A80000F072FA012000F069FD1B21CD22302077
:1083B80000F06AFA012000F061FD04210322302058
:1083C80000F062FA012000F059FD06210922302050
:1083D80000F05AFA012000F051FD07210822302050
:1083E80000F052FA012000F049FD082170223020E7
:1083F80000F04AFA012000F041FD1E213020B02291
:1084080000F042FA012000F039FD052191223020C8
:1084180000F03AFA012000F031FD0D21032230204E
:1084280000F032FA012000F029FD0E210022302050
:1084380000F02AFA012000F021FD142180223020CA
:1084480000F022FA012000F019FD0B2188223020CB
:1084580000F01AFA012000F011FD0C2182223020D0
:1084680000F012FA012000F009FD122188223020C4
:1084780000F00AFA012000F001FD13218C223020BF
:1084880000F002FA012000F0F9FC00210A46302031
:1084980000F0FAF9012000F0F1FC3D210222302021
:1084A80000F0F2F9012000F0E9FCFFF74DFEFFF7BC
:1084B80091FEFFF7D5FE30200021012200F0E4F9FB
:1084C800012000F0DBFC3D216422302000F0DCF9C3
:1084D800012000F0D3FC03210022302000F0D4F961
:1084E800012000F0CBFC04210022302000F0CCF960
:1084F800012000F0C3FC00210122302000F0C4F963
:10850800012000F0BBFC0C210822302000F0BCF94F
:10851800012000F0B3FC0D210822302000F0B4F94E
:10852800012000F0ABFC0E210822302000F0ACF94D
:10853800012000F0A3FC0F210822302000F0A4F94C
:10854800012000F09BFC00210A46302000F09CF935
:10855800012000F093FC02224021302000F094F921
:10856800012000F08BFC30204121002200F08CF922
:10857800012000F083FC3F21D422302000F084F950
:10858800012000F07BFC00210122302000F07CF962
:10859800012000F073FC10210F22302000F074F944
:1085A800012000F06BFC11210F22302000F06CF943
:1085B800012000F063FC12210022302000F064F951
:1085C800012000F05BFC13210022302000F05CF950
:1085D800012000F053FC09213C22302000F054F91E
:1085E800012000F04BFC00210122302000F04CF962
:1085F800012000F043FC30203421024600F044F909
:10860800012000F03BFC30203721024600F03CF905
:10861800012000F033FC36210322302000F034F929
:10862800012000F02BFC39210322302000F02CF926
:10863800012000F023FC3B213C22302000F024F9EB
:10864800012000F01BFC3C210A46302000F01CF9F8
:10865800012000F013FC00210A46302000F014F934
:10866800012000F00BFC5121C022302000F00CF951
:10867800012000F003FC52213020002200F004F910
:108688000120BDE8084000F0F9BB00BF2DE9F04F1C
:10869800454E464D93B001214FF4001008F022FAE0
:1086A800304607F0C5F94FF0C0630293404B03937F
:1086B800404B002404934FF4B4794FF400334FF443
:1086C80080684FF400674FF4005A4FF4807B3046BF
:1086D80002A90C9301930997CDF818900594079473
:1086E800CDF82080CDF828A0CDF82CB00D9407F057
:1086F8002BFA22463046304907F081FA30460121EC
:1087080007F087FA01210A464FF0402008F058FC8C
:10871800284607F08DF9294A019B0392284A0C93B1
:1087280004922846402202A9059209970294CDF89E
:1087380018900794CDF82080CDF828A0CDF82CB05B
:108748000D9407F001FA224628461E4907F057FA09
:108758002846012107F05DFA42F210770122022132
:10876800194808F02DFC384600F088FB30460121F6
:1087780007F025FA0121284607F021FA384600F0CB
:108788007DFB0B238DF8443011A801238DF845405B
:108798008DF846408DF8473000F08EFD384600F0E1
:1087A8006DFB13B0BDE8F08F106002408860024096
:1087B8000C400040F2220020521D00200C3C0040DA
:1087C80022200020821A0020003C0040024810218C
:1087D800012207F06BBA00BF1060024013B50220F7
:1087E800012108F07FF94FF410730E4C0093022317
:1087F8008DF804308DF8053001238DF806302046B9
:10880800002369468DF8073007F0C4FD204606218D
:10881800042207F03FFE20460921042207F03AFE11
:108828001CBD00BF0004024030B5154D85B00121C4
:108838004FF4001008F07AF9284607F041FE0023AB
:10884800ADF804304BF6FF73ADF806303323ADF8BE
:1088580008304FF48063ADF80A304FF48043ADF828
:108868000C3004AC074B2846012144F8103D07F0B2
:10887800C9FE2846694607F051FE05B030BD00BF65
:1088880000540040801A060073B54FF4961306464C
:108898000D461446019304E0019B5A1E0192002BD9
:1088A80057D031484FF4003107F0C4FF0028F3D106
:1088B8002D48012107F0B2FE4FF48053019304E0E4
:1088C800019B5A1E0192002B45D02748274907F0E3
:1088D8009CFF0028F4D024483146002207F0B6FE59
:1088E8004FF48053019304E0019B5A1E0192002B20
:1088F80033D01D481E4907F088FF0028F4D01A48D5
:10890800294607F026FF4FF48053019303E0019BAB
:108918005A1E01921BB31448164907F076FF002827
:10892800F5D01148214607F014FF4FF49613019330
:1089380003E0019B5A1E01929BB10B480E4907F0B8
:1089480079FF0028F5D00848012107F073FE0020C0
:1089580008E0012006E0022004E0032002E00420F1
:1089680000E005207CBD00BF00540040010003006A
:1089780082000700800007000400001037B54FF49C
:10898800961304460D46019305E0019B5A1E019279
:10899800002B00F09B8056484FF4003107F04AFF47
:1089A8000028F2D15248012107F038FE4FF48053D5
:1089B800019305E0019B5A1E0192002B00F088806C
:1089C8004B484C4907F021FF0028F3D0484821467E
:1089D800002207F03BFE4FF48053019304E0019B13
:1089E8005A1E0192002B75D04148434907F00DFFEC
:1089F8000028F4D03E48294607F0ABFE4FF48053D8
:108A0800019304E0019B5A1E0192002B64D0384860
:108A18003A4907F00FFF0028F4D03548012107F044
:108A2800FDFD4FF48053019304E0019B5A1E01920F
:108A3800002B53D02E482F4907F0E7FE0028F4D02A
:108A48002B482146012207F001FE4FF48053019381
:108A580004E0019B5A1E0192002B41D0244C284966
:108A6800204607F0E7FE0028F3D02046002107F053
:108A7800F5FD20460121238B07F0DCFD4FF48053E0
:108A8800019304E0019B5A1E0192002B2AD018483A
:108A98001C4907F0CFFE0028F4D0154807F05BFE0C
:108AA8004FF480530193124A03E0019B591E019130
:108AB800D3B113889B05F8D4012104460C4807F06C
:108AC800CDFD0B48104907F0CFFE0EE001240CE065
:108AD80002240AE0032408E0042406E0052404E054
:108AE800062402E0072400E0082420463EBD00BF1B
:108AF8000054004001000300820007000400001039
:108B080002000010400000100004001013B54FF4DC
:108B180096130446019305E0019B5A1E0192002B0F
:108B280000F0AF8060484FF4003107F083FE002862
:108B3800F2D15D48012107F071FD4FF48053019394
:108B480005E0019B5A1E0192002B00F09C805648BC
:108B5800564907F05AFE0028F3D05348A0210022B6
:108B680007F074FD4FF48053019305E0019B5A1EF2
:108B78000192002B00F089804B484D4907F045FED3
:108B88000028F3D0210A484807F0E3FD4FF480534A
:108B9800019304E0019B5A1E0192002B77D04248B2
:108BA800444907F047FE0028F4D0E1B23E4807F0F8
:108BB800D0FD4FF48053019304E0019B5A1E0192AB
:108BC800002B66D038483B4907F034FE0028F4D023
:108BD8003548012107F022FD4FF48053019304E04A
:108BE800019B5A1E0192002B55D02F482F4907F0A0
:108BF8000CFE0028F4D02C48A121012207F026FD04
:108C08004FF48053019304E0019B5A1E0192002BFC
:108C180043D0254C2849204607F00CFE0028F3D005
:108C28002046002107F01AFD20460121238B07F07A
:108C380001FD4FF48053019304E0019B5A1E0192F9
:108C4800002B2CD018481D4907F0F4FD0028F4D05B
:108C5800154807F080FD4FF480530193124A03E052
:108C6800019B591E0191E3B113889905F8D401219C
:108C780004460D4807F0F2FC0B48114907F0F4FDD3
:108C880010E001240EE002240CE003240AE004248E
:108C980008E0052406E0062404E0072402E008248E
:108CA80000E0092420461CBD0054004001000300D8
:108CB80082000700040000100200001040000010AD
:108CC8000004001013B54FF496130446019305E011
:108CD800019B5A1E0192002B00F0AF8060484FF4B0
:108CE800003107F0A7FD0028F2D15D48012107F007
:108CF80095FC4FF48053019305E0019B5A1E0192A5
:108D0800002B00F09C805648564907F07EFD00284D
:108D1800F3D05348A021002207F098FC4FF4805369
:108D2800019305E0019B5A1E0192002B00F08980F7
:108D38004B484D4907F069FD0028F3D0210A4848FF
:108D480007F007FD4FF48053019304E0019B5A1E7E
:108D58000192002B77D04248444907F06BFD002868
:108D6800F4D0E1B23E4807F0F4FC4FF4805301938D
:108D780004E0019B5A1E0192002B66D038483B49FB
:108D880007F058FD0028F4D03548012107F046FCCB
:108D98004FF48053019304E0019B5A1E0192002B6B
:108DA80055D02F482F4907F030FD0028F4D02C4823
:108DB800A121012207F04AFC4FF48053019304E0FB
:108DC800019B5A1E0192002B43D0254C284920466E
:108DD80007F030FD0028F3D02046002107F03EFCC4
:108DE80020460121238B07F025FC4FF48053019383
:108DF80004E0019B5A1E0192002B2CD018481D49F3
:108E080007F018FD0028F4D0154807F0A4FC4FF42B
:108E180080530193124A03E0019B591E0191E3B16B
:108E280013889C05F8D4012104460D4807F016FC68
:108E38000B48114907F018FD10E001240EE0022448
:108E48000CE003240AE0042408E0052406E00624D4
:108E580004E0072402E0082400E0092420461CBDA1
:108E680000540040010003008200070004000010C5
:108E780002000010400000100004001082B000231F
:108E880004E0019B01330193009B01330093009B95
:108E98008342F6D302B0704737B54FF48053044687
:108EA8000D46019304E0019B5A1E0192002B6DD0E0
:108EB8003C484FF4003107F0BDFC0028F3D1394895
:108EC800012107F0ABFB4FF48053019304E0019BB1
:108ED8005A1E0192002B5BD03248334907F095FCAB
:108EE8000028F4D02F48A021002207F0AFFB4FF450
:108EF8008053019304E0019B5A1E0192002B49D034
:108F080028482A4907F081FC0028F4D0210A25487E
:108F180007F01FFC4FF48053019304E0019B5A1E95
:108F28000192002B38D01F48214907F06EFC002819
:108F3800F4D0E1B21B4807F00CFC4FF480530193C6
:108F480003E0019B5A1E019243B31648184907F0E3
:108F58005CFC0028F5D01348294607F0FAFB4FF4CB
:108F68009613019303E0019B5A1E0192C3B10D4869
:108F7800104907F05FFC0028F5D00A48012107F0E6
:108F880059FB0D48FFF77AFF00200AE0012008E0AE
:108F9800022006E0032004E0042002E0052000E0AF
:108FA80006203EBD00540040010003008200070077
:108FB8008000070004000010A0860100F7B54FF4F8
:108FC800805304460D461646019304E0019B5A1E41
:108FD8000192002B74D040484FF4003107F02AFC6E
:108FE8000028F3D13C48012107F018FB4FF48053C7
:108FF800019304E0019B5A1E0192002B62D036486F
:10900800364907F002FC0028F4D03348A02100229A
:1090180007F01CFB4FF48053019304E0019B5A1E98
:109028000192002B50D02C482D4907F0EEFB002868
:10903800F4D0210A284807F08CFB4FF480530193A1
:1090480004E0019B5A1E0192002B3FD0224825497B
:1090580007F0DBFB0028F4D0E1B21F4807F079FBEA
:109068004FF48053019304E0019B5A1E0192002B98
:109078002ED019481B4907F0C8FB0028F4D000245B
:109088004FF4961710E0295D134807F062FB01972B
:1090980003E0019B5A1E0192E3B10F48124907F001
:1090A800C9FB0028F5D00134E3B2B342EBD30A4838
:1090B800012107F0BFFA0D48FFF7E0FE00200AE0A3
:1090C800012008E0022006E0032004E0042002E07A
:1090D800052000E00620FEBD00540040010003000A
:1090E800820007008000070004000010A08601002D
:1090F80013B50520012107F0F5FC184C4FF4E05397
:10910800009302238DF804308DF8053020460023A3
:1091180069468DF806308DF8073007F03BF9204690
:109128000A21062207F0B6F920460C21062207F08C
:10913800B1F9062220460B21A4F5006407F0AAF92C
:109148004FF4004320466946009307F023F9204670
:109158000F21062207F09EF91CBD00BF000802403F
:109168001FB50446FFF7C2F8FFF75EFBFFF7EAF802
:10917800FFF7BEFF01214FF4004007F0D7FC02942F
:109188000F4C1023ADF80230204600236946ADF895
:109198000430ADF80C30ADF80030ADF8063007F00B
:1091A800F4FD69464FF0402007F0C3FE2046012138
:1091B80007F073FE4FF04020012107F06EFE1FBD3F
:1091C800003C004082B0002304E0019B013301937E
:1091D800009B01330093009B8342F6D302B0704793
:1091E80007B50420012107F07DFC01214FF48040E0
:1091F80007F0A8FC4FF40073009300238DF80430A7
:109208000348012369468DF8073007F0C3F80EBDFF
:10921800000802400D4B07B51A680D484FF47A73E1
:10922800B2FBF3F20B4B013A5A600B4AF02182F879
:10923800231000229A6007221A60084B084A0093FC
:109248000121084B01F0F8FF0EBD00BFE40100202A
:109258005026002010E000E000ED00E000030020B0
:10926800E40200204C020020054B1A6812B11A686B
:10927800013A1A60034B1A6801321A60704700BF3E
:109288000C2600202426002082B0044B0190019A6D
:109298001A601A68002AFCD102B070470C26002018
:1092A800704700BF40F0BE60024B40F42020D860F9
:1092B800704700BF00ED00E0C37810B503B3164B4C
:1092C8004278DB688478DB43C3F30223C3F10401EB
:1092D800C9B202FA01F10F2242FA03F2C9B22240DE
:1092E8000A430E4B01781201CB18D2B283F800233F
:1092F80003780122590903F01F0302FA03F307E078
:1093080003780122590903F01F0302FA03F32031FD
:10931800024A42F8213010BD00ED00E000E100E013
:1093280021F0604121F07F01014B084398607047AC
:1093380000ED00E0044B1A6909B1104301E022EA8C
:1093480000001861704700BF00ED00E0044B1A6888
:1093580004280CBF42F0040222F004021A6070478D
:1093680010E000E0014B93ED000A7047702C0020DC
:10937800014B93ED000A7047682C0020014B93EDD8
:10938800000A70477C2C0020014B93ED000A7047BF
:109398006C2C0020014B93ED000A7047802C0020B4
:1093A800014B93ED000A7047742C00200000000068
:1093B80008B5FDF743FE0020012324210246FDF7EE
:1093C800A7FE124B1B78013BDBB20020012B05D80E
:1093D8000146FDF776FF0120002104E00721FDF793
:1093E80070FF01200721FDF76CFF63221221C020C6
:1093F800FFF74AFA02200121FDF763FFFEF740F864
:109408000120BDE80840FEF730B800BF1C0E002060
:109418000E4B1B78062B05D10D4B0E4A19681268A6
:109428008A181A600C4B1B78013BDBB2012B084BE6
:10943800196805D8094A914207DD01321A60704758
:10944800074A914201DD01321A607047CD2500209C
:10945800442C0020C42500201C0E00207FD1F008D9
:10946800FF27ED080F4B1B78062B05D10E4B0F4A33
:10947800196812688A1A1A600D4B1B78013BDBB217
:10948800012B094B05D80B4A1968914208DC1A6070
:1094980070471A68B2F57A2FDCBF4FF47A221A6047
:1094A800704700BFCD250020442C0020C425002093
:1094B8001C0E002020A107002DE9F04F6A4B6B4CD1
:1094C8001B688DB019220A9069485343B0FBF1F02C
:1094D8001C190D4608F096FE41EC100B0AF0E4FF4B
:1094E80051EC100B09F0C6F910F0010F804618BFB7
:1094F80000F1FF3805FB08F008F084FE0646204618
:109508000F4608F07FFE02460B463046394609F002
:1095180019F804460D4645EC104B0AF0C5FF57EC08
:10952800106B204632463B46294608F02DFDCDE912
:1095380002013946304609F09DF947A3D3E90023D3
:109548000B90DDE9020109F04FF9002858D10120FC
:1095580000264FF01509314607464FF0000A4FF034
:10956800000B03E030463946069E049FA7FB0A23FA
:10957800541807FB0B333F4A43F100050023A2426E
:10958800AB41CDE904453ED3A6FB0A23141806FBDC
:109598000B33384843F100050021A042A941CDE929
:1095A800064530D3DDE902012DA3D3E90023049C4D
:1095B800069D09F019F940BBDDE9022300202E4978
:1095C80008F0C0FF82468B464BEC10AB0AF06CFFEC
:1095D8005046594653EC102B8DED080B08F0D4FC7F
:1095E800CDE90201DDE9080109F012FC09F1FF39B2
:1095F8005FFA89F982468B46B9F1000FB2D104E0CF
:109608000125002401E035463C460B9A0A9BD1B25D
:109618005BB9184622462B46FDF77AFD0A980123C6
:10962800009301464246034609E022462B460120A4
:10963800FDF76EFD01200090014642460023FDF72C
:109648005AFEFDF71DFF01200DB0BDE8F04FFDF7F4
:109658000CBF00BFAFF30080956479E17FFDA53DA5
:10966800BBBDD7D9DF7CDB3D403A002040787D0187
:1096780000E9A435FFFF0F000000F03F244A254B06
:109688001278013AD2B2012A10B5186009D8224AD4
:10969800904201DD01321A60204A1B6893420DDCBA
:1096A8000AE01F4A904201DD01321A601B68B3F5D7
:1096B8007A2F03DC4FF47A22164B1A60154B194A9D
:1096C8001968194B194C1B68CB18934223601ADC94
:1096D8000020FFF7F1FE01202168FFF7EDFE0C4B9B
:1096E8001B78013BDBB20020012B05D80146FDF7B2
:1096F800E8FD0120002104E00721FDF7E2FD01203B
:109708000721FDF7DEFD034B1A68094B1A6010BDEF
:109718001C0E0020442C00207FD1F00820A1070057
:10972800FF27ED0880D1F0085C2C0020602C002079
:1097380028360020014B1868A0E700BF402600200B
:109748007047FEE7FEE7FEE7FEE7704770477047A1
:1097580002F02EB910B5094CA37A4BB1084B1A6820
:1097680022F006021A6000F013F8204600F041FECD
:109778004FF48020BDE8104006F068BB502600205A
:1097880010ED00E0014801F003B800BF50260020AA
:10979800364BD3F8882042F47002C3F88820344B43
:1097A8001A6842F001021A6000229A60196821F0D2
:1097B800847121F4803119602E495960196882B08A
:1097C80021F480211960DA60009201921A6842F44B
:1097D80080321A601A6802F400320192009A01324B
:1097E8000092019A1AB9009AB2F5A06FF2D1204BF3
:1097F8001B6813F4003318BF01230193019B012B4D
:109808002ED11B4B1A6C42F080521A641A4A116806
:1098180041F4804111609A689A609A6842F4004263
:109828009A609A6842F4A0529A60144A5A601A6878
:1098380042F080721A6019680D4A8901FBD5104BF5
:1098480040F205611960936823F0030393609368FD
:1098580043F002039360936803F00C03082BFAD1DA
:10986800024B4FF000629A6002B0704700ED00E0D2
:1098780000380240103000240070004008544007AF
:10988800003C0240184B194A996801F00C01042960
:1098980003D0082903D0164B19E0164B17E0596876
:1098A8005A6811F4800F596814BF124B104B02F01C
:1098B8003F02B3FBF2F30C4A5268C2F30142C1F310
:1098C8008811013252004B43B3FBF2F3074A13608D
:1098D800054B9A68054BC2F303129A181968127956
:1098E80021FA02F21A60704700380240E4010020B1
:1098F8000024F40000127A0037B51C230124002547
:1099080001A88DF804308DF805508DF806408DF8C3
:109918000740FFF7D1FC2046214607F007F90A491E
:1099280040F2E1434B6040F24F130B800D814D80B4
:109938004FF0804007F0A2FC4FF0804021462246BD
:1099480008F061F83EBD00BF842C002008B54FF038
:109958008040012108F06CF860B101214FF080408F
:1099680008F071F8FEF746FA034B044A11781A78A2
:109978008A181A7008BD00BFF02500203C3A002064
:1099880008B5402006F054FA30B1FCF785FD4020B8
:10999800BDE8084006F05ABA08BD0000014608B5FF
:1099A800044808F00FFA0348402108F0B8FA0028E4
:1099B800F9D008BD00440040F0B589B04FF4E13358
:1099C8000120019300232B4CADF808301E460146B8
:1099D800ADF80A30ADF80C30ADF810300C23ADF806
:1099E8000E3007F07FF84FF40030012107F09EF8A1
:1099F80020680221072206F04DFD07226068032136
:109A080006F048FD0125022704232068059305A9CF
:109A18008DF81A608DF81B508DF818708DF8197034
:109A280006F0B8FC08236068059305A98DF818703E
:109A380006F0B0FCA06801A908F01AF92A4640F21D
:109A480025510D4808F052FA262307A88DF81C3036
:109A58008DF81D608DF81E608DF81F50FFF72CFCE7
:109A6800A068294608F081F9044A054B1A6009B034
:109A7800F0BD00BFF801002000440040A59900088F
:109A8800CC3B0020024B9868002108F06EB900BF5B
:109A9800F801002010B5094C40F22551204608F085
:109AA80048FA50B1A288D2B2112A02D1044B01213E
:109AB8001970044B19884A401A8010BD00440040B0
:109AC8007D0D0020880D00207047704773B5012078
:109AD800014607F007F8264C4FF4D85300930223A9
:109AE80003268DF804302046002369468DF8063099
:109AF8008DF807308DF8056006F04CFC20460821EB
:109B08000A2206F0C7FC204609210A2206F0C2FCF8
:109B180020460B210A2206F0BDFC0A2220460C2111
:109B280006F0B8FC01254FF480632046694600938F
:109B38008DF806508DF807508DF8056006F02AFC60
:109B48000A210A46204606F0A5FC29464FF4804023
:109B580006F0F8FF8020294606F0D0FF4FF080502D
:109B6800294607F01FF8284606F070F97CBD00BFAB
:109B78000000024007B54FF4C060FFF793FB432392
:109B88008DF804300322012301A88DF805308DF8E3
:109B980006208DF80730FFF78FFB0EBD782358435A
:109BA8000723B0FBF3F0002301338342FCD970474D
:109BB8004FF47A735843F1E737B50023104C0193FB
:109BC80005460320FFF7EAFFEB681A69013C01929A
:109BD80013D0019A002AF4DA019A42F001020192A4
:109BE800019A1A61064A1969013A019102D001994C
:109BF800C907F8D40320FFF7D1FF00203EBD00BFFE
:109C0800410D030010B5C47874B900EB820003332A
:109C18009B10D0F8D000224603E051F8044C0132E2
:109C2800046004319A42F8D1002010BD033230B5E7
:109C38009210D0F8D0400B46002003E02568013090
:109C480043F8045C04339042F8D101EB800030BD46
:109C58000122F0B50023827040220129C37082805E
:109C68000CD108230370042343704FF4A073C380FE
:109C780002230372C1724FF0A04309E041B90C23DB
:109C88000370062343704FF4A063C3801F4BC17257
:109C980003F500620261C3604678044601461A462D
:109CA800002508E002F5106C02F530620A65C1F87B
:109CB80014C001353A460431B54202F12007F1D308
:109CC80003F58062426103F58862C0F8CC2006780B
:109CD80003F5A0650146002203E0C1F88C5001326B
:109CE80020350431B242F8D31946002202E0C4F804
:109CF800CC1001320434B24201F58051F7D303F598
:109D08006063C0F80C310020F0BD00BF00000440C3
:109D180038B5037AC2680025012B044625D1936B18
:109D2800417A65F3104309B143F480139363D36810
:109D380023F4800323F0500343F010036FF3C303AD
:109D48006FF3C7136FF351436FF3D343D3602046C8
:109D5800FFF732FFE378012B3ED1052363F3440577
:109D6800E36845F020059D6036E0D36843F0400382
:109D7800D360FFF721FF237A627A032B14BF4FF4D5
:109D880034134FF43C130AB143F48013E2681420EF
:109D98009363FFF70DFFE268217AD368032908BFB0
:109DA80043F48033D360237A032B15D1156B012339
:109DB80063F39B656FF3D7552D2345F0805563F307
:109DC80016451563C820FFF7F3FEE36845F4000560
:109DD8001D63C820FFF7ECFEE378012B07D1E36889
:109DE8009D68052262F3440545F020059D6000202A
:109DF80038BDC3689A6842F001029A600020704733
:109E0800C3689A6822F001029A600020704707B57B
:109E180000230193019B43F020030193019B61F30D
:109E28008A130193019BC2681361064B1169013BB8
:109E3800019102D001998806F8D40320FFF7AEFEFD
:109E480000200EBD410D030007B500230193019BBF
:109E580043F010030193019BC2681361064B11691B
:109E6800013B019102D00199C906F8D40320FFF7FC
:109E780095FE00200EBD00BF410D030008B5C26865
:109E8800D36801296FF35D736FF39E7302D143F0BA
:109E9800005302E009B943F080433220D360FFF752
:109EA80087FE002008BDC368586900F001007047AC
:109EB800C3685B6913F0010F14BF002001207047CD
:109EC800C368586900F001007047C3685A69986907
:109ED80010407047C3685868704703691A6861F38F
:109EE80001021A607047C268002393614FF0FF3384
:109EF8005361536053610B4B9361C3789169002B95
:109F080014BF4FF400634FF4016343F4701343F438
:109F1800405343F0080321EA03010B4393610020F7
:109F2800704700BF00080080F8B5D0F80C31002257
:109F38001A60036915461A6865F3CC221A60C37A59
:109F4800012B04461BD10321FFF7C7FFE3688021DB
:109F58004FF4800261F30F0259629A62C02262F3E1
:109F68000F0561F31F454FF4A072C3F8045162F363
:109F78000F056FF31F45C3F80851C3F80C511021A2
:109F88002046FFF744FF2046FFF75EFF22690023C3
:109F98004FF0FF311361204653611E469161FF2542
:109FA800D361214610E082691768C7F3076707F095
:109FB8008007FFB2002F14BF4FF0904700271760AB
:109FC800013316610430956062789342EBD3002325
:109FD8001D46FF2010E04A6D1668C6F3076606F0B6
:109FE8008006F6B2002E14BF4FF090460026166089
:109FF800013315610431906062789342EBD3236991
:10A008001A6942F480721A61E278012A04D1054A79
:10A01800402161F359421A632046FFF764FF00208C
:10A02800F8BD00BF0301010003699B68C3F3410346
:10A03800013B022B9ABF024AD05C0320704700BF45
:10A04800A8AA040810B5036981699C680A68C4F362
:10A058004100022802D06FF30A0202E0032060F3F5
:10A068000A020A605A6842F480725A60002010BDE1
:10A0780030B54D780B780022012D00EB830405D113
:10A0880005FA03F3A46963F30F0205E0012505FA55
:10A0980003F3646D63F31F422368C3F3072505F0D8
:10A0A8008005EDB26DB98D6865F30A03CD78C9886E
:10A0B80065F3934361F3995343F0805343F40043AA
:10A0C80023600369D9690A43DA61002030BD30B5DD
:10A0D8004D780B780024012D224600EB830105D131
:10A0E80005FA03F3896963F30F0205E0012505FA10
:10A0F80003F3496D63F31F4203696FF3CF340C60B8
:10A10800D96921EA0202DA61002030BDF8B54F783A
:10A118000B78012F00EB830349D19E694C693568A0
:10A1280033692A4664F3120314B967F3DC430BE07E
:10A138008F68E419013CB4FBF7F7CC7867F3DC438C
:10A14800012C08BF64F35E733361C378012B06D119
:10A158000B780C6900EB83039B695C610CE0CB789E
:10A16800012B09D04B693BB103690C785E6B012761
:10A1780007FA04F434435C63CB78012B07D10369F5
:10A188009B68DB0554BF45F0005245F080520B78C0
:10A1980000EB830342F004429B691A60CB78012BE1
:10A1A80038D10A788B8AC968FFF72CFD32E05E6DDA
:10A1B8004F6935688C6833692A462FB964F31203EE
:10A1C800012464F3DC430AE03F19013FB7FBF4F7CD
:10A1D800BF05BF0D67F3DC437C4364F312033361AF
:10A1E800C378012B05D10B780C6900EB83035B6DF9
:10A1F8005C61CB78012B06D14B7913B145F0005245
:10A2080001E045F080520B7800EB830042F00442F5
:10A21800436D1A600020F8BD73B54D78012D3DD10E
:10A2280083694A691E681C690094E4B242B962F302
:10A2380006048DF800409DF8024065F3C4040EE062
:10A248008D68AA4286BF4D6165F3060462F3060471
:10A258008DF800409DF80240012262F3C4048DF895
:10A268000240009A1A61C278012A05D10A780C695D
:10A2780000EB82029269546146F004421A60C37886
:10A28800002B34D14B69002B31D003690A78586B05
:10A29800012101FA02F202435A6328E00B784E6961
:10A2A8008C6800EB83035B6D1A681D690095EDB23D
:10A2B80006B14C6164F306059DF802408DF8005024
:10A2C800012565F3C4048DF80240009C1C61C37825
:10A2D800012B05D10B780C6900EB83035B6D5C6186
:10A2E8000B7800EB830042F00442436D1A600020B3
:10A2F8007CBD4B78012B0B7800EB83000AD1826977
:10A308001368C3F3076101F08001C9B221B143F0BA
:10A31800804301E0426D136843F40013136000208A
:10A3280070474B78012B0B78C97800EB83000CBF82
:10A338008269426D02391368C9B26FF35553012916
:10A3480098BF43F0805313600020704703699A69EF
:10A35800D8691040000C704700EB810102694B6D11
:10A368009B6850691840704703699869DB69184011
:10A3780080B2704782B000230093C0238DF8033069
:10A388000122002362F3C4038DF8023018238DF8EC
:10A398000030009A436D1A61C278012A06D100F58F
:10A3A800B96058611A684FF080221A6002B070478D
:10A3B800D0F8143110B50446D3B103699A68D207AE
:10A3C80016D5827A42B1D0F80C21D0F80C116FF36F
:10A3D80041026FF300020A605A6842F001025A60B3
:10A3E8000520FFF7E5FB23695A6822F001025A604D
:10A3F80010BD837A63B103699B68D90708D5D0F883
:10A408000C31D0F80C216FF341036FF30003136094
:10A418007047012310B5002280F812310446034624
:10A42800FF2104E058698160186D0132816060780D
:10A4380004338242F6D3236900221A615A61DA6131
:10A448004FF0FF329A612046FFF7FEFC20461021AC
:10A45800BDE81040DBE44B78012B0B7800EB830060
:10A468000FD183691868C0F3074000F02003DBB2FE
:10A47800CBB900F00200C0B200280CBF3020202069
:10A488007047436D1868C0F3074000F02003DBB243
:10A498005BB900F00200C0B200280CBF4FF4405076
:10A4A8004FF400507047102070474FF480507047A9
:10A4B8004B78012B0B7810B500EB83030AD19C690C
:10A4C800102A236802D1BDE8104012E7202A0CD0D8
:10A4D800302A0FE05C6DB2F5805F236802D143F447
:10A4E80000131BE0B2F5005F02D143F0006315E0F2
:10A4F800B2F5405F0FD1C3F3074202F02002D2B297
:10A5080022B100234B71BDE810400AE743F0806395
:10A5180043F0802302E00AB962F3CF33236010BD11
:10A52800F8B50446FFF794FB0122002384F81221B2
:10A5380084F8133128271646194640250CE007FBF6
:10A5480003F000F58C7022182354D3805670D17014
:10A558009560D1605161013362789342EFD3002353
:10A568002826194640250CE006FB03F000F55C7030
:10A5780022182354D3805170D1709560D1605161F5
:10A58800013362789342EFD32046FFF739FC204627
:10A59800FFF7BEFB00212046FFF770FC2046FFF7BF
:10A5A800C3FC2046BDE8F840FFF723BC70B5CDB228
:10A5B8000C464FF0280601F07F0106FB010115F05B
:10A5C800800F14BF01F58C7101F55C7104F07F04F4
:10A5D800ED090C704D708A60CB7005B1CC80022BF0
:10A5E80001D100230B71FFF743FD002070BD10B5AA
:10A5F800CAB201F07F034FF0280404FB030312F0F2
:10A60800800F14BF03F58C7303F55C7301F07F01B1
:10A61800D20919705A701946FFF759FD002010BD6C
:10A6280038B501F07F0528246C4304F55C740119E2
:10A638004B6100238B614B70EBB20355CA60C47841
:10A64800012C08BF0A6113B9FFF7E6FD01E0FFF727
:10A658005DFD002038BD70B501F07F0428256543F5
:10A6680005F58C7541190126E4B2CA600A61002219
:10A678004E7044558A614B6114B9FFF7CDFD01E076
:10A68800FFF744FD002070BDCAB212F0800F10B56C
:10A698004FF0280306D001F07F0403FB040303F501
:10A6A8008C7303E003FB010303F55C73D2090124F7
:10A6B80001F07F0119709C705A701946FFF719FE56
:10A6C800002010BDCAB212F0800F10B54FF0280359
:10A6D80006D001F07F0403FB040303F58C7303E049
:10A6E80003FB010303F55C730024D20901F07F0129
:10A6F80019709C705A701946FFF713FE204610BD5A
:10A7080008B50B0604D501F07F01FFF780FB01E0D7
:10A71800FFF79AFB002008BD0369002261F30A12C3
:10A7280019680A431A60704703695A6803206FF36F
:10A7380041025A60FFF73CBA03695A68032042F0A5
:10A7480002025A60FFF734BA11F0800F4FF0280365
:10A7580006D001F07F0103FB010101F58C7103E0D4
:10A7680003FB010101F55C71FFF775BE11F0800F65
:10A778004FF0280306D001F07F0103FB010101F52A
:10A788008C7103E003FB010101F55C71FFF790BEDA
:10A798002DE9F74F0446FFF78BFB002800F03F82B6
:10A7A8002046FFF792FB0546002800F03882C0F3E8
:10A7B800074000F00800C0B2002861D02046FFF72B
:10A7C800C5FDA146824627464FF00008DFF86CB366
:10A7D8002E4650E01AF0010F46D05FFA88F2114673
:10A7E80020460092FFF7B8FD10F0010F0546009AC9
:10A7F80020D07B6D01259D60E178A94207D11B69B6
:10A80800D9F87813C3F31203CB1AC9F88833DBF8E5
:10A81800003020461B6811469847E378012B09D180
:10A82800B8F1000F06D194F81131052B02D120465A
:10A83800FFF7A0FD05F00203DBB213B17B6D022523
:10A848009D6005F00403DBB213B17B6D04259D60A8
:10A8580005F00805EDB23DB1DBF8003020469B68F5
:10A8680098477B6D0820986008F101084FEA5A0A5A
:10A87800043709F12809BAF1000FABD13546012098
:10A88800C5F3074303F00403DBB2002B00F0AF80ED
:10A898002046FFF769FD264683464FF000080195DC
:10A8A8009FE01BF0010F00F0978023695FFA88F999
:10A8B80019695D6B04EB890225FA09F59269ED01C6
:10A8C8009268EDB20D431540EA071CD55A6B01207A
:10A8D80000FA08F122EA01025A63B369974A9860BC
:10A8E800136805465B68204649469847E378AB42BB
:10A8F80009D1B8F1000F06D194F81131042B02D117
:10A908002046FFF737FD05F00403DBB213B1B36946
:10A9180004259D6005F00803DBB213B1B36908256F
:10A928009D6005F01003DBB213B1B36910259D607B
:10A9380005F02003DBB213B1B36920259D6005F053
:10A948004003DBB213B1B36940259D6005F00203F3
:10A95800DBB213B1B36902259D6025F07F0515F0C0
:10A96800FF0F39D0282505FB084505F58C75C2462B
:10A97800AB696A69C3EB020CAB689C4528BF9C466F
:10A988000CF1030CB3694FEA9C0C9B696746A0461F
:10A9980014E0AA68E9681C1B944228BF1446A3B2B5
:10A9A80040464A46FFF72EF9EB681B19EB60AB6986
:10A9B800E71C1C19AC61B3699B69BF089BB2BB4219
:10A9C80005D9AC696B699C4201D2002BE1D1B3690E
:10A9D800802544469D60D04608F101084FEA5B0B8C
:10A9E8000436BBF1000F7FF45CAF019D012005F038
:10A9F8000203DBB213B1E36802225A61C5F30763AD
:10AA080003F08003DBB2CBB1A37A43B1D4F80C31A5
:10AA1800D4F80C216FF341036FF30003136023692B
:10AA28005A6822F001025A60444B1B6820469B6911
:10AA38009847E3684FF000425A610120C5F30723A5
:10AA480003F00803DBB2F3B13C4B1B6820465B699B
:10AA580098472369E2689B684FF400615161A27AC4
:10AA680082B1DB070ED5D4F80C311A6842F0010226
:10AA78001A601A6842F003021A60314B1A6942F0F0
:10AA880006021A61012005F00803DBB243B12B4B23
:10AA98001B682046DB689847E36808225A61012052
:10AAA80005F01003DBB2002B33D0E3689A6922F07B
:10AAB80010029A611F6A282607F00F0306FB034657
:10AAC800C7F34343022B06F55C7602D0062B1AD156
:10AAD8000EE047F6F0733B40ABB1C7F30A172046C8
:10AAE800F1683A46FFF7A2F8F368DB19F36007E06C
:10AAF80004F5B96120460822FFF798F8C7F30A174A
:10AB0800B369DF19B761E3689A6942F010029A6184
:10AB18000120C5F3072303F01003DBB2002B39D063
:10AB280023695A68002622F001025A6031462046FD
:10AB3800FFF76DF923463246FF2108E09402002012
:10AB480000ED00E058698160186D0132816060781D
:10AB580004338242F6D3236901274FF0FF3267F3AB
:10AB68000F069A6167F31F460F22DE615A612F2292
:10AB78001A611A686FF30A121A602046FFF7FAFB87
:10AB8800E3684FF480525A61264B1B6820461B69C4
:10AB980098473846C5F3072303F02003DBB2EBB12F
:10ABA8002046FFF74FFAE3682046DE68FFF73CFAD5
:10ABB800032806D10023A3704FF40073A380092350
:10ABC80004E00123A3704023A380052363F38D26AB
:10ABD800E3684FF40052DE6001205A61C5F3074371
:10ABE80003F01003DBB24BB10E4B1B682046DB6948
:10ABF8009847E3684FF480125A610120C5F307456E
:10AC080005F02005EDB255B1064B1B6820461B6ABE
:10AC18009847E3684FF400125A610120FFE7BDE846
:10AC2800FE8F00BF9402002043230B80004870472A
:10AC38000402002038B51F4B1A68511C052A1960F8
:10AC480035D11979002201291A6030D09968B1F5F7
:10AC5800006F08BF9A60174B9968DC68A1421A46D2
:10AC680002D100221A7122E086BFC1F50063136188
:10AC7800C1EB0404D0F8EC3598BF14611569B3F83A
:10AC880039300C4C9D428AB204D95918ED1AA1608A
:10AC9800256104E06918A1600021ABB22161054972
:10ACA80001240C7104498A188121FFF7D4FC002083
:10ACB80038BD00BF8C0D0020232D002038B5282377
:10ACC8000A4D03FB01010A4BB1F888131B690446BE
:10ACD80028469847D4F8EC352046B3F8403001218F
:10ACE8002A46FFF79DFC002038BD00BFDB2C002062
:10ACF8008002002070B50B7813F0600506460C46FC
:10AD080025D0202D1FD1CD88B5B113F0800F4878FC
:10AD180008D0214B21499B682A469847E2881F4959
:10AD2800304625E01E4B1D4958641E4B30465D6178
:10AD38002A4600F022FB1DE0174B48789B682946FD
:10AD48002A46984725E000F077FB022521E04B785A
:10AD58000A2B11D00B2B14D0062B1AD14B881B0AA7
:10AD6800212B03D1CA883A2A28BF3A220E493046F5
:10AD780000F0EAFA00250CE00C49012200F0E4FAA0
:10AD880007E08B781BB9074A1D46936101E000F084
:10AD980053FB284670BD00BF800200201B2D0020F9
:10ADA800040200208C0D002016020020A40D0020B3
:10ADB80010B581210446FFF71AFC01212046FFF750
:10ADC80016FC82212046FFF712FC024B5B6898476D
:10ADD800002010BD8002002038B5D0F8EC350446BC
:10ADE800B3F8392081210223FFF7E0FBD4F8EC35D2
:10ADF8000121B3F8402020460223FFF7D7FB822128
:10AE0800082203232046FFF7D1FB094B0222002525
:10AE18001A715D71074B1B689847D4F8EC35064AE0
:10AE2800B3F8403020460121FFF7FAFB284638BD29
:10AE3800C402002080020020DB2C002010B5074C43
:10AE4800606CFF2807D0064B064A9B680649526982
:10AE58009847FF236364002010BD00BF0402002050
:10AE6800800200208C0D00201B2D002038B51049D1
:10AE78000B79012B19D10C690CB90C7115E0D0F8BC
:10AE8800EC358D68B3F839309C42AAB203D95D1904
:10AE98008D60E41A03E0A3B22C198C6000240C61C5
:10AEA800044952188121FFF7D6FB002038BD00BFA6
:10AEB8008C0D0020232D00200020704700207047B3
:10AEC8000023F0B5084A094E1D4609E01468C75C1E
:10AED800375501340133B4F5006F146008BF1560AD
:10AEE8008B42F3D10020F0BD980D0020232D0020C7
:10AEF800104B114AD3F800C000232DE9F0410F4F41
:10AF080016461D460DE0146810F8038007F8048003
:10AF18000134802C08BF2C4614603468644505D081
:10AF280001338B42EFD10020BDE8F0810220BDE85B
:10AF3800F08100BFA4350020B8350020243500205A
:10AF480021280FD1084B1A680A701A68120A4A7029
:10AF58005A888A70DA78CA701A790A715A794A71E5
:10AF68009B798B71002070477802002007B502ABEF
:10AF7800012103F8010D1846FFF7A2FF0EBD0021BD
:10AF880000E00131435C002BFBD199E798E70B4BBC
:10AF98000B491A68096891420BD00A498A5C027009
:10AFA8001A680132802A1A6005D100221A6001202D
:10AFB8007047002070470120704700BFA43500206B
:10AFC800B835002024350020204B1A68204B1B6818
:10AFD8009A42F0B509D135E00133802B08BF002330
:10AFE8009A4203D11A4B1A602CE01A4CE15C0029F2
:10AFF800F2D00A29F0D00D29EED0154C1549134D81
:10B0080023600E460023CF182268BA5CC254226817
:10B0180001339F18802F08BF53422F689A18974210
:10B0280010D0B25C1AB10A2A01D00D2AEBD1002245
:10B03800C254074A116859187F29116003D9803909
:10B04800116000E000231846F0BD00BFB8350020AD
:10B05800A435002024350020704700BFD0F8E4351F
:10B0680010B51B6904469847032384F81231002061
:10B0780010BD08B5042380F81231D0F8E435DB6838
:10B088009847002008BD08B5D0F8E035DB6903B162
:10B098009847002008BD08B5D0F8E0351B6A9847E6
:10B0A800002008BD08B5D0F8E0355B6A9847002055
:10B0B80008BD002110B5402204460B46FFF776FA7A
:10B0C8008021402200232046FFF770FA012384F8EC
:10B0D8001231D4F8E435A0785B689847002010BD99
:10B0E80013B56946044600F085F99DF8001001F093
:10B0F8001F03012B07D0022B0AD073B920466946DB
:10B1080000F026FA0FE02046694600F007FA0AE048
:10B118002046694600F0A2F905E021F07F01C9B296
:10B128002046FFF7B1FA00201CBD38B504460029B7
:10B138003DD190F81131022B42D1D0F83421D0F80A
:10B1480020319A4211D9C178D21A0129C0F8342184
:10B1580004D1D0F82411CB18C0F8243192B220467B
:10B16800D4F8241100F000F92AE0D0F83821B2FB15
:10B17800F3F503FB152565B99A420AD3D0F83C319B
:10B188009A4206D229462A4600F0EEF8C4F83C5105
:10B1980016E0D4F8E035DB682BB194F81221032AC5
:10B1A80001D120469847204600F00FF908E0D0F872
:10B1B800E0355B6923B190F81221032A00D1984742
:10B1C800002038BD10B5044659BB90F81131032B47
:10B1D80030D1D0F88C23D0F878339A4214D9C1787A
:10B1E800D21A0129C0F88C2304D1D0F87C13C918CD
:10B1F800C0F87C139A4228BF1A4692B22046D4F867
:10B208007C1300F0CAF815E0D0F8E0351B6923B1CB
:10B2180090F81221032A00D19847204600F0C6F87A
:10B2280008E0D0F8E0359B6923B190F81221032A91
:10B2380000D19847002010BD2DE9F041069F044633
:10B24800164698460D46FEF741FC20462946C4F8A6
:10B25800E085C4F8E475C4F8E865FFF761F9D4F847
:10B26800E4351B6898472046BDE8F041FEF782BCEC
:10B2780000207047D0F8E03510B504461B689847A1
:10B28800D4F8E4359B689847002010BD08B5D0F87D
:10B29800E0355B689847002008BD000012230B804A
:10B2A80000487047C402002004230B800048704700
:10B2B800D602002010B5044C04480A46214600F086
:10B2C80075FA204610BD00BFBC35002076AF0508D2
:10B2D8000A4608B50248034900F068FA014808BD63
:10B2E80089AF0508BC3500200A4608B5024803495D
:10B2F80000F05CFA014808BD97AF0508BC3500208E
:10B3080008B50A4608B9044800E00448044900F0B2
:10B318004DFA034808BD00BFA2AF0508AFAF050846
:10B32800BC35002008B50A4608B9044800E00448BE
:10B33800044900F03BFA034808BD00BFBCAF05084C
:10B34800DDAF0508BC35002010B513460C46C0F823
:10B358003821C0F83421022280F811210021224628
:10B36800FFF779F9002010BD10B50C4613460021EF
:10B378002246FFF770F9002010BD10B513460C46A1
:10B38800C0F89023C0F88C23032280F811210021F3
:10B398002246FFF745F9002010BD10B50C461346AC
:10B3A80000212246FFF73CF9002010BD00210423AC
:10B3B80010B50A46044680F811310B46FFF74BF9E1
:10B3C8002046FEF7D7FF002010BD0021052310B549
:10B3D8000A46044680F811310B46FFF721F920464A
:10B3E800FEF7C8FF002010BD282303FB0100B0F8BA
:10B3F8008803704790F8C8350B7090F8C9354B70C2
:10B4080090F8CB2590F8CA3503EB02234B8090F8CF
:10B41800CD2590F8CC3503EB02238B8090F8CF250F
:10B4280090F8CE3503EB02239BB2CB80C0F83C31B9
:10B43800012380F81131704710B591F90030002BC5
:10B44800044601DBCB880BB9802100E00021FFF71F
:10B458001BF92046BDE81040FEF78CBF38B50D46F5
:10B4680004466B780979012B10D027D3032B51D1CF
:10B4780090F81231022B28D0032B47D16B889BB947
:10B4880091B1802910D0FFF7FFF80DE090F8123144
:10B49800022B1AD0032B39D16B88002B3AD149B132
:10B4A800802907D0FFF70EF9D4F8E03520469B68CD
:10B4B800294698472046FFF779FF2BE090F812318C
:10B4C800022B02D0032B21D106E019B3802921D009
:10B4D8002046FFF7D9F81DE011F0800F4FF0280340
:10B4E80006D001F07F0103FB010393F81A2103E062
:10B4F80003FB010191F87223074B02B101221A6084
:10B50800204605490222FFF71FFF03E0204629468F
:10B51800FFF792FF002038BDA80D002038B590F83D
:10B528001231032B04460D460CD10B79012B09D897
:10B53800D0F8E0359B689847EB883BB92046FFF781
:10B5480035FF03E020462946FFF776FF002038BD87
:10B5580073B54B7804460D46092B00F21C81DFE8D1
:10B5680013F0D10008011A01E4001A0172000A0060
:10B578001A01C00092004B881A0A013A062A00F202
:10B588000A81DFE812F007001A0027000801080105
:10B5980008010801D4F8E835A0781B680DF1060108
:10B5A8009847EB88402B014603D094F81231012BC1
:10B5B8003AD10823ADF8063036E0D4F8E035A07863
:10B5C8009B6A0DF106019847022343700146C4F8AF
:10B5D800EC0529E0DBB2052B00F2DD80DFE803F0A3
:10B5E80003080D12171CD4F8E835A0785B6817E03B
:10B5F800D4F8E835A0789B6812E0D4F8E835A0784C
:10B60800DB680DE0D4F8E835A0781B6908E0D4F8C9
:10B61800E835A0785B6903E0D4F8E835A0789B6941
:10B628000DF1060198470146BDF80630002B00F0E1
:10B63800B680EA88002A00F0B2809A4228BF1A46EB
:10B64800ADF806205CE08B88002B40F0A480CB8806
:10B65800002B40F0A08094F812214B88032A00F0B8
:10B668009A8003F07F05204684F813512946FFF796
:10B6780053F82046FFF79AFE0DB1022300E001239C
:10B6880084F812318BE08978464E0129317100F235
:10B69800828094F81231022B02D0032B7BD108E070
:10B6A800002962D00121032384F8101184F8123193
:10B6B80013E041B9022384F8123184F810112046AE
:10B6C800FFF7E4FD51E094F81011012920464DD010
:10B6D800FFF7DCFD317984F810112046FFF7CAFD29
:10B6E80043E0CA88012A56D194F81231022B02D0BD
:10B6F800032B50D102E020462B4913E004F5887152
:10B7080020460FE094F81231023B012B43D8D4F8BD
:10B7180014312449002B0CBF0123032341F80C3FAB
:10B7280020460122FFF710FE39E04B88012B29D073
:10B73800022B34D18B8813F0FF0F30D121691B0AFB
:10B74800013B4A68042B0FD8DFE803F0030507091B
:10B758000B00012306E0022304E0032302E0042394
:10B7680000E0052363F306124A602046FFF71EFE39
:10B7780015E094F81231023B012B0CD84B88012BB1
:10B788000DD10023C4F81431D4F8E03520469B6865
:10B7980029469847E9E720462946FFF74DFE00204D
:10B7A8007CBD00BFA80D0020B00D002030B5C8B189
:10B7B8000023DDB20133C41814F8014C002CF8D171
:10B7C8006B1C5B0013800B7003234B70022305E096
:10B7D800CA545A1CD2B202338C54DBB210F8012B73
:10B7E800002AF5D130BD00BF7047704770477047D9
:10B7F800704770477047000008B5FCF729FA094BF5
:10B808005A78187002435A701AB19A7801329A70AD
:10B8180030B99B78034A012B02D9002353709370E7
:10B8280008BD00BFB80D00202DE9F84F3F4B1B782D
:10B83800012B2DED028B09D002D3022B0FD108E08A
:10B848003B4B1A68802392FBF3F206E0384B1A68E8
:10B8580003E0374B1B6803225A43364B5A61364B79
:10B868001A8892B2002AFBD0334B00221A80FDF7C7
:10B8780079FD10EE105AFDF77BFD284610EE104AB0
:10B8880006F0E2FC80462046894606F0DDFC41ECE5
:10B89800100B41EC180B08F0AFFD57EC106BB0EE35
:10B8A800480AF0EE680A08F0A7FE32463B464046D2
:10B8B80049465BEC10AB06F01BFD06F0FBFF9FED65
:10B8C8001F8A07EE100ADFED1E7A57EE087A194C28
:10B8D80052465B46C4ED007A4046494606F008FDEC
:10B8E80006F0E8FF07EE900A27EE888A84ED018AC1
:10B8F800FDF750FD84ED020AFDF752FD84ED030AC1
:10B90800FCF7B4F80F4B62691B68D31A0E4A07EEAE
:10B91800100A1268F8EEC77A93FBF2F3C4ED047AC2
:10B928002383BDEC028BBDE8F88F00BF1C0E0020FE
:10B93800442C0020EC370020680D00200000F04265
:10B9480000008C4240260020C425002007B50420B2
:10B95800012105F0C7F84FF46043009301238DF8E7
:10B96800043002238DF805300448002369468DF819
:10B9780006308DF8073004F00DFD0EBD00080240BA
:10B98800084B1A684FF47A73B2FBF3F2064B013A8C
:10B998005A60064AF02182F8231000229A60072292
:10B9A8001A607047E401002010E000E000ED00E0BC
:10B9B800034B5A6812B15A68013A5A60704700BF7F
:10B9C800B80D0020024B58605A68002AFCD1704715
:10B9D800B80D002030B585B004460D4601A862496F
:10B9E8000A220BF001FA614B1B78032B10D8DFE811
:10B9F80003F00205080B01A85D4907E001A85D49AD
:10BA080004E001A85C4901E05C4901A80BF0D6FA02
:10BA180004AA131913F80C3C5D19EDB22F2D01D8A7
:10BA28000A3502E0392D01D90A3DEDB204AB1C19E3
:10BA38004FF6FF7004F80C5CFAF796FA0020FAF754
:10BA480095FB0DF103050F24204623345A210023CA
:10BA580015F8012FA4B2FAF7A3FBB4F5A57FF3D12B
:10BA680064205A212C220023FAF79AFB0023CD20C8
:10BA78005A212C22FAF794FB0020FAF775FA3B4B6F
:10BA88001B78032B6ED8DFE803F0022E576201A95A
:10BA980037480BF093FA0A22002135480CF0B6FB20
:10BAA800374A384B12781860012A0BD002D3022A81
:10BAB80015D109E0B0F5FA5FBCBF4FF4FA521A602D
:10BAC800314A07E0314A00E0314A904201DC013254
:10BAD8001A60304A1B689342C4BF2A4B1A602E4B27
:10BAE8001A682E4B26E001A922480BF067FA0A22B1
:10BAF800002120480CF08AFB214A294B1278186053
:10BB0800012A0BD002D3022A2CD109E0B0F5FA5F42
:10BB1800BCBF4FF4FA521A601B4A07E01B4A00E008
:10BB28001B4A904201DC01321A601A4A1B68934290
:10BB380018DD1B4B1A6015E001A90F480BF03EFAFF
:10BB48000D4800210A220CF061FB164B09E001A9FF
:10BB58000A480BF033FA094800210A220CF056FB78
:10BB6800114B186005B030BDFEAF05083F26002018
:10BB780010260020342600204A2C0020FC25002016
:10BB88001C0E00204C26002050DA11001FA10700CF
:10BB98007FF0FA0280D1F00840260020442C0020D3
:10BBA800642C0020402C0020F825002010B50D4BF7
:10BBB8000D4C1A680D4821460BF0D8F90C4B0D486E
:10BBC8001A6821460BF0D2F90B4B0C481A6821462B
:10BBD8000BF0CCF90A4B0B481A682146BDE8104017
:10BBE8000BF0C4B94C260020DEA50508102600205D
:10BBF800642C002034260020402C00204A2C0020F1
:10BC0800F8250020FC2500209FED010A704700BFA1
:10BC1800000000009FED010A704700BF000000000F
:10BC28009FED010A704700BF0000000018B101280D
:10BC380001D1034B00E0034B1868FDF71FBD00BF9F
:10BC4800302600204026002010B9034B18687047A2
:10BC5800024B1868704700BF4C2600204026002081
:10BC680010B9034B18687047024B1868704700BF3B
:10BC7800642C00203026002008B54FF49570FBF79F
:10BC880009FF40F26523C31A584240EB030008BD80
:10BC980008B5C620FBF7FEFE40F28D13C21A5042CB
:10BCA80040EB020008BD4FF4957040F26521FBF7A8
:10BCB800E3BEC62040F28D11FBF7DEBEDCE760EE86
:10BCC800A00AB7EE007AF0EE606A70EE077A40EEEE
:10BCD800006A47EEA70A36EEC77A08B5C7EE200A0B
:10BCE80010EE900A06F0B0FA0022084B06F000FBAE
:10BCF8000022074B06F04AF906F0DCFD07EE900A31
:10BD0800FDEEE77A17EE900A9F3008BD0000594013
:10BD18000000E03F38B52DED028BF7EE008AB0EE5B
:10BD2800608A70EE288A10EE900A28EE088A06F0DB
:10BD38008BFA08EEA88A00220F4B06F0D9FA0446BF
:10BD480018EE100A0D4606F07FFA02460B4620460A
:10BD5800294606F0F7FB0022084B06F017F906F013
:10BD6800A9FD07EE900AFDEEE77A17EE900A773004
:10BD7800BDEC028B38BD00BF000069400000E03F09
:10BD88002DE9F04F884F2DED068B97E80F0091B005
:10BD98000CAC103784E80F000FCF05AE0FC697E83C
:10BDA80007004FF6FF7386E807009F20772164227B
:10BDB800F7F77FFDA020772164224FF6FF73F7F78E
:10BDC80078FD9E20772164224FF6FF73F7F771FD07
:10BDD8009F20762164224FF6FF73F7F76AFD4FF62E
:10BDE800FF73782164229F20F7F763FD0020F9F79D
:10BDF8007AF99F2077216522FAF7F8F80C349F200A
:10BE080077216422FAF7F2F80DF12C0A0394F7EE81
:10BE1800009A4FF00F0B00E04D460AF1040AF7EEC6
:10BE2800008A9AED009A0024B0EE68AA01E0B846AC
:10BE3800354618EE900A06F007FA59A3D3E900230D
:10BE480006F056FA06F036FD08EE900A38EEE98A52
:10BE5800B0EE490AF0EE480AFFF731FFB0EE490AA2
:10BE6800F0EE480A0646FFF755FFB2B2074683B21E
:10BE78002CB9104619460F22F9F700FA06E0A8B2C5
:10BE88001FFA88F1CDF800B0F9F7FAFF0134B4F5DC
:10BE9800967FCCD13D46F7EE008A002401E0454666
:10BEA8004E4618EE900A06F0CFF93DA3D3E90023D9
:10BEB80006F01EFA06F0FEFC08EE900A39EEE88A53
:10BEC800B0EE490AF0EE480AFFF7F9FEB0EE490A6B
:10BED800F0EE480A8146FFF71DFF1FFA89F28046F7
:10BEE80083B22CB9104619460F22F9F7C7F905E0B5
:10BEF800B0B2A9B2CDF800B0F9F7C2FF0134B4F579
:10BF0800967FCCD1039B9A4586D104AD0DF12C0BBD
:10BF18004FF0000A01E0B846B146043595ED009AA5
:10BF2800F7EE008A002401E0B846B14618EE900A00
:10BF380006F08AF91AA3D3E9002306F0D9F906F026
:10BF4800B9FC08EE900A38EECA8AF0EE490AB0EE5B
:10BF5800480AFFF7B4FEB0EE480AF0EE490A064672
:10BF6800FFF7D8FEB2B2074683B22CB9104619467D
:10BF78002246F9F783F907E01FFA89F01FFA88F1DA
:10BF8800CDF800A0F9F77CFF0134B4F5C87FCBD118
:10BF98005D45C0D111B0BDEC068BBDE8F08F00BF88
:10BFA800295C8FC2F528F03FACAA0408121A06EEE5
:10BFB800902A081AB8EEE67A06EE900AF8EEE67AC3
:10BFC80008B5C7EE277A17EE900A06F03DF9002269
:10BFD800044B06F08DF90022034B05F0D7FF06F05D
:10BFE80021FC08BD000074400000E03F8A1A06EEFC
:10BFF800902A081AB8EEE67A06EE900AF8EEE67A83
:10C0080008B5C7EE277A17EE900A06F01DF9002248
:10C01800044B06F06DF90022034B05F0B7FF06F05C
:10C0280001FC08BD000069400000E03F70B506460D
:10C038000D460024610704D5A0B231462A46F9F717
:10C048001DF90134B4F5A07FF4D170BD70B5064672
:10C058000D460024600704D5A1B230462A46F9F7F8
:10C068000DF90134C82CF5D170BD234B1B78012B79
:10C0780003D011D3022B3DD123E0204B1A68204B6B
:10C088001A60204B1A68204B1A60204B1A68204B04
:10C098001A60204B1A6811E0184B1A68184BD20125
:10C0A8001A60184B1A68184BD2011A60174B1A6895
:10C0B800174BD2011A60174B1A68D201164B1A6037
:10C0C80070470E4B0E4A1968032391FBF3F1116078
:10C0D8000C4A11680C4A91FBF3F111600B4A116884
:10C0E8000B4A91FBF3F111600A4A126892FBF3F3D1
:10C0F800094A1360704700BF1C0E00204C26002020
:10C1080040260020642C002030260020402C0020EF
:10C11800C42500201C2600205C2C0020014B186838
:10C12800FDF7ACBA4026002008B5FFF79EFFBDE832
:10C138000840F3E770B500210A222748274D284E0A
:10C14800284C0CF063F800210A22286026480CF0DD
:10C158005DF800210A22306024480CF057F80021CD
:10C168000A22206022480CF051F8224B32681860ED
:10C178002B682149D31A06EE903A2368B8EEE67A7E
:10C1880006EE903AF8EEE67AC7EE277AFCEEE77A02
:10C1980017EE903A9AB20B80531C07EE903AB8EE1D
:10C1A800E77ADFED167A67EE277A154BFCEEE76A39
:10C1B80016EE901A8AB206EE902AB8EEE67A198040
:10C1C80077EEC77AF5EEC07AF1EE10FA01DD0132AA
:10C1D8001A80BDE87040A7E7102600204C260020F2
:10C1E800642C0020402C0020342600204A2C0020FB
:10C1F800FC250020F82500202C3A00200000803D76
:10C20800C03A00200022F0B51346202603254FF03F
:10C218002C0C00E02646303EF6B217460132092EB5
:10C2280010F8014B0AD897FBF5F605FB16772FB9DE
:10C23800CE1801F803C07470023301E0CC54013306
:10C24800092AE7D12022CA54CB1848225A707A22E8
:10C258009A700022DA70F0BDF0B51F46144B1E78B4
:10C26800012E8DB005460C4620D0A6F1030CDCF15A
:10C27800000646EB0C06CEB90E4908A80AF076FE71
:10C2880008A86946FFF7BEFF0B496A4604A80AF0EA
:10C298006DFEBDF84800F9F767FE3846F9F77AFEF3
:10C2A8002846214604AA3346F9F798FF0DB0F0BD99
:10C2B800CD250020DEA5050842AD050810B50121F1
:10C2C8000446F9F701F8014B1C8110BDB80D002098
:10C2D80008B50021C620FBF7CFFB4FF4957000216D
:10C2E800BDE80840FBF7C8BB014B9F221A81704785
:10C2F800B80D002000200146C82240F23F13F9F78C
:10C30800F7B807B50DF10700FEF741FE9DF80700E5
:10C318000EBD08B5FFF7F5FF0028FBD108BD30B505
:10C32800044687B010EE100A0D4605F08DFF024650
:10C338000B4601A805490AF019FE2046294601AA1C
:10C348000023F9F74BFF07B030BD00BF08B0050860
:10C3580008B5084803F080FA0648022103F04DFBAF
:10C368000028F9D0034803F0A3FA07EE900AB8EEC4
:10C37800670A08BD0020014010B52DED028B9FED26
:10C38800098A1924FFF7E4FF013CE4B238EE008A79
:10C39800002CF7D19FED040A28EE000ABDEC028BB1
:10C3A80010BD00BF00000000ACC868392DE9F04F8F
:10C3B800994B9A4C5D695F682DED068B93ED00AA49
:10C3C800C7B006461AEE100A93ED038AD3ED04AA05
:10C3D800D3ED028A93ED069A05F036FF41EC100B77
:10C3E800CDE9040108F0ECF932468D493BA88DED02
:10C3F8000C0B0AF0BBFDA06805F026FF02460B46B1
:10C408002BA888490AF0B2FDE06805F01DFF024636
:10C418000B462FA884490AF0A9FD1AEE900A05F0E8
:10C4280013FFCDE90A01DDE90A23804933A80AF0A0
:10C438009DFD284605F008FFCDE90601DDE9062344
:10C448007B4937A80AF092FD18EE900A05F0FCFE29
:10C458008046894642464B46764913A80AF086FD2F
:10C4680018EE100A05F0F0FE82468B4652467249D5
:10C478005B4617A80AF07AFDDDE904236F491BA87B
:10C488000AF074FD384605F0DFFE5BA3D3E900230C
:10C49800CDE9080105F02CFF02460B461FA86849A4
:10C4A8000AF064FD49EC118B4BEC10AB08F000F975
:10C4B80051A3D3E9002351EC100B05F019FF0246F4
:10C4C8000B4627A85F490AF051FD19EE100A05F03E
:10C4D800BBFE0B4602465C4923A80AF047FDD4ED93
:10C4E800047AFDEEE77A594917EE902A0FA80AF068
:10C4F8003DFD0022564BDDE90C0105F0F9FE06F082
:10C50800D9F905F0A1FE02460B4643A851490AF0A5
:10C518002DFDB5EEC08AF1EE10FADFED4F9A37D552
:10C52800304605F07FFE36A3D3E9002305F0E0FE90
:10C53800F1EE487A044617EE900A0D4605F084FE9F
:10C5480002460B462046294605F0D2FE02460B4617
:10C558002DA1D1E9000105F0F5FF06F0ABF99FED3B
:10C568003F7A07EE900AF4EEC77AF1EE10FAC6BFEA
:10C57800C7EEA97A3A4C3B4CF4EEE97AF1EE10FAA0
:10C5880038DD9FED357A384D384CC7EE877A78E03C
:10C598001FA3D3E900235046594605F0A9FE0446D7
:10C5A80030460D4605F03EFE15A3D3E9002305F0FD
:10C5B8009FFE02460B462046294605F0C3FF06F0BB
:10C5C80079F907EE900AB7EE007AF4EEC77AF1EE41
:10C5D80010FA46BF67EEA97A254C264CF4EEE97AA4
:10C5E800F1EE10FA4CDD9FED1C7A234D234CC7EE7B
:10C5F800877A46E01C4D44E06666666666A64C404F
:10C608001F85EB51B81E1940000000A2941A6D4214
:10C618000000000080842E41DC390020EC37002027
:10C628002AB0050834B005083FB005084AB0050827
:10C6380054B005085EB0050869B0050874B005086F
:10C648007FB005088AB0050895B00508A1B00508AF
:10C65800000034C0AEB0050800007A4400247449D4
:10C6680019B0050816B00508BAAF050822B00508C4
:10C678001FB005081CB0050825B0050827B0050837
:10C688009D4D17EE900A05F0DFFD2A46CDE9000121
:10C698003FA89A4902940AF069FC994B1A68994B89
:10C6A8001B689642CCBF002201229E42964BD8BFFF
:10C6B8000022DA60954B1B78082B40F0AE800220F0
:10C6C800F9F754FD4FF6FF70F9F764FC1F20F9F7EE
:10C6D8004BFC192100238E4A2D20F9F77FFD4FF6D8
:10C6E800FF70F9F757FC00200024F9F73DFC0F20F4
:10C6F800B42132464FF6FF730094FFF7ADFD0F20CB
:10C708006E2123462BAAF9F769FDB0206E21234636
:10C718002FAAF9F763FD0F20382123461BAAF9F742
:10C728005DFDB020382123461FAAF9F757FD0F20D9
:10C738005C21234633AAF9F751FD2346B0205C213A
:10C7480037AAF9F74BFD0F204A21234613AAF9F718
:10C7580045FDB0204A21234617AAF9F73FFD0F20CF
:10C768009B21234623AAF9F739FD0F20842123466C
:10C778003FAAF9F733FDB0208421234627AAF9F709
:10C788002DFDB0209B2143AA2346F9F727FD614BD5
:10C798001B68B3F57A7FCCBF4FF4FC604FF4784048
:10C7A800F9F7F8FB0023A020B4210FAAF9F716FD2A
:10C7B800594B1C78012C0CD002D3022C1DD111E04E
:10C7C8004FF6E070F9F7E6FB4FF48C700221534AFC
:10C7D80010E04FF4FC60F9F7DDFB4FF48C70022198
:10C7E8004F4A07E04FF6E070F9F7D4FB4D4A4FF493
:10C7F8008C7021460023F9F7F1FC0020F9F7CAFBF9
:10C808004FF4FC60F9F7B0FBFFF7B6FD0F20DC2111
:10C81800FFF785FD1F20F9F7BDFB3C4B1B789A1FDE
:10C82800D2B2012A02D90B2B40F053823E4B1B781F
:10C83800023B052B00F24D82DFE813F006007E0074
:10C84800EF004801E6016501DFED387A2AEE27AAF4
:10C858001AEE100A05F0F8FC9DED080B8046894693
:10C8680007F0CAFD404653EC102B494605F040FD41
:10C878001DA3D3E9002305F089FB05F0D3FF9DED47
:10C88800080B044607F0B8FE404653EC102B494607
:10C8980005F02EFD02460B4615A1D1E9000105F071
:10C8A80073FB05F0BFFF4FF6E073009305460023C6
:10C8B8000520DC213246FFF7CFFC134BDB6853B170
:10C8C8001B4B18881B4B4FF4784719880097A2B266
:10C8D800ABB2F9F7D5FA164B1C60164B4FF6E07061
:10C8E8001D60F9F741FBF4E10000000000E063403F
:10C8F8000000000000C05D4025B00508BCB0050878
:10C90800642C00204C260020B80D0020CD250020E6
:10C91800C9B00508741A00201C0E002024AF0508B1
:10C9280028AF05082CAF0508582C00200000C84285
:10C9380028380020CC3A0020A74B1868A74B32466D
:10C948001968FFF733FBA64B1B784FF4FA7292FB7A
:10C95800F3F307EE903AB8EEE79ADFEDA27AF4EE39
:10C96800498AF1EE10FAC8BFF0EE498AF5EE408A1E
:10C97800F1EE10FA48BFF0EE678AF4EEC98AF1EEDC
:10C9880010FA044620D8F4EEE78AF1EE10FA1BDB21
:10C99800FDEEC97AFDEEE88A17EE901A18EE902A95
:10C9A8000020FFF723FB904BDB68054653B18F4B04
:10C9B80018888F4B4FF6FF7719880097A2B2ABB251
:10C9C800F9F75EFA8A4B1D60B4EE498AF1EE10FA67
:10C9D800C8BFB0EE498AF1EE497AB4EE678AF1EE43
:10C9E80010FA48BFB0EE678AB4EEC98AF1EE10FAC1
:10C9F80000F26F81B4EEE78AF1EE10FAC0F26981B5
:10CA0800FDEEE77ABDEEC99ABDEEC88A17EE900A28
:10CA180019EE101A18EE102AAEE06F4B18686F4B1B
:10CA280032461968FFF7C2FAF5EEC0AAF1EE10FA1D
:10CA3800044627DDDDE90A0159A3D3E9002305F0FF
:10CA4800C9FEF8B158A3D3E90023DDE90A0105F0CE
:10CA58004FFC0B4602466749002005F095FA05F0A1
:10CA6800E1FE614BDB68054653B1604B1888604BAB
:10CA78004FF6FF7719880097A2B2ABB2F9F700FA20
:10CA88005B4B1D60DDE9060149A3D3E9002305F0EE
:10CA9800BFFE002800F01D81DDE9060140A3D3E9AF
:10CAA800002305F097FE002800F0138142A3D3E984
:10CAB8000023DDE9060105F01BFC02460B460020B9
:10CAC8004D4905F061FA05F0ADFE57E0424B186894
:10CAD800424B32461968FFF769FA39A3D3E90023B4
:10CAE8000446DDE9040105F093FE50B19DED040B09
:10CAF80007F066FE002251EC100B404B05F0F8FBE6
:10CB0800D2E0C825D3E030A3D3E90023DDE908014A
:10CB180005F0EEFB2EA3D3E9002305F013FD05F085
:10CB2800C9FE2D4B08EE100A18682C4B32461968BE
:10CB3800FFF73CFADFED327A4AEE677A2A4BFDEED0
:10CB4800E77ADB6817EE905A044625EAE57553B193
:10CB5800264B1888264B4FF6FF7719880097A2B204
:10CB6800ABB2F9F78DF9BDEEC88A214B18EE102A41
:10CB78001D606FF0B300B421FFF738FA1A4BDB6879
:10CB8800054653B1194B18881E4B4FF4FC6719889A
:10CB98000097A2B2ABB2F9F773F91A4B96E000BF4F
:10CBA8009A9999999999B93F0000000000409F40CF
:10CBB8009A9999999999B9BF0000000000408F404F
:10CBC80089B5F81400E3693F000000000080764052
:10CBD8001F85EB51B81E19404C260020642C0020FC
:10CBE8001C03002000000000B80D00202838002099
:10CBF800CC3A00200000694000005940000054C0B1
:10CC080000004843183600203B4B187805F00AFB13
:10CC180002460B460020394905F094FC05F04AFE0F
:10CC280008EE100A05F010FB41EC100B07F0C8FDE8
:10CC3800B4EE489AF1EE10FAC8BFB0EE489AB4EED6
:10CC4800C89AF1EE10FA5BEC10AB42D82C4B18687E
:10CC58002C4B32461968FFF7A9F9044619EE100A59
:10CC680005F0F2FA41EC100B07F0AAFD59465046C0
:10CC780059EC108B05F01EFE9FED237A07EE900A03
:10CC8800C7EE277A17EE900A05F0DEFA42464B46C1
:10CC980005F02EFB02460B4600201C4905F074F9EE
:10CCA80000221B4B05F072F905F0BCFD0546194B37
:10CCB800DB6853B1184B1888184B4FF6FF77198863
:10CCC8000097A2B2ABB2F9F7DBF8144B1D60124B18
:10CCD8001C60134B1B78022B09D043B14FF6FF732E
:10CCE80000930520DC2132460023FFF7B5FA47B050
:10CCF800BDEC068BBDE8F08F1C03002000005940F6
:10CD08004C260020642C00200000484300006940A5
:10CD18000000E03FB80D002028380020CC3A002061
:10CD2800582C002010B54FF4C770FAF7B3FEDB2873
:10CD380005D14FF4C870FAF7ADFE84B219E041F29C
:10CD4800E104214644F20100FAF796FE44F201009C
:10CD5800FAF7A0FEA04214BF80244FF4007421B259
:10CD68004FF4C870FAF788FE4FF4C770DB21FAF762
:10CD780083FE204610BD024B00221A60704700BF98
:10CD88003436002070EEA10A88B030EE010A08B0EF
:10CD9800704770EEE10A88B030EE410A08B070477B
:10CDA800F0EE407A20EEA10A60EE810A47EEA10A71
:10CDB80088B017EE810A08B07047D0B561EEA17A45
:10CDC80041EE017A2DED048B17EE900A88B0B0EE93
:10CDD800409AF0EE609AF0EE418AB0EE618A05F072
:10CDE80033FA0022002306460F4605F0E9FCE8B9AD
:10CDF80069EE887A49EE287A29EE088A17EE900AB1
:10CE080005F022FA32463B4605F09CFB19EEA88A4B
:10CE180005F050FD044618EE100A05F015FA3246E2
:10CE28003B4605F08FFB05F045FD01E0044804464C
:10CE380000EE900A00EE104A08B0BDEC048BD0BD9D
:10CE48000050C347F0B58E4B2DED068B93ED001ABD
:10CE5800D3ED011A8FB0F0EE408AB0EE608A8DED06
:10CE6800060ACDED070A30EE410A70EEE10A38EE07
:10CE7800811A78EE211A8DED0C1ACDED0D1A8DED73
:10CE88000A0ACDED0B0AFFF798FF8DED040ACDEDE8
:10CE9800050A04AA92E8030008AB83E80300DDED65
:10CEA800099A9DED08AA69EEA97A4AEE0A7A17EE60
:10CEB800900A05F0C9F941EC100B07F007FD51EC99
:10CEC800100B05F0F7FC09EE100A19EE900A05F0B0
:10CED800BBF904461AEE100A0D4605F0B5F945EC03
:10CEE800104B41EC110B07F0E3FB51EC100B05F074
:10CEF800E1FC68EE087A48EEA87AB1EE48AAC8EED6
:10CF0800A79A604B604D5A691B8B6860EA612B8455
:10CF180004468AEE27AA85ED009A19EE100AC5ED97
:10CF2800028A85ED038AC5ED049A85ED05AA05F008
:10CF38008BF94DA3D3E9002305F06AFCDFED537AA2
:10CF4800002818BFB0EE679AB7EE007A79EE077A34
:10CF580037EE497A4E4BC7EE877A1B78033BC5ED0F
:10CF6800067A042B71D8DFE803F0032738664F00F0
:10CF780018EE100A05F068F9044618EE900A0D46F6
:10CF880005F062F906460F4647EC116B45EC104B6D
:10CF980007F08EFB36A3D3E9002351EC100BCDE943
:10CFA800004505F0A5F93246CDE902013B4639496D
:10CFB800394809F0DBFF48E019EE900A05F044F91A
:10CFC80004461AEE100A0D4605F03EF92246CDE950
:10CFD80000012B46304831492AE019EE100A05F0C5
:10CFE80033F941EC100B07F0EBFB00222C4B51EC12
:10CFF800100B05F07DF905F05DFC05F025F90246FA
:10D008000B46254827491EE019EE100A05F01CF9C1
:10D01800064620460F4605F017F917A3D3E9002363
:10D0280005F066F9CDE900011B481F4932463B4629
:10D0380009F09CFF09E017EE900A05F005F9024691
:10D048000B461548194909F091FF134C002302209B
:10D05800CA212246F9F7C2F8002323700FB0BDECAD
:10D06800068BF0BDAFF30080AE47E17A14AEEF3F18
:10D078006666666666A64C40F6285C8FC2A54C407C
:10D088005C360020EC370020DC390020A4707D3F9E
:10D09800582C0020E8B00508F835002002B1050832
:10D0A800000034C012B1050824B1050840B10508D4
:10D0B80000B560EEA07A40EE007A2DED028B17EEF7
:10D0C800900A87B0B0EE408AF0EE608A8DED020AD1
:10D0D800CDED030A05F0B8F841EC100B07F0F6FBAC
:10D0E80051EC100B05F0E6FBDFED117A07EE100AA4
:10D0F80078EEA78A38EE078A68EEA87A48EE087AAA
:10D10800C7EE277A17EE900A05F09EF841EC100B4F
:10D1180007F0DCFB51EC100B05F0CCFB00EE900A9D
:10D1280020EE880A60EEA80A07B0BDEC028B00BDAD
:10D1380000000000F0B52DED028BDFED3A1A3A4BF6
:10D148008DB030EEA17AF0EE407AB7EE001A8DED90
:10D15800020A83ED001A30EE010AC3ED011A31EE1E
:10D16800671A71EEE01ACDED030AF0EE470A8DED6D
:10D17800077A8DED081ACDED091A8DED060AFFF72D
:10D188001CFE8DED000ACDED010A9DE8030004ABFD
:10D1980083E803009DED058ADDED048A68EE087AD0
:10D1A80048EEA87A17EE900A05F04EF841EC100BFD
:10D1B80007F08CFB18EE100A57EC106B05F044F8DA
:10D1C800044618EE900A0D4605F03EF845EC104B63
:10D1D80041EC110B07F06CFA3946304655EC104B10
:10D1E80005F068FB05F030F841EC100B07F062FA27
:10D1F800002251EC100B0D4B05F07AF805F05AFBA4
:10D2080029460646204605F055FB00EE900AF6EE44
:10D21800007A60EEA70A00EE106A0DB0BDEC028B32
:10D22800F0BD00BF00000000343A00200000E03FDD
:10D23800F0EE407A86B020EE200A67EE810A06B04A
:10D2480070472DE9F04F2DED028B85B0FCF78AF879
:10D2580010EE105AFCF78CF8284610EE104A04F02D
:10D26800F3FF80462046894604F0EEFF41EC100BA0
:10D2780041EC180B07F0C0F857EC106BB0EE480AF9
:10D28800F0EE680A07F0B8F932463B464046494690
:10D298005BEC10AB05F02CF805F00CFB9FED138A46
:10D2A80007EE100ADFED127A57EE087A114C5B464A
:10D2B800C4ED007A52464046494605F019F805F093
:10D2C800F9FA07EE900A27EE888A04AB84ED018A02
:10D2D80094E8030003E90300DDED030A9DED020A6B
:10D2E80005B0BDEC028BBDE8F08F00BF0000F04236
:10D2F80000008C42C43A002030B53F4B2DED088B1E
:10D30800D3ED008AD3ED019A3C4BD3ED00AAD3EDBF
:10D3180001BA3B4B93ED008A93ED019A394B93ED9B
:10D3280000AA93ED01BA38EEEA0A79EEEB0A38EE74
:10D338004A1A79EE4B1A93B08DED0A0ACDED0B0A15
:10D348008DED0C1ACDED0D1AFFF72AFD8DED000AB3
:10D35800CDED010A9DE803003AEE6A0A7BEE6B0AFE
:10D3680004AB38EE681A79EE691A83E803008DED8C
:10D37800081ACDED091A8DED0E0ACDED0F0AFFF74B
:10D388000FFD8DED000ACDED010A9DE8030006AB07
:10D3980083E803009DED040ADDED050A9DED061AFC
:10D3A800DDED071AFFF709FD8DED000ACDED010A45
:10D3B8009DE8030002AD85E80300134B9DED021ABA
:10D3C80093ED000AD3ED010ADDED031AFFF7E8FC3F
:10D3D8008DED000ACDED010A9DE8030012AB03E9CB
:10D3E80003006C46DDED110A85E803009DED100A87
:10D3F80013B0BDEC088B30BDF03500204836002056
:10D40800B83A0020483A002010380020F7EE007A99
:10D4180077EEC07A20EE022A20EE210A07EEA00A53
:10D42800F0EE420A47EE810A88B008B070472DE94D
:10D43800F0432DED028B924B1B78012B89B081466E
:10D44800884646D14FEAC00901291FFA89F92BD825
:10D4580009F58065A8B2FAF761FB8A4C0435A8B2D1
:10D4680084ED000AFAF75AFB09F58645A8B284ED5F
:10D47800010AFAF753FB844C043584ED000AA8B27C
:10D48800FAF74CFBA9F5FC4084ED010A80B2FAF7E3
:10D4980045FB7E4CA9F5FA40FC3884ED000A80B2C1
:10D4A800FAF73CFB84ED010A08F1FF385FFA88F8C7
:10D4B800B8F1010F00F2DF80A9F57C5080B2FAF7CD
:10D4C8002DFB734CA9F57A5984ED000AA9F17C0962
:10D4D800CBE0022B40F0CF806E4B6F4A1B680129CE
:10D4E80092ED007A00F2AC8007EE900AF8EE676AD7
:10D4F80007EE903A46EE877ABDEEE77A17EE104AC5
:10D50800A4B207EE104A04F18005ED00B8EE478A90
:10D51800ADB2284637EEC88AFAF700FB0435A8B240
:10D5280004F50665EE008DED020AFAF7F7FAB6B2D1
:10D5380030468DED030AFAF7F1FA043604F58257FE
:10D54800B0B28DED040AFE00FAF7E8FAB6B230463A
:10D558008DED050AFAF7E2FA0436B0B281348DEDA2
:10D56800060AE400FAF7DAFAA4B220468DED070AB3
:10D57800FAF7D4FA434E0434A0B286ED000AFAF75B
:10D58800CDFA6C1CE400A4B2204686ED010AFAF735
:10D59800C5FA3D4D0434A0B285ED000AFAF7BEFA8B
:10D5A8007C1CE400A4B2204685ED010AFAF7B6FA1D
:10D5B800364F0434A0B287ED000AFAF7AFFAD6ED79
:10D5C800001A96ED012ADDED020AF0EE408A87ED99
:10D5D800010A9DED031AB0EE480AFFF717FF8DED1B
:10D5E800000ACDED010A9DE80300D5ED001A95ED7E
:10D5F800012AB0EE480ADDED040A86E803009DED35
:10D60800051AFFF703FF8DED000ACDED010A9DE82D
:10D618000300D7ED001A85E80300B0EE480ADDEDF7
:10D62800060A9DED071AB0EE682AFFF7EFFE8DEDAA
:10D63800000ACDED010A9DE8030087E803006C4667
:10D6480008F1FF385FFA88F8B8F1010F13D809F527
:10D65800C1594FEAC9091FFA89F94846FAF75EFA2B
:10D668000B4C84ED000A09F104091FFA89F0FAF756
:10D6780055FA84ED010A09B0BDEC028BBDE8F083D0
:10D68800C9010020B83A002048360020483A002056
:10D69800F0350020C8250020082600202DE9F04F8D
:10D6A8006E4B2DED048B1C78012CC7B0054605D0B8
:10D6B80006D3022C0CBF3024002402E0002400E032
:10D6C80010244FF47670FAF7E5F907464FF47570B1
:10D6D800FAF7E0F980464FF47470FAF703FA032D6D
:10D6E800C0B21D9040F094805D4A5E4924A809F0BC
:10D6F8003DFCC1B224A8FDF749FC3B4642465A49C5
:10D7080024A809F033FCC1B224A8FDF73FFC574A0E
:10D71800544924A809F02AFCC1B224A8FDF736FC14
:10D7280004F1C800FAF7DEF9064604F1CC00FAF76E
:10D73800D9F9054604F1D000FAF7D4F9074604F1FF
:10D74800D400FAF7CFF9AB1B06EE903AB8EEE67ABA
:10D7580006EE907AF8EEE67A2B46C7EE277A32463E
:10D7680001904349009724A8FDEEE77ACDED027AAF
:10D7780009F0FCFBC1B224A8FDF708FC3D4A394971
:10D7880024A809F0F3FBC1B224A8FDF7FFFBE820A9
:10D79800FAF7A8F90546EC20FAF7A4F90446F020B0
:10D7A800FAF7A0F90646F420FAF79CF9631B07EE8E
:10D7B800903A06EE906AB8EEE77AF8EEE67A2A46EC
:10D7C800C7EE277A01902A490096234624A8FDEE41
:10D7D800E77ACDED027A09F0C9FBC1B224A8FDF7BA
:10D7E800D5FB1D9A022A06D1234924A809F0E6FB95
:10D7F80024A8142109E01D9B012B40F089821F49B0
:10D8080024A809F0DBFB24A81021FDF7BFFB7FE269
:10D818001D9A012A40F00E8104F1C800FAF762F956
:10D828001B9004F1CC00FAF75DF9074604F1D0002B
:10D83800FAF758F91B9B1C90FF1A06EE907AB8EE7F
:10D84800E67A06EE900AF8EEE67A0024C7EE277A22
:10D85800FDEEE77ACDED1F7AE7E000BF1C0E002051
:10D8680050B105084BB105085AB1050867B105085C
:10D878006DB10508B7B10508BDB10508D2B10508F5
:10D888001C9B1B9A2046012103FB042AFFF7CFFDAE
:10D89800914B924A18681768D3ED018A92ED019A64
:10D8A8008F4B904AD3F80090D3ED019A1368012D5D
:10D8B800209392ED018A7ED1F5EEC08AF1EE10FA3E
:10D8C80054BF4FF0000C4FF0010CB5EEC09ABCF1FC
:10D8D800000F0CBF4FF02B084FF02D08F1EE10FA97
:10D8E80054BF4FF0000E4FF0010EF5EEC09ABEF196
:10D8F800000F0CBF2B262D26F1EE10FA54BF002185
:10D908000121B5EEC08A00290CBF4FF02B0B4FF058
:10D918002D0BF1EE10FA54BF00220122002A0CBF91
:10D928002B232D231E93BCF1000F01D0F1EE688A42
:10D93800BEF1000F01D0B1EE499A09B1F1EE699A32
:10D948000AB1B1EE488A04F07FFCCDE9000118EE77
:10D95800900ACDF8088004F077FCCDE90401384638
:10D9680004F072FCCDE9060119EE100A089604F0DD
:10D978006BFCCDE90A01484604F066FCCDE90C01D0
:10D9880019EE900ACDF838B004F05EFCCDE910012C
:10D99800209804F059FC1E9ACDE9120118EE100ADD
:10D9A800149204F051FC5246CDE9160124A84E49C0
:10D9B80009F0DCFA2FE0022D2ED1FFF79DFC8DED4A
:10D9C800220ACDED230A22AB93E8030046AB03E914
:10D9D8000300DDED457AF5EEC07AF1EE10FA4498D1
:10D9E80005D5F1EE677A17EE906A2D2702E017EE5B
:10D9F800906A2B2704F028FC02460B463046CDE9F6
:10DA08000023029704F020FC5246CDE9040124A823
:10DA1800364909F0ABFAC6B224A83146FDF7B6FA82
:10DA28000120FDF7CFFF0134A4B21F9BA342BFF62C
:10DA380027AF6AE11D9A022A40F06781E820FAF7C9
:10DA480051F81B90EC20FAF74DF80646F020FAF74B
:10DA580049F81B9B1C9006EE900AF61AB8EEE68A67
:10DA680006EE906AF8EEE67A04F1C800C7EE887A06
:10DA7800FDEEE77ACDED1E7AFAF734F8064604F1A2
:10DA8800CC00FAF72FF8074604F1D000FAF72AF885
:10DA9800BF1B07EE100A06EE907AF8EEC77AB8EECA
:10DAA800E67A1B9A1F9087EE277A931B012D06EEC4
:10DAB800903ABDEEC77A88EE278A0D4B8DED207A15
:10DAC800B8EEE67A87EE277A83ED007A094B83ED84
:10DAD800008A40F0D0808FE0B83A00204836002015
:10DAE800483A0020F0350020E3B105081EB20508C9
:10DAF800C8250020082600201F9A002102FB046286
:10DB080020462192FFF793FC95ED018AD8ED018A12
:10DB1800B5EEC08AF1EE10FA54BF4FF0000C4FF08A
:10DB2800010CF5EEC08A9AED019ABCF1000F0CBF0A
:10DB38002B272D27F1EE10FA54BF4FF0000E4FF0AF
:10DB4800010EB5EEC09ABEF1000F0CBF4FF02B0BC3
:10DB58004FF02D0BF1EE10FA54BF00210121286877
:10DB6800D8F80090DAF8003000290CBF2B222D22BB
:10DB7800BCF1000F01D0B1EE488ABEF1000F01D010
:10DB8800F1EE688A09B1B1EE499A19921A9304F034
:10DB98005BFBCDE9000118EE100A029704F054FB74
:10DBA800CDE90401484604F04FFBCDE9060118EE23
:10DBB800900ACDF820B004F047FB1A9BCDE90A0182
:10DBC800184604F041FB199ACDE90C0119EE100A28
:10DBD8000E9204F039FB219ACDE910014F4924A88F
:10DBE80009F0C4F9C1B224A8FDF7D0F90134012025
:10DBF800FDF7E8FEA4B205E0494DDFF83481DFF80F
:10DC080034A10024209BA342BFF676AF0024454DE3
:10DC18002DE01C9B1B9A2046022103FB0426FFF7DC
:10DC280006FC95ED018AB5EEC08AF1EE10FA286877
:10DC380003D5B1EE488A2D2700E02B2704F004FB1A
:10DC4800CDE9000118EE100A029704F0FDFA3246F9
:10DC5800CDE90401344924A809F088F9C1B224A8FF
:10DC6800FDF794F90120FDF7ADFE0134A4B21E9B27
:10DC7800A342CEDA49E0022D47D142E01C9B1B9A11
:10DC88000121204603FB0425FFF7D1FBFFF734FBF6
:10DC98008DED220ACDED230A22AB93E8030046ABB3
:10DCA80003E90300DDED457AF5EEC07AF1EE10FAEE
:10DCB800449806D5F1EE677A17EE908A4FF02D0951
:10DCC80003E017EE908A4FF02B0904F0BDFA0646E0
:10DCD8000F464046CDE90067CDF8089004F0B4FA45
:10DCE8002A46CDE90401104924A809F03FF9C1B238
:10DCF80024A8FDF74BF901340120FDF763FEA4B217
:10DD080000E000241E9BA342B8DA084B1D9A1A7043
:10DD180047B0BDEC048BBDE8F08F00BF32B20508F8
:10DD2800B83A0020F035002060B20508C90100208B
:10DD380048360020483A0020F0B52DED028B044605
:10DD48008DB0002800F0D480714B18890419A4B252
:10DD580022B2002A05DB40F23F139A42C8BF1C4694
:10DD680000E00024F7F79EFAA0B24EF29C71F7F794
:10DD7800ABFA674B1C81674B586804F065FA5EA3E1
:10DD8800D3E9002304F0B4FA04F094FD624B186060
:10DD9800624B1B780A2B054624B23DD107EE104A88
:10DDA800F8EEC77A17EE900A04F04EFA5C4B064676
:10DDB80018680F4604F036FA02460B4650A1D1E91E
:10DDC800000104F0BFFB02460B463046394604F01A
:10DDD8008FFA064628460F4604F036FA02460B46E6
:10DDE8003046394604F084FA00224E4B04F0AAFB70
:10DDF80004F060FD04F028FA02460B4604A84A49DC
:10DE080009F0B4F80020F8F7B1F90520D72104AAE1
:10DE18000023F8F7E3F96BE0444B1888604304F0FB
:10DE280001FA39A3D3E9002304F08CFB04F042FD86
:10DE38003F4B08EE100A1B68FCEEC87A07EE103A52
:10DE480017EE905AF8EEC77A3A4B68EE277A1B68B5
:10DE5800FDEEE77AADB217EE906A28460121F61872
:10DE6800FFF7E5FAFFF748FA8DED020ACDED030A50
:10DE780002AC94E8030008AB83E80300681C80B296
:10DE88000121FFF7D4FAFFF737FA8DED020ACDED3D
:10DE9800030A94E803000CAB07EE105A03E90300E9
:10DEA800B8EEC70ADDED080A38EE400A9DED091AFA
:10DEB800DDED0A1A9DED0B2AFFF7A8FA8DED020A8F
:10DEC800CDED030A94E8030006AB83E803004FF6A0
:10DED800FF73009305200023DC213246FEF7BCF9CE
:10DEE800154B9DED060A1878DDED070AFEF7AAFF27
:10DEF8000DB0BDEC028BF0BD7B14AE47E17A843FD8
:10DF0800000000A0D954BD410000000000F073409B
:10DF1800B80D00201C030020AC3A0020CD250020BD
:10DF2800642C00200000F43F73B205082C3A00204E
:10DF3800402C00204C260020582C00202DE9F843C6
:10DF4800461F8846B6B200250D4F12E008EB0401C3
:10DF580089B23046F7F75AF929F814000A20013433
:10DF6800FAF78CFF062CF1D116350136F22DB6B230
:10DF780004D06FF0040407EB0509E7E7BDE8F88370
:10DF8800683A00202DE9F04F85B00B1A0193431E23
:10DF98009BB20293431C441F00F1060901F1FF3AAA
:10DFA80001F1010B9BB20F461646A4B21FFA89F97C
:10DFB8001FFA8AFA1FFA8BFB0393804620465146C4
:10DFC8003246F7F75BF9204639463246F7F756F9F5
:10DFD800204659463246F7F751F9019B0298E51851
:10DFE800ADB229463246F7F749F940462946324646
:10DFF800F7F744F90134039829463246F7F73EF912
:10E00800A4B20A20FAF73AFF4C45D7D105B0BDE8CB
:10E01800F08F2DE9F843461F8846B6B200250E4F0B
:10E0280012E008EB040139F8142089B23046F7F7FA
:10E0380025F901340A20FAF721FF062CF1D116350B
:10E048000136F22DB6B204D06FF0040407EB0509CF
:10E05800E7E7BDE8F88300BF683A00202DE9F04300
:10E068002DED068B70EE007A8DB017EE900AB0EEAB
:10E07800408A10EE904A20EE009A04F0E5F8064631
:10E0880020460F4604F0E0F8F7EE008A41EC100B4A
:10E0980041EC1A0B06F0B0F979EE287A55EC104BE2
:10E0A80017EE900A04F0D0F82246804689462B469F
:10E0B8003046394604F01CF902460B4640464946AC
:10E0C80003F062FF04F0F6FBB0EE4A0AF0EE6A0ACB
:10E0D80009EE900A38EEC99ADFED377A89EE299A67
:10E0E80029EE279A06F088FA304653EC102B394669
:10E0F80004F0FEF8044619EE900A0D4604F0A4F860
:10E1080002460B462046294604F01CFA00222B4BF7
:10E1180004F0EEF804F0CEFBB4EE688ADFED287A5E
:10E12800284BF1EE10FA044619EE100A08BFB0EEBB
:10E13800678A1D6804F088F802460B4603A822493E
:10E1480008F014FF204604F07FF802460B4606A8A4
:10E158001E4908F00BFF78EE287A38EEC88A87EE59
:10E16800888A18EE100A04F06FF802460B4609A8D0
:10E17800174908F0FBFE0520014603AA0023F8F71B
:10E188002DF80520142106AA0023F8F727F8C8203F
:10E19800052109AA0023F8F721F84FF6E073009348
:10E1A8000520DC212A460023FEF756F80DB0BDEC09
:10E1B800068BBDE8F08300BF0000484200004940DC
:10E1C800A4707D3F083800207CB2050884B2050899
:10E1D8008CB205082DE9F04F494B2DED048B1D78C5
:10E1E800022D85B080467BD1464E348A01212046D7
:10E1F800FFF71DF9FFF780F88DED000ACDED010A54
:10E208009DE8030004AB03E9030028469DED020ADC
:10E21800DDED030AFEF716FE3B4B1A683B4B1B6805
:10E2280002FB04343A4B1C603A4BDFED3B7A93ED2A
:10E23800008A68EE277A5F6817EE900A04F004F8FF
:10E24800824638468B4603F0FFFF41EC100B41EC49
:10E25800190B06F0D1F8504653EC102B594604F030
:10E2680047F823A3D3E9002303F090FE04F002FB50
:10E27800B0EE490AF0EE690A054684B206F0BCF928
:10E28800504653EC102B594604F032F80B46024620
:10E2980019A1D1E9000103F077FE04F0EBFAB37C91
:10E2A80081461FFA80FA1BB9B08AF18AFFF7B1FEDE
:10E2B800002320465146B374FFF740FE20465146DE
:10E2C8001F22FFF75FFEB0EE480A00EE907AFFF7D4
:10E2D800C5FE338AB5829844A6F81080A6F8169031
:10E2E80005B0BDEC048BBDE8F08F00BFAFF3008034
:10E2F8000000000000E063400000000000C05D4036
:10E30800582C0020B80D0020402C00204C2600205E
:10E3180008380020DC3900200000C842124B1B7866
:10E32800022B10B50CD1114B1B78022B08D1104CC5
:10E338002078C0B140B2FFF74DFF0023237010BD15
:10E348000C4C237E23B99F20F6F786FF0123237602
:10E35800064B1B78022B06D1054C94F90000FFF7F9
:10E36800EBFC0023237010BD582C0020343800200B
:10E37800811A0020B80D0020034B00201860034BC1
:10E388001870FDF753BC00BF343600203438002025
:10E39800034B00201860034B02221A70FDF746BC9D
:10E3A800343600203438002037B500242546A0B282
:10E3B80028213223024601340095F7F761FDB4F5B0
:10E3C800A07FF4D13EBD2DE9F04F2DED088B02283A
:10E3D80097B080468DED070AB34B05D0032805D0CA
:10E3E800012805D10C2202E0092200E00B221A7054
:10E3F8001878F2F771FB042103914FF00009F3EE4E
:10E408000EAA9FEDAABADFEDAABA7DE1A94B1A6858
:10E41800A94B1B6802FB093307EE103A01211FFACA
:10E4280089F0B8EEC78AFFF702F8FEF765FF8DEDB1
:10E43800080ACDED090A08AD95E803000AAB83E8A0
:10E4480003009E4B1A6802EBC9030EAF19689C4B78
:10E4580019600399521812685A60FEF74DFF8DED46
:10E46800080ACDED090A95E803000CAB83E8030020
:10E47800DDED0A9A9DED0BAADDED0C8A9DED0D9A56
:10E48800B0EE690AF0EE4A0AB0EE681AF0EE491AE0
:10E49800FEF786FC8DED080ACDED090A95E8030024
:10E4A800B0EE691AF0EE4A1A87E80300B0EE680A7F
:10E4B800F0EE490AFEF781FC8DED080ACDED090A58
:10E4C80095E8030010AB83E803009DED0E0ADDED2F
:10E4D8000F0AFEF7EDFD8DED080ACDED090A95E866
:10E4E800030016AA02E903009DED100ADDED110AEA
:10E4F800149EFEF7DDFD8DED080ACDED090A95E8BD
:10E50800030087E80300DDED0F0AF5EEC00AF1EE1F
:10E5180010FA48BFF1EE600A9DED0E0ACDED0F0A24
:10E52800FEF708FE8DED080ACDED090A08AA92E863
:10E53800030012AB83E803000798129D03F084FEE2
:10E548005D4B139FD3F800B05E4BBDEEC87AD3F88D
:10E5580000A0CDE9040117EE102A58465146FDF7F0
:10E5680025FD07EE10AAF8EEC77A07EE10BAB4EE4A
:10E57800E78AF8EEC77AF1EE10FAB4EEE78A8CBFB4
:10E5880000220122504B0690F1EE10FAD4BF00226F
:10E5980002F00102B8F1020FDA6012D0B8F1030FED
:10E5A8003ED0B8F1010F68D1304603F04DFE36A3D6
:10E5B800D3E9002303F09CFE0022444B03F0E6FC61
:10E5C8002AE0284603F040FEDDE9042304460D4610
:10E5D8002FA1D1E9000103F0B5FF02460B46204602
:10E5E800294603F085FE2CA3D3E9002303F080FE1F
:10E5F80004F060F907EE900AC7EEAA7A17EE900ABF
:10E6080003F022FE41EC100B06F0DAF8002251EC80
:10E61800100B2F4B03F06CFE04F004F904462CE0B9
:10E6280018EE100A03F010FE044638460D4603F0B3
:10E638000BFE17A3D3E9002303F05AFEDDE90423F8
:10E6480003F080FF04F036F903F0FEFD14A3D3E9CC
:10E65800002303F04DFE02460B462046294603F0F0
:10E6680071FF04F027F907EE900AB0EE6B7A07EE17
:10E678008B7AFDEEC77A17EE904A002C2ADBC72C5E
:10E68800A8BFC72427E000BF8716D9CEF753F5BF28
:10E698008FC2F5285CAF4340000000000090704036
:10E6A80000000080DBC48641582C00200000C8C34D
:10E6B8000000C843402C00204C26002020360020B3
:10E6C800F0350020642C0020B80D002000006940BF
:10E6D800000049C00024114BDB685BB1104B18885F
:10E6E800104B1988069B4FF6FF759AB2A3B2009596
:10E6F800F7F7C6FB0B4B039A1C600699084B0832C8
:10E70800196009F101090392074B1B884B45BFF6B5
:10E718007DAE17B0BDEC088BBDE8F08FB80D0020BA
:10E7280028380020CC3A00202C3A00202DE9F0436C
:10E738002E4B85B01878F2F7CFF92D4B0B221A70B3
:10E748002C4B1C78012C05D006D3022C0CBF30248E
:10E75800002402E0002400E01024274B1B78012B42
:10E7680007D104F1C800F9F7BDF9064604F1D00055
:10E7780004E0E820F9F7B6F90646F020F9F7B2F90F
:10E7880000240746DFF880901C4DDFF8808020E0E9
:10E7980007FB0463204601216B61A8F82040FEF7BF
:10E7A80046FEFEF7A9FD8DED000ACDED010A9DE8B4
:10E7B800030004AB03E903000C4B9DED020A187833
:10E7C800DDED030AFEF73EFB6869FDF7EFFD013456
:10E7D800A4B2B9F80030A342DADA094B02221A705F
:10E7E800084B00221A7605B0BDE8F083582C0020AB
:10E7F800CD2500201C0E0020C9010020EC37002088
:10E8080034380020B80D00202C3A0020DC390020D4
:10E818007FB5FDF709F8274A274B11685268196038
:10E828005A60264C264B22681B68264DD31A06EEE2
:10E83800903AB8EEE67AD5ED006AF8EEE67A00216D
:10E84800C7EE277AFCEEE77A17EE906AB0B2FEF7C9
:10E85800EEFDFEF751FD8DED000ACDED010A9DE8B4
:10E86800030004AB03E90300174B9DED020A187877
:10E87800DDED030AFEF7E6FA144B1868144B1B6823
:10E8880036B200FB0630FDF791FD124B226893F972
:10E898000010286800FB01200F4A126890421C46AD
:10E8A80005DCFAF7EBFE0D4B1868FDF78BF8002333
:10E8B80023707FBDEC370020F0350020283600207B
:10E8C80040260020C4250020582C0020402C002081
:10E8D8004C260020F025002030260020F8250020B6
:10E8E80008B5FFF795FF0C4B1A680C4B1B689A424A
:10E8F80010DB4FF08040002102F055FD084B1868EE
:10E90800FAF7BCFE074B02221A70074A002313705D
:10E91800064A137608BD00BF28360020302600209E
:10E928004026002034380020F0250020B80D0020B3
:10E9380010B500214FF0804002F035FD0A4B00244D
:10E948001C700A4B20461C70F7F73AFB084B1868F6
:10E95800FAF794FE074B084801221A70074B1C70FF
:10E96800BDE81040F3F7D5B8F02500203836002070
:10E9780040260020582C0020FC170020CD25002020
:10E9880007EE100A034BF8EE477A0022C3ED007A2F
:10E998005A6070475C36002007EE100A034BF8EE09
:10E9A800477A0022C3ED007A5A6070471038002079
:10E9B8000F4B10491A68104B1B68D31A06EE903A91
:10E9C8000E4B1B68B8EEE67A06EE903AF8EEE67A59
:10E9D800C7EE277AFCEEE77A17EE903A9AB20B80E8
:10E9E800074B188890422CBF00200120704700BFB9
:10E9F800642C00202C3A00204C260020402C0020BB
:10EA08004426002013B502AB011D23ED010A054A77
:10EA180089B213F8014B1454013080B28842F8D1FE
:10EA28001CBD00BF6A3700202DE9F8431F4F07407F
:10EA3800002F04460D4603DA013F67F00F07013740
:10EA4800BFB2DFF874804FEAC7091FFA89F9484650
:10EA580098ED000A09F10409FFF7D4FF1FFA89F0BD
:10EA680098ED010AFFF7CEFF114B10261B8894FB87
:10EA7800F6F6F6019C42B6B20CD1701980B20D4977
:10EA88008022FAF79BFA00B1FEE721B24FF47F70BB
:10EA9800F8F7F2FF0F2F07D17519A8B205498022A0
:10EAA800FAF78CFA00B1FEE7BDE8F8830F000080A2
:10EAB8002C3A00206A370020EC3700202DE9F0437B
:10EAC800744B2DED028B1888FF2898BF4FF4807087
:10EAD80093B0C00007F0D8FE6F4B0546186028B900
:10EAE8000520B4216D4A2B46F7F778FB0024694FBF
:10EAF8006B4E4FF000086AE0FCF796FE20464FF494
:10EB08004141FFF791FF674B1A685B68326000214B
:10EB180073602046FEF78BFCFEF7EEFB8DED020AD4
:10EB2800CDED030A0DF1080999E803000AAB83E863
:10EB380003005D4B9DED0A1A93ED007AD3ED017A3F
:10EB4800DDED0B1A31EE470A71EEE70A31EE071ACE
:10EB580071EEA71A8DED0E0ACDED0F0A8DED101A84
:10EB6800CDED111AFEF729F98DED020ACDED030A54
:10EB780099E803000CAB83E80300FF2C4FEAC403B9
:10EB88002B4404D9C3F80080C3F8048003E00C9A2E
:10EB98001A600D9A5A603B8840F23F10604390FB20
:10EBA800F3F080B24FF4FC6302462821009332232D
:10EBB800F7F766F93D4B18683D4B1B68C018FAF724
:10EBC8005DFD3C4B1868FCF7FDFE0134A4B23B88A0
:10EBD800A34291DA012213464FF4807105A804F08C
:10EBE800FFFE354EDFF8F880294605A805F0DAF96A
:10EBF80008233370314B01241C700020F6F7AEFC5B
:10EC08002F48F2F786FF3078F1F766FF2D4B9FED1E
:10EC18002E8ADFED2E8A1C700024D5ED007AB0EE26
:10EC2800687A07EEC87A2046FCEEC77A17EE906A33
:10EC380003F0F8FA264B002203F05AFB03F01AFE01
:10EC4800B6B2A3B2C72E28BFC72687B253B1214B8D
:10EC5800B8F8000019884FF6FF7300933A46334618
:10EC6800F7F70EF91B4BC8F8007001340835B4F5F6
:10EC7800807F1E60D1D1184B1868FAF7FFFC114B42
:10EC880002221A70154B00221A7613B0BDEC028BC3
:10EC9800BDE8F0832C3A0020203600204DAA050854
:10ECA800F0350020EC3700205C36002028360020A4
:10ECB800C4250020F8250020582C0020790D0020BC
:10ECC8005817002034380020000016430000C842BE
:10ECD8000000F43FCC3A002040260020B80D002068
:10ECE80028380020F0B5294B294F2A4D2A4E0122F9
:10ECF80085B01A7000243AE0284B1A68336802FB82
:10ED080004336B61264B1C84FCF78EFD20464FF4C0
:10ED18004141FFF789FE234B2A681A606A6820463A
:10ED28005A600021FEF783FBFEF7E6FA8DED000A34
:10ED3800CDED010A9DE8030004AB03E903001A4B7B
:10ED48009DED020A1878DDED030AFEF77BF8686985
:10ED5800FDF72CFB154B1868154B1B68C018FAF704
:10ED68008DFC144B1868FCF72DFE0134A4B23B88C7
:10ED7800A342C1DA104B1868FAF780FC034B022251
:10ED88001A700E4B00221A7605B0F0BD34380020F8
:10ED98002C3A0020EC3700204C260020402C002084
:10EDA800DC390020F0350020582C002028360020BF
:10EDB800C4250020F825002040260020B80D00209A
:10EDC80038B5FDF7ABF9124B124D9F221A81124B41
:10EDD800012418782C70F1F77FFE104B00221A607E
:10EDE8000F4B1B78072B04D00B2B0DD0062B0ED105
:10EDF80002E0BDE8384075E74FF0804021462C70AE
:10EE0800BDE8384002F0CFBABDE838408EE438BDDE
:10EE1800B80D002034380020582C0020343600204B
:10EE2800CD2500202DE9F743002581462C46154EB7
:10EE3800154FDFF85C801FE0FCF7F6FC49462046DA
:10EE4800FFF7F2FDD8F800303868C018FAF716FC5A
:10EE58000E4B1868FCF7B6FD308895FBF0F080B2D1
:10EE68004FF4FC630093282102463223F7F708F891
:10EE780005F59E75013403353388A342DCDABDE815
:10EE8800FE8300BF2C3A002028360020F8250020F9
:10EE9800C425002010B5104C4FF47570B4F900105B
:10EEA800F8F7EAFD0D4B4FF47670B3F90010F8F758
:10EEB800E3FD40F2D230F8F7EDFDB02804D040F27F
:10EEC800D230B021F8F7D8FD2088FFF759FD034B61
:10EED8001888BDE810405FE5C4010020C00100208B
:10EEE80000210A2208B509F091F9D0F1010038BFD4
:10EEF800002008BD73B5041D0E46A4B20C220023E1
:10EF08004FF6E075204601360095F7F75DF80023C7
:10EF18000C22B1B220460095F7F756F80D4B1B7836
:10EF2800012B16D10C4E0D4D308829880024043051
:10EF380080B20C2223460094F7F746F830882988D7
:10EF480000940430013180B289B20C222346F7F7CD
:10EF58003BF87CBD143600205A3600200C380020BF
:10EF680008B54FF6FF70F6F7FFFF0020F7F7FEF839
:10EF7800E12023212C4A0023F7F730F9E12046212C
:10EF8800294A0023F7F72AF9E1206921264A0023B4
:10EF9800F7F724F9E1208C21244A0023F7F71EF91A
:10EFA8002348FFF79DFF20B121482249012207F09D
:10EFB800DDFF4B2023211E4A0023F7F70FF91E48D7
:10EFC800FFF78EFF20B11C481A49012207F0CEFF37
:10EFD8004B204621184A0023F7F700F91748FFF796
:10EFE8007FFF20B115481349012207F0BFFF4B20CE
:10EFF8006921124A0023F7F7F1F81148FFF770FF6B
:10F0080020B10F480B49012207F0B0FF4B208C219B
:10F0180000230B4AF7F7E2F80A4B18880A4B1988BD
:10F02800BDE8084066E700BF5DA8050898B2050876
:10F0380010260020DEA50508342600204A2C0020D2
:10F04800FC250020443A00200C3A002070B5044604
:10F0580000200D461646F7F789F80020F6F79AFFC4
:10F068004FF4FC60F6F780FF2046294656BB1E4A3F
:10F078003346F7F7B3F81D48FFF732FF20B11B48B6
:10F088001B49012207F072FF04F17006B6B2304640
:10F098002946164A0023F7F7A1F81648FFF720FF7C
:10F0A80020B114481249012207F060FF3235ADB291
:10F0B80020462946104A0023F7F790F8304629469B
:10F0C8000C4A07E00D4A0023F7F788F832350B4A57
:10F0D800A9B220460023F7F781F8094B1888094B95
:10F0E8001988BDE8704005E79DB20508B03A0020D0
:10F0F800F8A90508203A0020A5B2050898AA05082D
:10F10800443A00200C3A002030B5144D9DF80C40CC
:10F118002C70134D2880134D02FB04002980124DDA
:10F1280080B22880114D2980114D2A80114A138000
:10F13800114B1880114B1980114B1249E2B21A7009
:10F1480000230B7010490A709DF810200134013219
:10F1580054430E4A14700E4A137030BDC83B002049
:10F16800A83A0020EA370020443A00200C3A002050
:10F1780068370020D43A00205A3600200C38002086
:10F188000E3A002039360020463A00201536002075
:10F198001436002038B5054600200C46F6F7E6FF81
:10F1A8000020F6F7F7FE4FF4FC60F6F7DDFE0B489B
:10F1B800FFF796FE28B1094809490A4B002207F0D3
:10F1C800D5FE284621460023044AF7F707F8064BE0
:10F1D8001888064B1988BDE838408BE65036002061
:10F1E800BBAE05080000F03F443A00200C3A00206E
:10F1F800114B1B68002B70B505460C4604DA5B42C0
:10F208000E480F492D2202E00C480D49202207F034
:10F21800ADFE0020F6F7AAFF0020F6F7BBFE4FF47C
:10F22800FC60F6F7A1FE054A284621460023BDE802
:10F238007040F6F7D3BF00BF403A002018380020CE
:10F24800ADB205080F4B10B519684FF4E170F8F727
:10F2580030FC40F23D114FF4E070F8F70DFC00204F
:10F26800F6F784FF0020F6F795FE4FF4FC60F6F7FA
:10F278007BFE054A192064210023BDE81040F6F7FB
:10F28800ADBF00BF403A0020B5B2050808B54FF43D
:10F29800E070F8F7FFFB40F23D13984205D14FF4B8
:10F2A800E170BDE80840F8F71DBC002008BD38B57E
:10F2B800054600200C46F6F759FF0020F6F76AFECF
:10F2C8004FF4FC60F6F750FE0B48FFF709FE28B133
:10F2D80009480A490A4B002207F048FE28462146F9
:10F2E8000023054AF6F77AFF064B1888064B19885B
:10F2F800BDE83840FEE500BF2C360020BBAE05084F
:10F308000000F03F443A00200C3A002038B5C5010F
:10F31800ADB20024601980B2F9F7F8FB0134C0B22D
:10F32800FBF724FEA4B24FF47A70F9F7A7FD802CFE
:10F33800F0D138BD73B5104D00240E20FBF716FE32
:10F34800002609E00DF10700FBF721FE20B19DF82A
:10F358000730AB550136F6B23306F3D5E00180B27B
:10F3680005498022F9F72AFE00B1FEE70134A4B26C
:10F37800B4F5007FE1D17CBD6A37002007EE100AA2
:10F38800F8EE477A7FB517EE900A02F05DFF024665
:10F398000B4601A8054907F0E9FD0A20962101AAB4
:10F3A8000023F6F71BFF07B000BD00BFBCB205087D
:10F3B8000EB403B070470A2810B5044602D10D20D8
:10F3C800FFF7F9FF064A13681BB103F8014B1360F6
:10F3D80010BD044B1B680BB12046984710BD00BFF9
:10F3E800D80D0020CC3B002010B5044601E0FFF703
:10F3F800E2FF14F8010B0028F9D110BD2DE9F04FF8
:10F40800044685B00D464FF00A0A00E035462078DC
:10F41800002800F0C480252801D0013467E0607816
:10F42800302803D1A0780123033407E02D2802D027
:10F438000234002302E0A078022303344FF00008CE
:10F4480005E00AFB080814F8010BA8F13008A0F140
:10F458003002D2B2092AF4D96C2801D04C2803D141
:10F4680014F8010B43F00403002800F0988060288A
:10F4780086BFA0F12002D2B202464F2A3DD006D85C
:10F48800432A2DD0442A09D0422A30D133E0552AC4
:10F4980004D0582A29D0532A29D101E00A272DE07F
:10F4A8002E1D2F68002500E001357A5D002AFBD16A
:10F4B80004E02020FFF77FFF4D4601E0980704D4C1
:10F4C800454505F10109F4D34D463846FFF78CFF51
:10F4D80003E02020FFF76FFF01354545F9D395E795
:10F4E80028782E1DFFF767FF90E7102706E0FFF743
:10F4F80062FF2E468AE7022700E008272E1D442ACD
:10F50800296804D1002902DA494243F0080300229D
:10F5180000E02A46B1FBF7FE07FB1E11CDB2092D0C
:10F52800714607D9782814BF4FF0070C4FF0270C05
:10F538006544EDB230350DF80250551CBEF1000F90
:10F5480002D0102DE5D10F22190705D504A94D19B0
:10F558002D2105F8101C951C13F0010F0CBF4FF05E
:10F56800200B4FF0300B9B072F4604D508E0584678
:10F57800FFF721FF4F46474507F10109F7D34F46EB
:10F58800013D1DF80500FFF716FF002DF8D103E037
:10F598002020FFF710FF01374745F9D336E705B0BC
:10F5A800BDE8F08F70B5064D0C462E68286001E066
:10F5B800FFF701FF14F8010B0028F9D12E6070BD88
:10F5C800CC3B00200FB407B504A951F8040B0191F6
:10F5D800FFF714FFBDE80E4004B070470EB417B52E
:10F5E80005A9084C51F8043B206018460191FFF723
:10F5F80005FF2268002313702360BDE81E4003B096
:10F60800704700BFD80D00200EB433B505A9074CCC
:10F6180051F8043B2568206018460191FFF7EEFE7B
:10F628002560BDE83C4003B0704700BFCC3B0020DC
:10F6380070B51E4604461C481546FFF7C3FF022E48
:10F648001FD0042E25D0012E2AD105E0A15D174830
:10F65800FFF7B8FF013600E00026AE42F6DB2020B7
:10F66800FFF7A9FE002609E0A05DA0F12003DBB2A8
:10F678005E2B88BF2E20FFF79EFE0136AE42F3DBDD
:10F688000EE034F8021B0A48FFF79CFF013DF8D151
:10F6980006E054F8041B0748FFF794FF013DF8D132
:10F6A8000A20BDE8704086E6C3B20508CAB205085C
:10F6B800D0B20508D6B2050808B501214FF480700C
:10F6C80001F07CFA4FF480700021BDE8084001F099
:10F6D80075BA43680A6823F0407323F480731343B0
:10F6E8000A7943EA02234360CA680B6930B51A43B2
:10F6F80084688D68084B2A43234013434A7943EAB8
:10F70800420383600B7DC26A013B22F47002DBB2C4
:10F7180042EA0353C36230BDFDF7FFC00023036014
:10F72800037143718360C3600361012303757047EC
:10F73800074A084B516810B50B4090E81200214366
:10F748008468C068214301430B43536010BD00BF68
:10F7580000230140E030FCFF002303604360836026
:10F76800C3607047836811B143F0010301E023F0DF
:10F77800010383607047436823F4400323F4007354
:10F788000B4343607047416282627047436823F0CD
:10F798001F030B4343607047044B5A6810B142F48F
:10F7A800000201E022F400025A6070470023014081
:10F7B800044B5A6810B142F4800201E022F480023E
:10F7C8005A60704700230140092970B50CB20CD962
:10F7D80004EB44041E3CC6680725A54026EA050537
:10F7E800A34045EA0304C4600AE0066904EB440444
:10F7F8000725A54026EA050513FA04F42C430461FD
:10F80800062A0CD80523013A5A43446B1F23934018
:10F8180024EA0303914043EA0102426370BD0C2AC3
:10F8280012B20CD802EB8202233A046B1F239340D6
:10F8380024EA0303914043EA0102026370BD02EB2C
:10F848008202413AC46A1F23934024EA0303914089
:10F8580043EA0102C26270BD836843F0804383605B
:10F8680070478068C0F380507047836811B143F4D3
:10F87800806301E023F4806383607047836811B17B
:10F8880043F0020301E023F00203836070474368FA
:10F89800013923F4604343EA4133436070474368C6
:10F8A80011B143F4006301E023F40063436070473F
:10F8B800C06C80B27047014B18687047082301403C
:10F8C800836811B143F4807301E023F4807383608B
:10F8D8007047836811B143F4007301E023F40073A7
:10F8E80083607047044B5A6810B142F4005201E03B
:10F8F80022F400525A60704700230140092970B56C
:10F908000CB20CD904EB44041E3CC6680725A5407C
:10F9180026EA0505A34045EA0304C4600AE006692F
:10F9280004EB44040725A54026EA050513FA04F468
:10F938002C430461836BC3F30154121B0232D2B20D
:10F9480002EB82021F24944023EA040391400B43F4
:10F95800836370BD836B013923F4401343EA015379
:10F968008363704782B0002301930190019BCB18F9
:10F978000193019B1A6002B07047836823F47023D7
:10F988000B4383607047836823F440130B43836001
:10F998007047836843F48003836070478068C0F3CE
:10F9A80080507047436811B143F4806301E023F449
:10F9B800806343607047436811B143F4805301E0AA
:10F9C80023F480534360704782B000230193019071
:10F9D800019B28335B180193019B186880B202B021
:10F9E80070470123C9B213FA01F143680AB11943F8
:10F9F80001E023EA010141607047036819420CBF26
:10FA0800002001207047C9430160704743680068BF
:10FA180010EA112007D00122C9B212FA01F11942E5
:10FA28000CBF0020012070476FEA11210160704768
:10FA3800036823F0010303600023036043608360CD
:10FA4800C3600361212343612C4B98421CD02C4B8B
:10FA5800984220D02B4B984225D02B4B98422AD045
:10FA68002A4B98422FD02A4B984233D0294B9842A0
:10FA780037D0294B984204D14FF03D5243F8AC2C73
:10FA88007047264B984203D13D2243F8082C704713
:10FA9800234B984204D14FF4746243F8202C7047EA
:10FAA800204B984204D14FF4741243F8382C704715
:10FAB8001D4B984204D14FF0746243F8502C7047A4
:10FAC8001A4B984203D11A4A43F8642C7047194BD1
:10FAD800984203D1184A43F87C2C7047174B984238
:10FAE80003D1174A43F8942C7047164B984204BF29
:10FAF8004FF03D5243F8AC2C704700BF10600240F5
:10FB08002860024040600240586002407060024035
:10FB180088600240A0600240B86002401064024061
:10FB28002864024040640240586402407064024005
:10FB38003D00002088640240400F0020A06402407D
:10FB480000003D20B86402400268134B10B5134012
:10FB5800CC680A6822434C6922438C692243CC69E9
:10FB680022430C6A22434C6A22438C6A22434C6B20
:10FB780022438C6B22431343036042690C6BCB6AAC
:10FB880022F007022343134343610B6943604B6828
:10FB980083608B68C36010BD3F801CF00023036046
:10FBA80043608360C360036143618361C36103622F
:10FBB80043628362C362036343638363704703687A
:10FBC80011B143F0010301E023F001030360704722
:10FBD800036811B143F4004301E023F400430360D8
:10FBE8007047036811B143F0200301E023F02003BC
:10FBF8000360704741607047406880B2704703688F
:10FC080012B143F4002301E023F4002303600161EF
:10FC18007047036811B143F4802301E023F4802383
:10FC2800036070470AB101617047C160704700689E
:10FC3800C0F3C0407047006800F001007047406999
:10FC480000F0380070470A4A0A4B10B50A4CA04227
:10FC580088BF13468A004CBF5B681B6821F0F021FF
:10FC680021F0821119420CBF0020012010BD00BFF5
:10FC780000640240006002400F64024010B5084B67
:10FC8800084A094CA04288BF134611F0005F21F0D2
:10FC9800F02121F0821114BFD960996010BD00BF16
:10FCA80000600240006402400F6402400B0607D562
:10FCB800436912B143F0800301E023F080034361FC
:10FCC800802909D001F01E01036812B119430160AF
:10FCD800704723EA010101607047124B124A10B5C0
:10FCE800124CA0428CBF14461C4621F0F02323F08E
:10FCF800C3132BB1026802F01E0202EAD12202E00D
:10FD0800426902F0800288004CBF6368236821F0D2
:10FD1800F02121F08210184002D0101C18BF0120D9
:10FD280010BD00BF00600240006402400F64024042
:10FD380010B5084B084A094CA04288BF134611F079
:10FD4800005F21F0F02121F0821114BFD960996081
:10FD580010BD00BF00600240006402400F64024012
:10FD6800044B00221A605A609A60DA60024A5A61AB
:10FD7800704700BF003C0140FFFF7F00837910B54A
:10FD8800002B29D01A4B01681C68CA4314401C6018
:10FD98005C6822405A60027902F1804202F59E3284
:10FDA80014682143116002689C68D1430C409C6030
:10FDB800DC682140D9604179102906D1996811433E
:10FDC8009960D9680A43DA6010BD01F1804303F5F0
:10FDD8009E3319680A4308E00379016803F18043F8
:10FDE80003F59E331A6822EA01021A6010BD00BFAB
:10FDF800003C014000230C220360037142718371AF
:10FE08007047024B1A6902431A617047003C01406F
:10FE1800034B5B6918420CBF00200120704700BFEC
:10FE2800003C0140014B5861704700BF003C014055
:10FE3800054B1A685B69034004D010420CBF0020D0
:10FE48000120704718467047003C0140014B58613B
:10FE5800704700BF003C01404FF0204318B943F2FF
:10FE6800DB021A6003E043F2D20243F820204FF08D
:10FE78002042411C6FF0704342F8213002F5827233
:10FE880042F82030704770B584684568C368C16A15
:10FE9800026825431D4303691D4343691D43836964
:10FEA8001D43C3691D43036A1D43436A1D43836A97
:10FEB8001D43036B0D431D434FF02043082C43F8AB
:10FEC800225005D153F8224044F0400443F8224020
:10FED800436B9E691D6835435E6845EA06159E6852
:10FEE80045EA0625DE6845EA06451E695B6945EA76
:10FEF8000655541C45EA03654FF02043B1F5804F81
:10FF080043F8245010D1836B9869196801435868E5
:10FF180041EA0011986841EA002118695B6941EAE1
:10FF2800005141EA036101E06FF07041014B43F871
:10FF3800221070BD040100A0022242604FF48052DA
:10FF48004262416B4FF4005210B5826200230F22C7
:10FF5800FF2403608360C360036143618361C361FD
:10FF68000362C36203630A604A608C60CA600A6104
:10FF78004A618B61816B0A604A608C60CA600A6161
:10FF88004A618B6110BD4FF0204321B153F8202006
:10FF980042F0010203E053F82010024A0A4043F8F5
:10FFA80020207047FEFF0F0010280CBF064B074BA0
:10FFB8004FF040024FF0180119605A604FF0FC32C0
:10FFC8009A60DA60704700BF600000A0800000A05F
:10FFD80030B5836844681C43C36844F008041C4374
:10FFE80003691C43436944EA4324836944EA43346C
:08FFF800C36999685A68090405
:020000040801F1
:1000000041EA02211A68DB68114341EA0361036A8D
:100010009A685D68120442EA05221D68DB682A437B
:1000200042EA03620368102B0CBF034B034B1C60B6
:100030009960DA6030BD00BF600000A0800000A0C1
:1000400010230360C269002343608360C3600361BF
:1000500043618361FC23136053609360D360026A41
:10006000136053609360D360704741B110280CBF98
:10007000074B084B1A6842F004021A6070471028B8
:100080000CBF034A034A044B11680B4013607047CE
:10009000600000A0800000A0FBFF0F0041B110280D
:1000A0000CBF084B084B1A6842F040021A607047B8
:1000B00010280CBF034A044A044B11680B4013601C
:1000C000704700BF600000A0800000A0BFFF0F00CD
:1000D000102802D1024B58697047024B586970478B
:1000E000600000A0800000A0054B18221A600022CA
:1000F0005A604FF0FC329A60DA601A61704700BFB4
:10010000A00000A00268436842F0100242EA4322C5
:10011000836842EA4332144B10B51A60C268916892
:100120005468090441EA04211468D268214341EA71
:1001300002629A60026991685468090441EA0421E4
:100140001468D268214341EA0262DA604269916828
:100150005068090441EA00211068D268014341EA6D
:1001600002621A6110BD00BFA00000A0C268002397
:10017000036043608360FC23136053609360D3602B
:100180000269136053609360D360426913605360E7
:100190009360D3607047054B18B11A6842F00402AF
:1001A00002E01968024A0A401A607047A00000A0E5
:1001B000FBFF0F0062B1102801D10E4B03E0B0F538
:1001C000807F03D10C4B5A68114311E00B4BFAE7C7
:1001D000102804D1074B5A6822EA010108E0B0F563
:1001E000807F0CBF044B054B5A686FEA0101114038
:1001F00059607047600000A0800000A0A00000A02F
:10020000102801D1064B04E0B0F5807F0CBF054BF0
:10021000054B5B680B420CBF00200120704700BFFC
:10022000600000A0800000A0A00000A0102804D161
:10023000074B5A6822EA010108E0B0F5807F0CBF45
:10024000044B054B5A686FEA010111405960704731
:10025000600000A0800000A0A00000A0102801D134
:10026000084B04E0B0F5807F0CBF074B074B5B6881
:1002700013EA010004D013EAD1010CBF00200120D1
:10028000704700BF600000A0800000A0A00000A098
:10029000102804D1084B5A6822EAD10109E0B0F5D0
:1002A000807F0CBF054B064B5A684FEAD10122EA0A
:1002B00001015960704700BF600000A0800000A0ED
:1002C000A00000A008B52C4B984205D101200146A2
:1002D00000F048FC012048E0284B984205D102205C
:1002E000012100F03FFC02203FE0254B984205D160
:1002F0000420012100F036FC042036E0214B984216
:1003000005D10820012100F02DFC08202DE01E4B16
:10031000984205D11020012100F024FC102024E097
:100320001A4B984205D12020012100F01BFC20200F
:100330001BE0174B984205D14020012100F012FC30
:10034000402012E0134B984205D18020012100F09B
:1003500009FC802009E0104B98420BD14FF48070CB
:10036000012100F0FFFB4FF480700021BDE8084040
:1003700000F0F8BB08BD00BF0000024000040240CE
:1003800000080240000C024000100240001402402D
:1003900000180240001C0240002002402DE9F047F6
:1003A0000023D1F800801A464FF0010C03270CFA05
:1003B00002F404EA0805A5422ED1066817FA03F4F0
:1003C000E443264006600E79D0F8009006FA03FA5E
:1003D000013E4AEA0909012EC0F8009014D8866847
:1003E00091F8059026408660866809FA03F949EA83
:1003F00006068660466826EA050545608D794668EA
:100400009540ADB235434560C5682C40C460CC7999
:10041000C5689C402C43C46001320233102AC6D107
:10042000BDE8F0874FF6FF7303600023037143714B
:100430008371C371704782B04FF480330193019B85
:100440000B430193019BC361C161019BC361C369FC
:100450000193C369019302B07047036919420CBF4D
:10046000002001207047006980B27047436919423B
:100470000CBF002001207047406980B270470183A3
:100480007047418370470AB10183704741837047C9
:100490004161704743694B404361704701F0070376
:1004A000C908083130B59B0050F821500F249C40FA
:1004B00025EA040440F8214050F8214012FA03F3E1
:1004C0001C4340F8214030BD08B5134B984207D17A
:1004D0004FF40010012100F069FB4FF4001014E00C
:1004E0000E4B984207D14FF48000012100F05EFBD3
:1004F0004FF4800009E00A4B98420BD14FF4000002
:10050000012100F053FB4FF400000021BDE808403A
:1005100000F04CBB08BD00BF005400400058004034
:10052000005C00407FB50446868868460D4600F0B2
:100530006DFA02992C482B6826F03F063604B1FB71
:10054000F0F0360C80B20643A680228822F0010229
:100550001204120C2280254A93420AD85B00B1FB98
:10056000F3F301309BB280B22084032B98BF0423A5
:1005700021E0EE884BF6FF72964205D103225343E9
:10058000B1FBF3F39BB206E019225343B1FBF3F343
:100590009BB243F480431A054FF4967208BF43F0B0
:1005A000010350434FF47A7290FBF2F0013080B2B5
:1005B00043F400432084A38323886989AA889BB2DB
:1005C00043F001032380238823F4816323F0020393
:1005D0001B040A431B0C13439BB223802A89AB895B
:1005E00013439BB223817FBD40420F00A0860100D0
:1005F00041F288330360002383804BF6FF7203814E
:1006000043814FF48043C28083817047038819B1CE
:100610009BB243F0010303E023F001031B041B0C16
:1006200003807047038819B19BB243F4807303E0E1
:1006300023F480731B041B0C03807047038819B1DB
:100640009BB243F4007303E023F400731B041B0C00
:100650000380704712B141F0010101E001F0FE0199
:1006600001827047038819B19BB243F4806303E0B1
:1006700023F480631B041B0C0380704783899BB2A7
:1006800001F0FE0123F0FE030B4383817047838951
:1006900019B19BB243F0010303E023F001031B04F3
:1006A0001B0C83817047038819B19BB243F0400350
:1006B00003E023F040031B041B0C038070470388F6
:1006C00029B16FEA43436FEA53439BB201E05B04F5
:1006D0005B0C03807047038819B99BB243F0800319
:1006E00003E023F080031B041B0C03807047B1F56B
:1006F000804F838B04D023F480431B041B0C02E047
:100700009BB243F4804383837047B1F5006F038845
:1007100003D19BB243F4006303E023F400631B04A2
:100720001B0C03807047B1F5005F038803D19BB2B7
:1007300043F4005303E023F400531B041B0C038019
:100740007047038819B19BB243F0100303E023F014
:1007500010031B041B0C0380704701827047008A42
:10076000C0B27047038819B19BB243F4805303E0D1
:1007700023F480531B041B0C03807047B1F5006FFA
:10078000038803D19BB243F4006303E023F40063C6
:100790001B041B0C03807047038819B19BB243F004
:1007A000200303E023F020031B041B0C038070478D
:1007B000008BC0F307207047838819B19BB243F4C4
:1007C000006303E023F400631B041B0C8380704769
:1007D000838819B19BB243F4805303E023F4805320
:1007E0001B041B0C8380704782B00023019301908F
:1007F000019BCB180193019B188880B202B070470F
:1008000083889BB20AB1194301E023EA0101818088
:100810007047838A008B9BB243EA0040084020F077
:100820007F40431A584240EB03007047838A008B95
:100830009BB243EA004020F07F40704782B0002323
:10084000009301930B0F01900093009B21F07F41D7
:1008500013B1019B143302E0019B090C183301937F
:10086000019B1B6819420CBF0020012002B0704799
:10087000C94389B2818270478388808A80B20840E8
:100880009BB206D001F0E06113EA11410CBF0020D9
:1008900001207047C94389B2818270470A4B1A68A8
:1008A00042F001021A6000229A60196821F08471F6
:1008B00021F48031196005495960196821F48021BB
:1008C0001960DA60704700BF003802401030002421
:1008D000024B00221A701870704700BF02380240A5
:1008E000034B1A6822F0F80242EAC0021A6070470D
:1008F00000380240014B1860704700BF00004742BB
:10090000064B002201281A701A7002D0042804D164
:1009100001E01870704705221A7070477038024065
:10092000014B1860704700BF800E4742014341EA07
:10093000821200995B08013B42EA016141EA0341EE
:10094000014B5960704700BF00380240014B1860EE
:10095000704700BF600047428001034B40EA0171CD
:10096000C3F88410704700BF00380240014B186084
:10097000704700BF68004742014B1860704700BFD6
:100980004C004742034B9A6822F0EC6202430A4350
:100990009A60704700380240034B9A6822F0784210
:1009A00002430A439A60704700380240034B9A683A
:1009B00022F0030202439A60704700BF00380240F1
:1009C000024B986800F00C00704700BF00380240EE
:1009D000034B9A6822F0F00202439A60704700BF0E
:1009E00000380240034B9A6822F4E05202439A60B6
:1009F000704700BF00380240034B9A6822F46042FF
:100A000042EAC0029A607047003802401E4B9A6862
:100A100002F00C02042A10B503D0082A03D01B4BA5
:100A200018E01B4B16E059685A6811F4800F59689A
:100A300014BF174B154B02F03F02B3FBF2F3124AFF
:100A40005268C2F30142C1F3881101324B43520094
:100A5000B3FBF2F30C4903608B680E4A0468C3F3DE
:100A60000313D35C34FA03F343608C68C4F3822429
:100A7000145D33FA04F484608968C1F34231525C36
:100A8000D340C36010BD00BF003802400024F40012
:100A900000127A003403002000F44073B3F5407F65
:100AA000084B08D1996820F0704221F4F81122F423
:100AB00040720A439A601A6F000542EA10501867A4
:100AC000704700BF00380240014B1860704700BFFC
:100AD0003C0E4742014B1860704700BF400E474232
:100AE000014B1860704700BF5C014742044B1A6B12
:100AF00009B1104301E022EA00001863704700BF0B
:100B000000380240044B5A6B09B1104301E022EA5D
:100B100000005863704700BF00380240044B9A6BD6
:100B200009B1104301E022EA00009863704700BF5A
:100B300000380240044B1A6C09B1104301E022EA6C
:100B400000001864704700BF00380240044B5A6C24
:100B500009B1104301E022EA00005864704700BF69
:100B600000380240044B1A6909B1104301E022EA3F
:100B700000001861704700BF00380240044B5A69FA
:100B800009B1104301E022EA00005861704700BF3C
:100B900000380240044B9A6909B1104301E022EA8F
:100BA00000009861704700BF00380240044B1A6A89
:100BB00009B1104301E022EA00001862704700BF4B
:100BC00000380240044B5A6A09B1104301E022EA9E
:100BD00000005862704700BF00380240044B1A6D95
:100BE00009B1104301E022EA00001865704700BF18
:100BF00000380240044B5A6D09B1104301E022EA6B
:100C000000005865704700BF00380240044B9A6DE1
:100C100009B1104301E022EA00009865704700BF67
:100C200000380240044B1A6E09B1104301E022EA79
:100C300000001866704700BF00380240044B5A6E2F
:100C400009B1104301E022EA00005866704700BF76
:100C500000380240044B1A7809B1104301E022EA3F
:100C600000001870704700BF0D3802404309012B87
:100C7000074A01D1136803E0022B0CBF136F536FB7
:100C800000F01F0033FA00F000F00100704700BFD1
:100C90000038024007B5002301933120FFF7E6FF3B
:100CA000019B01330193019BB3F5A06F01D0002894
:100CB000F3D03120FFF7DAFF003018BF01200EBD5E
:100CC000024B5A6F42F080725A67704700380240F8
:100CD000034BDB6818420CBF00200120704700BFA7
:100CE00000380240014B1870704700BF0E380240B8
:100CF00008B5154B98420BD101214FF48050FFF7F6
:100D000061FF4FF480500021BDE80840FFF75ABF53
:100D10000E4B984207D14FF480400121FFF746FF68
:100D20004FF4804009E00A4B98420BD14FF4004049
:100D30000121FFF73BFF4FF400400021BDE80840D0
:100D4000FFF734BF08BD00BF00300140003800404D
:100D5000003C00400B88028810B54C8823438C88E7
:100D60002343CC8823430C8923434C8923438C8918
:100D70002343CC8902F44152234313439BB20380A3
:100D8000838B23F400631B041B0C83830B8A038275
:100D900010BD838B23F47B6323F00F031B041B0C18
:100DA0008383022303848B68F0B5858B022BADB25D
:100DB00038D0294A8E889468002E14BF0226012656
:100DC000240203D5946824F400049460D2F884408B
:100DD000D2F884705268DFF884C002F03F02BCFB96
:100DE000F2F2C4F388145443C7F30272B4FBF2F472
:100DF000CA88B2F5007F4FF00A0201D1240A02E04E
:100E00007601B4FBF6F46243B2FBF3F305330A2236
:100E10009BB2B3FBF2F303F001021202C3F34F03E0
:100E200092B200E000229C1EA4B2FE2C28BF002239
:100E3000CC8828BF0223134323439BB203840B882F
:100E40004A882B4343F4006313438A8813438A89F7
:100E500013439BB28383F0BD0038024000127A0036
:100E60000023038043808380C38003814381838187
:100E7000C38107230382704700230222038043803B
:100E80008380C380826083817047038819B19BB2DD
:100E900043F0400303E023F040031B041B0C0380DA
:100EA0007047838B19B19BB243F4806303E023F452
:100EB00080631B041B0C83837047038823F4006347
:100EC0001B041B0C038003889BB20B4303807047F9
:100ED000B1F5804F038803D19BB243F4804303E014
:100EE00023F480431B041B0C038070474FF6FF6301
:100EF0009942038803D09BB243F4807303E023F448
:100F000080731B041B0C03807047838819B19BB24C
:100F100043F0040303E023F004031B041B0C838051
:100F20007047838819B19BB243F0100303E023F0AC
:100F300010031B041B0C83807047838B23F47B639B
:100F400023F00F031B041B0C8383022303840B88F1
:100F5000828BB3F5007F10B592B205D0002B0CBF89
:100F60004FF48073002301E04FF480734C882243D8
:100F70008C88898942F4006222430A4392B2134367
:100F8000838310BD808980B2704781817047038858
:100F900019B19BB243F4005303E023F400531B0444
:100FA0001B0C0380704703889BB243F4805303807B
:100FB0007047012902D0008B80B27047808A80B2CE
:100FC0007047008A80B2704783889BB20AB1194388
:100FD00001E023EA010181807047090901238B4068
:100FE0009BB21AB1828892B2134303E0828892B214
:100FF00022EA030383807047038919420CBF002053
:1010000001207047C94389B20181704710B58488B7
:101010000089012301F00F0280B213FA02F210409E
:10102000A4B205D009098B401C420CBF002001204E
:1010300010BD01F00F0101238B40DB439BB2038104
:10104000704700BF08B501214FF48040FFF7BAFD9B
:101050004FF480400021BDE80840FFF7B3BD014BCD
:10106000186070470038014001F0030289080A4BFC
:10107000023130B5920053F821500F24944025EAF4
:10108000040443F8214053F8214010FA02F21443BB
:1010900043F8214030BD00BF00380140014B1860CB
:1010A000704700BFDC002742014B1860704700BF4B
:1010B00000042742024B186AC0F30020704700BFAB
:1010C0000038014030B5048C24F001042404240CC1
:1010D0000484058B048CADB2A4B225F0F30515434E
:1010E00024F00A0445EA031544F00104ADB20C43B0
:1010F0000583048430BD30B5048C24F0100424042E
:10110000240C0484048B058C24F44074ADB22405B3
:10111000240D25F0A00544EA022445F0100544EA18
:10112000033445EA0115A4B2ADB20483058430BD91
:1011300008B5474B984205D101200146FFF742FD13
:1011400001203DE0B0F1804F05D101200146FFF7BD
:101150002DFD012076E03F4B984205D10220012170
:10116000FFF724FD02206DE03B4B984205D104209F
:101170000121FFF71BFD042064E0384B984205D1A4
:1011800008200121FFF712FD08205BE0344B984254
:1011900005D110200121FFF709FD102052E0314B4D
:1011A000984205D120200121FFF700FD202049E0D1
:1011B0002D4B984209D102200121FFF703FD0220A7
:1011C0000021BDE80840FFF7FDBC284B984207D13D
:1011D0004FF480300121FFF7F5FC4FF48030EFE74A
:1011E000234B984207D14FF400300121FFF7EAFC6E
:1011F0004FF40030E4E71F4B984207D14FF48020B2
:101200000121FFF7DFFC4FF48020D9E71A4B984209
:1012100005D140200121FFF7C9FC402012E0174B07
:10122000984205D180200121FFF7C0FC802009E011
:10123000134B98420BD14FF480700121FFF7B6FC9D
:101240004FF480700021BDE80840FFF7AFBC08BD37
:10125000000001400004004000080040000C004075
:101260000010004000140040000401400040014014
:10127000004401400048014000180040001C0040AC
:10128000002000401C4A038890429BB212D002F515
:10129000806290420ED0B0F1804F0BD0A2F5803228
:1012A000904207D002F58062904203D002F580623E
:1012B000904203D14A8823F0700313430F4A9042AF
:1012C00008D002F58062904204D023F440730A896A
:1012D0009BB2134303804B68C3620B880385064BA4
:1012E000984203D003F58063984201D18B7A03863C
:1012F00001238382704700BF0000014000100040BE
:101300004FF0FF33436000230380038143808372E7
:101310007047018582827047038823F070031B04A5
:101320001B0C0B430380704741627047C1627047DA
:10133000406A7047008D80B27047038819B19BB234
:1013400043F0020303E023F002031B041B0C0380A1
:101350007047038819B19BB243F0040303E023F004
:1013600004031B041B0C03807047038819B19BB254
:1013700043F0800303E023F080031B041B0C038075
:101380007047038823F008031B041B0C03800388A9
:101390009BB20B4303807047038823F440731B0404
:1013A0001B0C038003889BB20B43038070470388A8
:1013B00019B19BB243F0010303E023F001031B04C6
:1013C0001B0C03807047038C23F001031B041B0CD0
:1013D000038470B5038C8488028B0D884E8822F0BC
:1013E00073021204120C2A438D8923F002031B049A
:1013F00035431B0CADB22B430E4DA842A4B203D013
:1014000005F58065A8420ED1CD894E8A23F00803E8
:101410002B438D8823F004032B430D8A354324F49A
:101420004074ADB22C43848002838A684263038493
:1014300070BD00BF00000140038C23F010031B04AB
:101440001B0C0384038C828830B5048B0D8824F434
:10145000E6442404240C23F0200344EA05241B045E
:101460008D891B0C43EA05134D8843EA0513134D80
:10147000A84292B2A4B29BB203D005F58065A842FF
:1014800015D1CD8923F080039BB243EA05134FF6B3
:10149000BF751D408B8845EA03130D8A22F4406214
:1014A00042EA85024D8A42EA85029BB292B282806C
:1014B0008A6804838263038430BD00BF000001405A
:1014C000038C23F480731B041B0C0384038C82881D
:1014D00030B5848B0D8824F073042404240C23F489
:1014E00000731B042C438D891B0C43EA05234D8894
:1014F00043EA0523124DA84292B29BB203D005F5F0
:101500008065A84215D1CD8923F400639BB243EADC
:1015100005234FF6FF351D408B8845EA03230D8ACE
:1015200022F4405242EA05124D8A42EA05129BB269
:1015300092B282808A688483C263038430BD00BF14
:1015400000000140038C23F480531B041B0C038414
:10155000038C30B58488828B0D8822F4E642120415
:10156000120C23F4005342EA05221B048D891B0C44
:1015700043EA05334D8843EA05330B4DA842A4B234
:1015800092B29BB203D005F58065A84205D10D8AC1
:1015900024F4804444EA8514A4B2848082838A6857
:1015A0000264038430BD00BF0000014000230380BB
:1015B0004380838083608381C38103824382704739
:1015C00030B5058C0124ADB28C4025EA040400F14D
:1015D0001803048409B1082907D149084FF68F7010
:1015E000CC582040C850C8580AE00439C1F34E0115
:1015F00048F6FF70CC582040C8501202C85892B22A
:101600000243CA5030BD4163704781637047C16374
:10161000704701647047038B23F070031B041B0C9D
:101620000B4303837047038B23F4E0431B041B0C21
:1016300043EA01239BB203837047838B23F070033B
:101640001B041B0C0B4383837047838B23F4E04301
:101650001B041B0C43EA01239BB283837047038B5B
:1016600023F008031B041B0C0B4303837047038BFD
:1016700023F400631B041B0C43EA01239BB2038386
:101680007047838B23F008031B041B0C0B438383DD
:101690007047838B23F400631B041B0C43EA012374
:1016A0009BB283837047038B23F004031B041B0C42
:1016B0000B4303837047038B23F480631B041B0CD1
:1016C00043EA01239BB203837047838B23F0040317
:1016D0001B041B0C0B4383837047838B23F48063B1
:1016E0001B041B0C43EA01239BB283837047038BCB
:1016F00023F080031B041B0C0B4303837047038BF5
:1017000009025B0441EA53439BB203837047838B16
:1017100023F080031B041B0C0B4383837047838BD4
:1017200009025B0441EA53439BB283837047038CF5
:1017300023F002031B041B0C0B4303847047038C30
:1017400023F008031B041B0C0B4303847047038C1A
:1017500023F020031B041B0C43EA01139BB20384F8
:101760007047038C23F080031B041B0C43EA011316
:101770009BB203847047038C23F400731B041B0C7F
:1017800043EA01239BB203847047038C23F4006374
:101790001B041B0C43EA01239BB203847047038C98
:1017A00023F400531B041B0C43EA01339BB2038454
:1017B000704710B5048C01238B40A4B224EA0303C4
:1017C0000384038C12FA01F10B439BB2038410BD16
:1017D00010B5048C04238B40A4B224EA03030384D1
:1017E000038C12FA01F10B439BB2038410BD00235A
:1017F0000122038043808280C38003817047406B55
:101800007047806B7047C06B7047006C7047038BEC
:1018100023F00C031B041B0C0383038B9BB20B43B1
:1018200003837047038B23F440631B041B0C038367
:10183000038B9BB243EA01239BB203837047F8B545
:101840000C464988A288B4F800E02389054600299F
:101850000CBF02270027012A14BF01260226BEF171
:10186000000F10D1FFF72EFC2846E188FFF7CFFFCD
:101870002846394632462389FFF73DFCE188284651
:10188000BDE8F840CEE7FFF736FC2846E188FFF7D1
:10189000C9FF2846394632462389FFF713FCE18801
:1018A0002846BDE8F840B2E7838B23F00C031B0405
:1018B0001B0C8383838B9BB20B4383837047838B87
:1018C00023F440631B041B0C8383838B9BB243EA8A
:1018D00001239BB283837047F8B50D460B88AA8815
:1018E000498804463BB92B89FFF7ECFBE988204681
:1018F000BDE8F8408BE7042B07D12B89FFF7FBFBF2
:10190000E9882046BDE8F8408CE7082BB5F808C008
:10191000078C1DD127F480773F043F0C0784868B0A
:10192000038CB6B29BB226F0F30623F4206346EA9A
:101930000C1C43EA01211FFA8CFC89B24CEA02021A
:1019400041F4807182830184E988BDE8F840ABE707
:1019500027F480573F043F0C0784868B038C26F4C2
:10196000407623F4005336055B04360D5B0C46EAE3
:10197000022243EA013342EA0C329BB2E98892B276
:1019800043F4805382830384BDE8F84097E74A8894
:101990000B8813438A881343CA8813430A89134365
:1019A0004A8913438A8913439BB2A0F84430704795
:1019B0000023038043808380C3800381438183812C
:1019C0007047B0F8443029B16FEA43436FEA53439C
:1019D0009BB201E05B045B0CA0F844307047838845
:1019E00019B19BB243F0040303E023F004031B048A
:1019F0001B0C83807047838819B19BB243F00103AD
:101A000003E023F001031B041B0C838070478389D0
:101A10009BB20AB1194301E023EA010181817047B9
:101A200081827047038A19420CBF00200120704751
:101A3000C94389B201827047038A828911EA03008F
:101A400092B203D011420CBF002001207047C9435D
:101A500089B2018270470A43A0F848207047838901
:101A60009BB20AB1194301E023EA01018181704769
:101A7000838819B19BB243F0080303E023F0080305
:101A80001B041B0C83807047038923F007031B048E
:101A90001B0C03817047038923F070031B041B0C8C
:101AA0000B43038103899BB243F007030381704713
:101AB00038B50D4611460122602D044602D1FFF7CC
:101AC0001AFB01E0FFF7FEFA238923F070031B04E1
:101AD0001B0C1D43258123899BB243F007032381FF
:101AE00038BD038923F070031B041B0C0B430381D7
:101AF0007047838823F070031B041B0C838083884A
:101B00009BB20B4383807047038923F007031B04B8
:101B10001B0C038103899BB20B430381704703892C
:101B200023F080031B041B0C038103899BB20B432E
:101B30000381704710B50489E4B20C43144344EAAE
:101B40000324A4B2048110BD10B50446FFF7F2FFD0
:101B500023899BB243F48043238110BD10B5044612
:101B6000FFF7E8FF238923F077031B041B0C43F0E6
:101B70007703238110BD70B50489068B058C26F48C
:101B80004076ADB226F0030624F00704360425F0B3
:101B900022052404360C1543240C46F4807645EACD
:101BA0000315214346F00106ADB201810683058489
:101BB00070BD838819B19BB243F0800303E023F02A
:101BC00080031B041B0C83807047A0F850107047E3
:101BD00008B5234B984205D110200121FEF7F2FFF2
:101BE000102037E01F4B984207D14FF400300121FD
:101BF000FEF7DCFF4FF4003009E01B4B98420BD19D
